:020000040800F2
:100000000050002099A2000839A30008918D000833
:1000100039A3000839A3000839A300080000000034
:1000200000000000000000000000000039A30008EC
:1000300039A300080000000039A300082149000886
:1000400039A3000839A3000839A3000839A3000820
:1000500039A3000839A3000839A3000839A3000810
:1000600039A3000839A3000839A3000839A3000800
:1000700039A3000839A30008CD7B000839A3000884
:1000800039A3000839A3000839A3000839A30008E0
:1000900039A3000839A3000839A3000839A30008D0
:1000A00039A30008017A000839A30008117A000872
:1000B000F5790008E5790008D5790008D520000811
:1000C000D9200008CF200008D320000839A3000859
:1000D00039A30008C57B0008BD7B000839A30008D0
:1000E0003149000839A3000839A3000800000000C6
:1000F0000000000000000000000000000000000000
:0C01000000000000000000005FF808F1A3
:10010C002DE9F04F664B674C97B02360002363607A
:10011C0007F064FA18B907F083FA04F0E1FF05F070
:10012C00ADF8614A614D1378614F43F001031370D0
:10013C00002309930A930B934FF4E0130C932B6851
:10014C00B87B43F480332B60AB6943F01003AB6195
:10015C002B6803F400330A93099B013309930A9B20
:10016C001BB9099BB3F5A06FF2D12B684F4913F45F
:10017C00003301D0022315E00A6842F001020A6044
:10018C0009932B6803F002030A93099B013309932B
:10019C000A9B1BB9099BB3F5A06FF2D12B689B0787
:1001AC0034D501230B93434B43491A683F4E42F01D
:1001BC0010021A601A6822F003021A601A6842F0E0
:1001CC0002021A606B686B606B686B606B6843F45F
:1001DC0080636B60394B1A68043B22F070425A60A2
:1001EC00374A1160696821F47C116960596841F0E3
:1001FC0000415960D96821F40041D9604FF4E011F5
:10020C000C910B990293012901D118E0FEE7022908
:10021C0019D168B10C9BB3F5801F02D14FF4A01318
:10022C0005E00C9BB3F5E01F02D14FF400130C93C7
:10023C000C996B680B4343F480336B6003E0736879
:10024C0043F4601373602B6843F080732B60296850
:10025C00164B8E01FBD5596821F003015960596882
:10026C0041F0020159606B68104903F00C03082B34
:10027C00F9D14B68DFF8509003F00C03042B03D03A
:10028C00082B03D00C4B27E0136825E04B6848681B
:10029C00C3F38343C00303F1020317D4094A1AE0E2
:1002AC003D4A0008A8030020EC1600200010024074
:1002BC00E80900200020024000127A0004100140DE
:1002CC002400002000093D00380000204968126815
:1002DC00890348BF52085343C9F800306B68BD4AC4
:1002EC00C3F30313D15CD9F800309046CB40C9F866
:1002FC000030029BDFF820B39B6816AE13F4004F5E
:10030C00B54B14BF022201221A70B44B4FF0000AF5
:10031C00CBF80C30AB69B24843F00103AB616B6AAC
:10032C00A3606B6A43F080736B62AB6943F01C0390
:10033C00AB614FF6FF7326F8183D31468DF842A09D
:10034C0001F096F9A748314601F092F93146A648DA
:10035C0001F08EF9A54A3046536843F000735360A0
:10036C0005F094FC109BA24AB646B3FBF2F3A14AEB
:10037C00DFF8A8C21360A04B4FF47A72C3F800A048
:10038C00D9F80030DFF89892B3FBF2F39B4A013BAB
:10039C005360F0238BF823300723C2F808A01360B6
:1003AC00BB68C9F80030BCE80F00AEE80F009CE851
:1003BC000300AB698EE8030043F01003AB61AB693B
:1003CC00029A43F01003AB61AB6943F01003AB61CD
:1003DC004FF480431361029A4FF400531361029A55
:1003EC004FF4004313610AF1040156F80A0031443A
:1003FC000AF1080A01F03CF9BAF1180FF3D1D9F857
:10040C0000301B0712D597F82231012B0ED8A268A9
:10041C007B4B12F0805B93F8233100F0768605E07D
:10042C00774B002283F8232105F0C6F8642004F0F2
:10043C0036FAA022734800210CF033FAEB69002243
:10044C0043F00703EB61AB6943F4006343F00C0327
:10045C00AB616D4D002305F10C01535401320E2A92
:10046C00F7D1FF22AA76EA762A776A77DFF8B4B159
:10047C00664ADFF8B4A1C2F800B0654A02211170D7
:10048C0050461946182203930CF00BFA0122039BD9
:10049C008AF80C2097F805A0ABF5B3722A623046A7
:1004AC001946142285F81EA00CF0FBF9BAF10E0FB8
:1004BC0004D00AF0EF0ABAF1080F02D101238DF82B
:1004CC004A30012003F01CFF18B14088003018BFDF
:1004DC000120D9F8003000F00100C3F340028DF880
:1004EC004620C3F380128DF84820C3F340328DF8B8
:1004FC004020C3F3C0328DF8432013F400628DF812
:10050C00450004D097F81621561E72427241B7F876
:10051C00D8508DF84420ADF84E50C3F30042DD04A2
:10052C00C3F3804003F001018DF84920C3F3C002EE
:10053C0048BF334B8DF8470048BFB3F8E030B7F8ED
:10054C00E40048BFADF84E30B0F5FA7F84BF00230D
:10055C00ADF84E3097F86631ADF84C002D4884F864
:10056C002430002384F8253043709DF84A308DF8F0
:10057C004110002B8DF842200CBF0023022301B93F
:10058C0002B1013308EB8308D8F828304FF000088B
:10059C00A3F1020A1A3303934FF6FF723AF8023FA3
:1005AC00934200F00A81D9B2DFF880909DF84500A3
:1005BC000F011B0A09EB07054A4618B1023901293C
:1005CC0040F2F780022B33D19DF84020002A71D1E4
:1005DC00EFE000BF40D40008FC1600200005FA052F
:1005EC0000080140000C01400010014000000140D7
:1005FC0040420F00F0070020F407002010E000E05C
:10060C00E8090020D0100020A80300209C0700203F
:10061C004C070020CD03002000ED00E050D4000872
:10062C00D00F0020620B002050070020F8E40008D7
:10063C00012B3FD19DF84130002B00F0BA80FF23F5
:10064C0084F86C3084F86D30D3195A7B586803F1F8
:10065C00080B1B890026ADF834300DA9022384F851
:10066C007060E5678DF837308DF8362084F8286097
:10067C00E66226636663A66684F86E6084F86F6033
:10068C0000F0F6FF9BF80210324659F8070006F00E
:10069C00CBFD284605F0B2F9B74BB849C4F8803009
:1006AC00B74BC4F88860C4F8843028460A1D07F09C
:1006BC0023FA7EE0022BDAB246D15FFA88F24FF0D1
:1006CC001C0909FB02F9DFF828C304EB0906012118
:1006DC0086F870100CEB070191F80DE001F108029F
:1006EC00486809894FF0000B86F87180ADF834101A
:1006FC0086F872B00DA986F87AB0F5678DF836E0F9
:10070C008DF83730CDF814C0049200F0B1FFDDF84D
:10071C0014C0049A5CF8070091785A4606F084FDE0
:10072C00284605F06BF9974A9449C6F88020964AFA
:10073C004944C6F88420C6F888B028460A1D07F03C
:10074C00DBF908F1010834E0032A32D19DF8473077
:10075C008E4E3BB194F82670284608214FF6FF7256
:10076C0000231BE0BDF84C208949B2F5FA7FBDF897
:10077C004E3091F826700BD986492846B1FBF2F21F
:10078C00082192B200F0A6FF834B46F827000AE03E
:10079C0082492846B1FBF2F2012192B200F09AFF95
:1007AC007F4B46F82700C36094F82630013384F859
:1007BC002630039B9A457FF4EFAE7A4B04221A70D5
:1007CC000026794D794B354433441036402E0FCBEF
:1007DC0085E80F00F5D106F0B7FA754B754E1A681F
:1007EC00039312F4802F02BF734B01221A703378DB
:1007FC00724D43F004030020337001F0FFF8B5F89C
:10080C00EC000496002840F0C684B5F9EE30002BBD
:10081C0040F0C184B5F9F030002B40F0BC8495F861
:10082C00FB3000210593664B0C221B686548B3F81E
:10083C005630B5F8F470069395F8F380B5F80C9033
:10084C0095F80FA00CF02DF85F4B002118461422E0
:10085C0007930CF026F85D490022C4F850210A7069
:10086C0001F035FC079B8346494E1C46002800F0DE
:10087C00B284574BB7F5807F2360564B6360564B61
:10088C00E360564B2361564B01D1002216E0BB2F7F
:10089C0001D9012212E0612F01D902220EE0292F89
:1008AC0001D903220AE0132F01D9042206E0092FF3
:1008BC0001D9052202E0002FE7D006221A70494B1D
:1008CC0001221A70484A136843F00103136043462F
:1008DC0046490022092B0A7001D90023F8E740F29F
:1008EC00B2324FF0010808FA03F10A40002A40F036
:1008FC00968011F04D0F00F092800793C6F85021AE
:10090C0001F0E5FB079B002800F0898006210A46D0
:10091C000DAB682001F03AFA9DF8391001EA080293
:10092C009DF8371001EA080101FA08F343EA820145
:10093C009DF8352002EA08030B430AD05BB243450D
:10094C0001D1002302E0022B0FD1012386F8543190
:10095C0050E00DF1230368200C21424601F016FAF9
:10096C009DF8233013F00F0303D1052003F0A1FFF2
:10097C0040E0042BE9D1E4E7B91200082804002078
:10098C00991300082116000891120008A0100020ED
:10099C00A803002000127A00B913000840420F008F
:1009AC00A91300087B100020DC02002078D400087A
:1009BC00D00F0020EC160020A0030020E809002036
:1009CC00480700202C01002060160020A103002005
:1009DC002D1D00084F2000082920000890C1793DEA
:1009EC000C0000202C000020E0060020FA1600204D
:1009FC00F8E400085D4B5E4A1A605E4A5A6096F84D
:100A0C005421002A0CBF6F226E221A725A4B0322F9
:100A1C005A705A4A136843F00203136002E0012B28
:100A2C003FF65BAF554B1A68984612F0020F02D096
:100A3C004E4B1B689847FFB25149BAF1000F2AD0B0
:100A4C00D8F800304FB940F2596213F0020F40F25F
:100A5C00712318BF13467D2208E09A0759BF4FF443
:100A6C007A731A464FF4FA634FF47A72994505DBA0
:100A7C00B9F57A6FA8BF4FF47A6900E09946531E16
:100A8C004B44B3FBF2F3013BDBB203FB022286F8CF
:100A9C0055310A6003E086F855A1C1F80090394B36
:100AAC001B689847059F384A00231370924617B16C
:100ABC00022F40F06B834FF0000916AB03F8249D16
:100ACC001E200A210122C6F8589101F05FF9C0B12D
:100ADC009DF83430482B40F082832C4B2C4AD9465D
:100AEC001A602C4A5A60BBF1000F00F07883224B3D
:100AFC000222DA70D8F8003043F00803C8F800304E
:100B0C0001E081466BE395F8E8300BB1224A137093
:100B1C0095F8E9300BB1214A137095F8EA300BB116
:100B2C008AF80030D8F80030DFF87C8013F0080F1A
:100B3C003CD0BDF918B04FF064099BFBF9F738466F
:100B4C0008F0F4F9824609FB17B000B208F0EEF990
:100B5C00134908F03FFA0146504608F033F91149A1
:100B6C0008F038FAC8F8000023E000BF2C01002080
:100B7C00DD1900088F2000082C000020E006002062
:100B8C00C401002060160020FB160020B8000020D5
:100B9C00891E0008151E0008A1030020FA1600206B
:100BAC008988883C00002041801100200023C8F86F
:100BBC000030049B049A1B780A2743F0020313703D
:100BCC00029A4FF400535361029A4FF4804313611D
:100BDC00029B029ADB68192083F40053D360029BBA
:100BEC00029ADB68013F83F48043D36003F057FE25
:100BFC00192003F054FE17F0FF07DFF83883E7D114
:100C0C004FF480434FF40059AC4FC8F81030C8F87B
:100C1C0010903B681B0709D5A94BC8F814901B68AA
:100C2C009847A84B0122C8F810901A70A64BDFF811
:100C3C0008831B68187B08F079F9A44908F0CAF9F5
:100C4C00A34908F0BFF804F0B2F88146B8F80000E8
:100C5C0008F06CF9494608F0BDF90BF081FF9D4B8B
:100C6C001880B8F8000008F061F901469A4808F0BD
:100C7C0065FA9A4908F062FA9449C6F85C01206951
:100C8C0008F0A8F9964908F0A5F9964C964BFF2167
:100C9C0018601B2220460BF004FE20460022227016
:100CAC003A68924B012112F0020F18BF6170197053
:100CBC001FBF032119700221A170540741BF19787D
:100CCC004C1C1C70032448BF445412F00A0F0CD067
:100CDC001A7804218154511CC9B205244454D11CE6
:100CEC0002321970D2B206218154039A126891060D
:100CFC0041BF19784C1C1C70072448BF44546979B7
:100D0C00082901D00E2904D119784C1C1C700B2415
:100D1C00445419780C274754570748BF734F01F1B7
:100D2C000104E4B248BF02311C7041BF39706D49F7
:100D3C0010270F55197812274C1CE4B2475457054D
:100D4C001C7008D595F88C712FB1684F0231397031
:100D5C00644913270F55970541BF19784C1C1C701B
:100D6C00152448BF4454D40548BF1A784FF00004EA
:100D7C0041BF511C19701A238354002198225C48DE
:100D8C000BF08FFD012003F067FCB8B3012C35D8B4
:100D9C004FF04C0B0BFB04F9DFF854A10AEB090CD8
:100DAC000CF1480898F8027017B10134E4B2ECE782
:100DBC0090F9003090F804E018464E4B03228DE871
:100DCC00840001213A4653F82E30CDF814C003F0BC
:100DDC0069FA029070B1DDF814C0394660465A4683
:100DEC000BF05FFD029B4AF8093001231C4488F884
:100DFC000230E4B2012003F015FCC6E73E4A3F4B3B
:100E0C00B5F8E2101A603E4BB5F8280119803D493F
:100E1C0000230B808B703C490A6081B23B4A22F85C
:100E2C0013100133122BF9D1039B1B68D9045CBF3F
:100E3C00B5F82E1111801B0740F1008195F8223175
:100E4C00062B00F2F580DFE803F004070E7994B26C
:100E5C00B20045F2F05201E042F6F8222C4B1A8017
:100E6C0004F057FEE3E042F6F822294B1A8008F012
:100E7C005DF8284908F0AEF8274907F0A1FF08F003
:100E8C0095FA0023254A42F823000133122BF9D19D
:100E9C00234A244940201160234A137003F0DCFBE1
:100EAC00002800F0C58001234FF0070C90F90000DA
:100EBC0040218DE808101D4A1D4BB3E0E0060020D0
:100ECC00B8000020D00000207001002035FA8E3CC4
:100EDC00DB0FC93F8C0100200AE81C4100401C4676
:100EEC00BD378635ED0600206C010020EC06002095
:100EFC003402002038D70008020B002080060020A6
:100F0C008406002098160020CC0F00201409002025
:100F1C00E0010020CDCCCC3F0000B044CC08002038
:100F2C002000002001570008040F00207D59000804
:100F3C00A0860100001001401E00002042F6F8229D
:100F4C00AA4B40201A80AA4AAA4B1A60AA4B10221C
:100F5C001A7003F081FB00286AD001234FF0000EB9
:100F6C0090F9000040218DE80840A44A4FF4E13389
:100F7C0058E042F6F8229D4B40201A80A04A9D4B27
:100F8C001A609D4B08221A7003F066FB00284FD0A4
:100F9C000123002790F9000040218DE88800994A30
:100FAC004FF4E13303F07EF9C6F860013CE042F601
:100FBC00F8218E4A062B11808F494FF00C02DFF876
:100FCC00B8C2DFF8B8E2904F904E914C91480A703D
:100FDC000DD000238CF800308EF800303B701B23B2
:100FEC0033700523227003704FF4E1340AE00021C2
:100FFC008CF800108EF80010397022702121864C6C
:10100C0031700370854A7B4B40201A6003F024FB3F
:10101C0070B10123002690F900008DE848002346AA
:10102C007F4A402103F03EF9003018BF012028B957
:10103C00082004F023F87B4A6E4B1A60039B1A6855
:10104C006D4B12F4804F1FBF082119707648694907
:10105C0018BF086042F20101114099B144F62060BA
:10106C0062490880910441BF082119706F48614999
:10107C0048BF0860D20741BF0C221A706C495D4A08
:10108C0048BF11601A78043A5A7003F0E1FB694BBF
:10109C0018606B79052B02BF674B4FF4C8721A802E
:1010AC00664B4FF47A721A80654A137843F0080342
:1010BC001370644A137823F002031370039B1A68AD
:1010CC0040F6020313406BB15F4A604B1A60604BF1
:1010DC0003221A705F4B01221A705F4A002313809F
:1010EC005E4A13805E4B4FF400425A61AB68039A20
:1010FC0013605C4B01221A70049B049A1B7863F0FA
:10110C007F03137017B0BDE8F08F013B092B3FF63E
:10111C008DA9029A4FF400535361534ADFF860A132
:10112C001068314630605046039300F0A1FA082253
:10113C00CAF810203C2003F0B2FB029B1A46039B1A
:10114C00136197F823319B45BFF66AA9029B4FF4B4
:10115C0080411961029B4FF4004205911A610823EA
:10116C0004927820CAF81430039303F08DFB029B91
:10117C000599049A5961029B78205A61039B0BF1E3
:10118C00010BCAF8103003F07FFBDAE7012F7FF672
:10119C00BAAC1F4687E4354B00221A7000B207F038
:1011AC00C5FE334907F016FF0D90B5F9EE0007F0B8
:1011BC00BDFE2F4907F00EFF0E90B5F9F00007F0B9
:1011CC00B5FE2B4907F006FF2A490F900DA803F036
:1011DC0061FEFFF724BB032003F06BFBE9E4012F56
:1011EC007FF691AC00278AF8009064E4E0010020BF
:1011FC00ED56000820000020040F0020D1580008F4
:10120C00D55600088558000874090020760900207E
:10121C00590800207709002090D0030001560008DF
:10122C00B1570008615700083157000851570008A2
:10123C0041570008BC01002092060020F81600203F
:10124C0086060020FD160020F40A0020340F002032
:10125C00E816002034000020180200201A0200209A
:10126C0000100140A0030020B8D400082800002082
:10127C0035FA8E3C100F00205A080020750900200A
:10128C000008014010F80A3C0133DBB20A2B84BF82
:10129C0010F8131C044A00F80A3C82BF002322F801
:1012AC00113000F80A3C704738090020334A70B5F9
:1012BC00136C9068194440F68C23081A984291607C
:1012CC00D060516013463BD9127893F94510104603
:1012DC008A420BD1111F082908D893F846101829F7
:1012EC0001D8013103E083F8442002E0002183F8A7
:1012FC00461093F944402149A24219D191F8474034
:10130C00B4B10C310024944206DA51F8046F1C4D30
:10131C0025F814600134F6E70C2805D01849002490
:10132C0021F810400130F7E71648017801310170BF
:10133C0083F84520002201211A7083F8471070BDF4
:10134C0092F84710C9B140F2DA51A0F2EF248C4266
:10135C0008D811780B2905D80B1D0131117042F8F2
:10136C00230070BD002283F84720074B03F13002A5
:10137C00002143F8041F9342FAD170BDD003002022
:10138C0038090020AD000020DC030020024A136C59
:10139C000133194411647047D0030020024B53F8F9
:1013AC0020301B6819807047A0100020074BA1F556
:1013BC007A7153F820301A681B8959434FF47A73A9
:1013CC0091FBF3F189B21180704700BFA01000208F
:1013DC008F4A70B51368988A80B2C1B2CE072ED5E9
:1013EC00198821F400610904090C1980198889B243
:1013FC0041F48061198000211171517999B1917971
:10140C0011B9D179FF290ED101219171117A0229DB
:10141C0001BF198889B241F400611980517A41F0F9
:10142C0001011982DFE0517A01F0FE011982D379B2
:10143C00FF2B00F0D880764BFF211971D3E08D077C
:10144C003AD5BFF35F8F107AC0B2012813D151790E
:10145C0089B1917979B1198821F480610904090C59
:10146C001980BFF35F8F198B1988907289B241F480
:10147C00007119801BE0198BBFF35F8F107A6449E0
:10148C0002280AD1487940B1897931B1198821F4FF
:10149C0080610904090C19809FE0107A5C490328CB
:1014AC0005D1487918B18979002940F0968099883E
:1014BC0089B241F4806195E04C0754D501219172B9
:1014CC005179002936D09179002933D0117A1888B6
:1014DC00022911791CD920F480600004000C1880BA
:1014EC001C8AD568C8B2E4B249B26C54198889B266
:1014FC0041F400711980811C1171198A0130C9B233
:10150C0040B22954998889B241F48061998026E0CF
:10151C0080B240F4007018801C8AD568C8B2E4B25E
:10152C0049B26C541C8A411C49B2E4B203306C546D
:10153C00107114E09179364809B9017C41B11988D0
:10154C0089B241F40071198011790131117106E0F1
:10155C00198889B241F4807119800121817119882F
:10156C00C905FCD43FE001F0400101F0FF04E1B1FA
:10157C0010791E8AD568C4B2611C40B2F6B22E54E2
:10158C00C9B2157A117149B2C81C854201BF98883D
:10159C0020F480600004000C08BF9880137A8B4202
:1015AC0021D11B4B02341C711DE006061BD5117991
:1015BC0048B2451C0AD054690131205CC9B218826A
:1015CC00107A117149B288420DD106E0D1791471AB
:1015DC001982517909B9117A29B9998821F4806154
:1015EC000904090C9980117A92F90400013188429E
:1015FC00074B0CD100219971997A31B119688B88FC
:10160C0023F440731B041B0C8B800023137670BDDA
:10161C000C05002038B510F80E2C044650F8043C8C
:10162C005AB9012200F80E2C20F80C1C997A186873
:10163C000222BDE8384005F0F7BD30F80C2C20F83C
:10164C000A1C891A89B220F8081C084A10F80F0CD9
:10165C00002522F8101004F80E5C1868997A2A46B6
:10166C0005F0E2FD04F8065C38BD00BF3809002027
:10167C00F0B5B1F800E000234EFA03F2D50725D5FA
:10168C008E784FEAD30CF40648BFCC7806F00F02E4
:10169C0003F0070748BF2243BF0050F82C500F241B
:1016AC00BC4025EA0404BA402243282E40F82C20E2
:1016BC0005D1C46801229A4024EA020205E0482EB2
:1016CC0004D1C46801229A402243C2600133102B1A
:1016DC00D2D1F0BD2DE9F7438E460546DFF898923E
:1016EC00114699F819400068164698467246631CD4
:1016FC0089F8193006F08EF92B8901A9ADF8043060
:10170C0018238DF80630686802238DF80730FFF730
:10171C00AFFFAB7A09F11C07240127442A6849461C
:10172C000C2B00F2F680DFE813F00D00F400F4004F
:10173C00F4005100F400F400F4008A00F400F4000A
:10174C00F400C200138CDFF834C223F001031B0435
:10175C001B0C1384138CB2F804E0108B624520F040
:10176C0073004FEA00404FEA10409BB21FFA8EFE06
:10177C0040F0700014D00CF5006C624510D00CF5E4
:10178C00406C62450CD00CF5806C624508D00CF5B1
:10179C00806C624504D023F0020343F0030307E09E
:1017AC0023F00E032EF4407E43F003034EF4807EB0
:1017BC00A2F804E01083A2F834801384138B23F076
:1017CC0008031B041B0C43F0080336E0138CDFF8F2
:1017DC00ACC123F010031B041B0C1384138CB2F844
:1017EC0004E0108B624520F4E6404FEA00404FEADB
:1017FC0010409BB21FFA8EFE40F4E04008D00CF56E
:10180C00006C624504D023F0200343F0300307E062
:10181C0023F0E0032EF4406E43F030034EF4806E60
:10182C00A2F804E01083A2F838801384138B23F4FD
:10183C0000631B041B0C43F40063138369E0138CDB
:10184C00DFF838C123F480731B041B0C1384138C36
:10185C00B2F804E0908B624520F073004FEA004030
:10186C004FEA10409BB21FFA8EFE40F0700008D079
:10187C000CF5006C624504D023F4007343F4407300
:10188C0007E023F460632EF4405E43F440734EF49F
:10189C00805EA2F804E09083A2F83C801384938BC2
:1018AC0023F008031B041B0C43F0080330E0138CDB
:1018BC00DFF8C8C023F480531B041B0C1384108C5A
:1018CC00B2F804E0938B20F4005023F4E6431B049D
:1018DC0000041B0C000C62451FFA8EFE43F4E0431F
:1018EC0040F4405003D00CF5006C624503D12EF44B
:1018FC00804E4EF4804EA2F804E09383A2F8408010
:10190C001084938B23F400631B041B0C43F40063BF
:10191C0093832B7B43B1B2F844306FEA43436FEAB5
:10192C0053439BB2A2F8443013889BB243F001039B
:10193C001380AB7A0C2B18D8DFE803F007171717B6
:10194C000B1717170F17171713000B1902F1340089
:10195C000AE00B1902F1380006E00B1902F13C0009
:10196C0002E00B1902F14000D86138460C44A68401
:10197C00226203B0BDE8F0830C050020002C01406E
:10198C00104B13B593F8DC201C46CAB90E4B1B68E0
:10199C00B3B11A681AB10D49886902438A619A88F1
:1019AC009868ADF8042002228DF8072004220DEB74
:1019BC0002018DF80620FFF75BFE012384F8DC3072
:1019CC0002B010BD0C050020F804002000100240ED
:1019DC0008B5FFF7D5FF074B1B7813B1012B03D0CC
:1019EC0008BD4FF4006201E04FF48052024B1A80A4
:1019FC0008BD00BFFC0400201E000020012828BFE9
:101A0C0001202DE9F04F0646142000FB06F3704F21
:101A1C0089B0F918FC586F4B0A691C6083F8DD60BB
:101A2C006D4BB1F80880DD69B1F80AA02A43DA6180
:101A3C00A2884D6822F440721204120C4AEA08097A
:101A4C00A28003A9C5F8109002228DF80E0028463A
:101A5C000193ADF80C908DF80F20FFF709FE019B58
:101A6C0000971F464FF0080BAA6818EA020F03D123
:101A7C000A2002F009FFF7E70A20C5F8148002F0EB
:101A8C0003FFC5F810800A2002F0FEFEBBF1010B2B
:101A9C00EAD1C5F814A00A2002F0F6FEC5F81480AD
:101AAC000A2002F0F1FEC5F810800A2002F0ECFECC
:101ABC000222C5F810A0284603A98DF80F201C227D
:101ACC008DF80E20ADF80C90FFF7D2FD434A03A819
:101ADC0094423A690BBF42F4001242F480023A611C
:101AEC003A610BBF3A693A6922F4001222F480027F
:101AFC003A61A38823F440731B041B0CA380238836
:101B0C009BB243F001032380A58804F0BFF805992C
:101B1C00334B25F03F05B1FBF3F32D042D0C1D4386
:101B2C00ADB2A5802288002522F001021204120C0D
:101B3C0022802C4A03A8B1FBF2F100298AB208BF1B
:101B4C00012242F400414FF4967253434FF47A72DF
:101B5C0093FBF2F301339BB22384A1832388009A75
:101B6C009BB243F001032380238823F4816323F089
:101B7C0002031B041B0C23804FF48043238114238A
:101B8C0003FB0626737B01248DF80C308DF80D5069
:101B9C008DF80E508DF80F4003F012FF337B9DF83B
:101BAC000F208DF80C308DF80D508DF80E501AB1A9
:101BBC0003A803F005FF08E05A0903F01F039C403B
:101BCC0002F12003084A42F8234009B0BDE8F08F27
:101BDC00E4D400080C050020001002400054004022
:101BEC0040420F00804F120000E100E010B5214C84
:101BFC002368998A89B211F4706F1CBF012284F892
:101C0C00DE2011F4E06F2BD01A8B9A88890522F410
:101C1C0080624FEA02424FEA12429A8020D41A881C
:101C2C0092051DD41A88D0050FD51A88D105FCD47D
:101C3C001A8892B242F400721A801A889205FCD467
:101C4C0094F8DD00FFF7DAFE0AE01A8892B242F44B
:101C5C0000721A809A8822F440721204120C9A8034
:101C6C002268938A23F470631B041B0C9382002359
:101C7C00237610BD0C050020064A08B513880133E5
:101C8C009BB21380044B93F8DD00FFF7B7FE0020E6
:101C9C0008BD00BFDE0600200C05002013B51F4B4D
:101CAC004000C0B2587202AC1868D97104F8012D0A
:101CBC00002101221A745C615971DC601A721A7667
:101CCC0083F8DE1040B38288920515D40288D405BF
:101CDC000DD447F230520188890502D5013AFAD168
:101CEC0012E08AB1028892B242F480720280828839
:101CFC0092B242F44072828047F23052197E11B196
:101D0C00013AFBD100E012B9FFF7B6FF04E0034B38
:101D1C0093F8DE0080F0010002B010BD0C0500202D
:101D2C0008B5FFF72DFE6B2180226820FFF7B6FF68
:101D3C00642002F0B4FD6B2103226820FFF7AEFF94
:101D4C000F2002F0ACFD0F4B19211A786820FFF719
:101D5C00A5FF0F2002F0A3FD0B4B1A211A78682067
:101D6C00FFF79CFF1B2118226820FFF797FF1C210F
:101D7C0010226820FFF792FFBDE808406820372149
:101D8C0002228BE7FD0400200C00002010B540005F
:101D9C001C4CC0B26072E171012000212174607191
:101DAC00227220762068E360636184F8DE1040B311
:101DBC0083889B0515D40388D9050DD447F230537D
:101DCC000288920502D5013BFAD112E08BB103884F
:101DDC009BB243F48073038083889BB243F44073BB
:101DEC00838047F23053227E12B1013BFBD100E0DD
:101DFC0013B9BDE810403FE7024B93F8DE0080F0CA
:101E0C00010010BD0C05002037B506220446032145
:101E1C006B461E20FFF7BAFF9DF801309DF80000BD
:101E2C00154D43EA002000B207F080F8296807F04E
:101E3C00D1F807F095FA9DF8033020809DF8020048
:101E4C0043EA002000B207F071F8A96807F0C2F865
:101E5C0007F086FA9DF80530A0809DF8040043EA4F
:101E6C00002000B207F062F8696807F0B3F807F0D9
:101E7C0077FA608003B030BD100000202DE9FF41DF
:101E8C00604B1B689BB11A681AB15F4988690243A1
:101E9C008A619A889868ADF8042002228DF8072090
:101EAC0004220DEB02018DF80620FFF7E1FB322036
:101EBC0002F0F5FC002111221E20FFF7EFFE01219C
:101ECC0060221E20FFF7EAFE642002F0E8FC0024EA
:101EDC0002A8FFF799FF274626460A250221012270
:101EEC001E20FFF7DBFE322002F0D9FC02A8FFF720
:101EFC008BFFBDF90820BDF90A1014448A42A8BF13
:101F0C000A46BDF90C300F4493421E44A8BF134639
:101F1C0013F5805F09DD3D4A013DD36883F400531E
:101F2C00D360DBD14FF0010801E04FF000081E2018
:101F3C0000211222FFF7B2FE0A25022101221E20E7
:101F4C00FFF7ACFE322002F0AAFC02A8FFF75CFF00
:101F5C00BDF90820BDF90A10A41A8A42A8BF0A4686
:101F6C00BDF90C307F1A9342A6EB0306A8BF1346AB
:101F7C0013F5805F07DD254A013DD36883F40053D8
:101F8C00D360DAD101E04FF00008204606F0CEFF16
:101F9C0001461F4807F0D2F81E4D20F00040286083
:101FAC00384606F0C3FF0146194807F0C7F820F081
:101FBC0000406860304606F0B9FF0146164807F04D
:101FCC00BDF820F00040A860002170221E20FFF711
:101FDC0065FE012120221E20FFF760FE1E2002213B
:101FEC000022FFF75BFE642002F059FCB8F1000FF1
:101FFC0004D14FF07E532B606B60AB6004B0BDE836
:10200C00F08100BF000500200010024000100140CC
:10201C0000406F461000002001C05E4613B501223F
:10202C000DF107033A2104466820FFF7AFFE0520A7
:10203C0002F02AFC9DF8073003B10123237002B093
:10204C0010BD13B506220446432168206B46FFF7EA
:10205C009DFEA0B19DF800209DF8013043EA0223BB
:10206C0023809DF802209DF8033043EA022363800D
:10207C009DF804209DF8053043EA0223A38002B0AA
:10208C0010BD13B5062204463B2168206B46FFF7B2
:10209C007DFEA0B19DF800209DF8013043EA02239B
:1020AC0023809DF802209DF8033043EA02236380CD
:1020BC009DF804209DF8053043EA0223A38002B06A
:1020CC0010BDFFF785B991E5FFF782B98EE507B52D
:1020DC00232002F0E4FB6820752101220DF1070397
:1020EC00FFF754FE28B19DF80700A0F16803584291
:1020FC00584103B05DF804FB7A4A7B4913682DE91B
:10210C00F04F03F59C4320330B60784B89B0186873
:10211C00884610F4804F0592019307D104F032F8F1
:10212C0020B998F80430013388F8043098F8056029
:10213C009EB16D4B013E5E71EEE03B68072C98BF83
:10214C00195D6B4B88BF21461B686A489847032C66
:10215C000AD908EB4404E0800136664BF4B21D78D2
:10216C00654FA542E9D81FE03A6804F10E0302EB73
:10217C0083039988DA880028EBD04FF47A73401ADD
:10218C005843531A90FBF3F040F6C90300F57A70EC
:10219C00984205DC40F2EE239842B8BF184601E0A5
:1021AC0040F6CA0080B2D4E798F804600324B6FB6A
:1021BC00F4F40F2388F82A3098F82C3004EB4404FC
:1021CC0003933B68341B029398F82BA0E3B2DFF81F
:1021DC0044B104930024AC4251DA484B670033F805
:1021EC001490BAF1000F09D103F0CCFF28B1039B76
:1021FC00002B08BF4FF0000900E0D146029B988AE3
:10220C00484502D8D88A48450ED2E0B203F092FF76
:10221C00032C8146DFBF98F82AE00120A0402EEA6B
:10222C000000D8BF88F82A0003F0ACFF18B134487E
:10223C0027F800901FE0049B98F876002BF8139079
:10224C0028B9022E14D9284B012083F87600BBF84C
:10225C000000BBF802300344BBF8040003442948D7
:10226C009BB23B521BB2032093FBF0F39BB200E0FA
:10227C004B4623483B5201340BF1060BABE798F865
:10228C002A202148A2F10F077A427A4188F890203F
:10229C001E4B6AB11E4A1268560109D40268D968ED
:1022AC009A60521AC82A37D9012283F8212033E0C8
:1022BC0002689868DA605B68121A9A4288BF134BFE
:1022CC004FF0000188F82B1088BF83F821100024F0
:1022DC00AC4221DAE0B203F02DFF094B23F81400D5
:1022EC000134F5E7F4160020EC050020D00F002097
:1022FC0020000020040F0020CC0F0020F20500204D
:10230C001409002064060020E41600209816002012
:10231C00E80600201A060020019B1B68DC0405D58A
:10232C00884B1B68D80701D406F01EFD864B1A6833
:10233C00937AFBB18549013B31F81300137B1BB138
:10234C00C0F53B60083080B200B2A0F57A70B0F5F1
:10235C007A7FA8BF4FF47A7020EAE07006F0E6FDB1
:10236C007B4906F0EBFE7B4906F034FE07F01EF8C5
:10237C00794B1880019B794C1B6813F4807F00F01B
:10238C000281059BDFF8DCA11A68754B9A4205D9CE
:10239C009AF8023013B901238AF802309AF8023005
:1023AC00002B00F0F0806F4B267893F82150654B92
:1023BC00691E4D424D411F68002DC6F38006C7F3C0
:1023CC008067029314BF4FF000094FF003099AF88D
:1023DC002030052B00F2D180DFE803F0034B507363
:1023EC00829F002E39D0D8F89400B8F8981002F0DB
:1023FC00C1F9012809D15C4A5C4B12681B68D28870
:10240C00642101FB0233CAF810306FB1564B1B68C4
:10241C001B794BB106F090F803238AF820304FF467
:10242C007A73CAF81C30D2E7002D40F0A6804F4BCF
:10243C00DFF830B11A68DAF810309A4209D906F090
:10244C007BF803238BF8203040F6B833CBF81C30E4
:10245C00BDE701238BF82030B9E74FF4806017B14A
:10246C0002F0FCFD01E002F0E8FD0023CAF8103098
:10247C0083E0002D46D106F05FF8A8E725B10523CF
:10248C008AF82030012100E0294666B1D8F8943052
:10249C004FF00209DA892D4B1A805A809A80324A01
:1024AC0012685288DA80314B1A68DAF814309A4282
:1024BC0001D8002E5ED147F23053CAF81C300323EA
:1024CC0021E0237843F00203237006F04DFC274BE8
:1024DC00DAF81C201B681344CAF81830042312E0E5
:1024EC00224B9DB11A68DAF818309A4245D9204B24
:1024FC001B781BB9029B1B68DA073ED4237823F0A8
:10250C000203237005238AF8203060E71B68DAF891
:10251C001C201344CAF818302FE0134A134B1268CE
:10252C001B68D288642101FB02334FF48060CAF827
:10253C00103000238AF820308AF8033002F07DFD39
:10254C0045E700BFE8060020CC0F0020140900204E
:10255C0000007A4400C07F443C070020FD16002098
:10256C00404B4C0098160020BC160020E4160020AE
:10257C001C00002000297FF42AAFB9F1000F02D013
:10258C00484602F023F99E4D05F58D70B5F8E21022
:10259C0002F0F0F8AA46814668B905F0BFFF994BE6
:1025AC000022C3F80090C3F80490C3F80890964B2F
:1025BC001A605A609A6023785B073AD5019B1B68B6
:1025CC00DF0636D598F89A30904DDE0631D4904B14
:1025DC001B7843B39AF87231B9F1000F11D15BB18A
:1025EC008C4B1A68D5F89C309B1A002B04DA06F039
:1025FC00BBFB85F8A0901CE0102002F0E7F801234B
:10260C000EE03BB1834A4FF47A71126801FB03234D
:10261C00C5F89C3098F8A0305BB102F0C5F80023E7
:10262C0088F8A03005E0B9F1000FE5D095F8A0309E
:10263C00F2E7002216469AF870719AF87111BAF8FE
:10264C002A51BAF82CE1744BB60833F912000293F4
:10265C00A842C4BF66F07F03DEB201327045B8BF3A
:10266C0046F04006042AEED198F8A1206748B24201
:10267C0005D190F8A220F92A04D8013200E00022FA
:10268C0080F8A220624A88F8A16092F800B0634DED
:10269C000392BBF1000F1CD12A68D00708D5B9F101
:1026AC00000F16D12278D10713D506F027FB10E0C6
:1026BC00227852070DD5554A92F82B204AB1584A28
:1026CC00D27832B911B106F04FFB02E0B9F1000F2C
:1026DC00F9D098F8A220DFF85891142A63D100376A
:1026EC0018BF0127BBF1000F13D05F2E02D087B1AA
:1026FC007D2E0ED1227802F0040202F0FF0B12B1F3
:10270C0006F032FB05E00B2002F060F83F4B83F83B
:10271C00A2B0227802F0040202F0FF01002A42D19A
:10272C00572E0BD13F4B4FF47A721A803E4B1B68DD
:10273C0013F0080337D13D4A138034E0019B1A682B
:10274C00530718D55A2E16D198F8A3302F4A2BB10F
:10275C00012382F8A31082F8A43024E092F8A5306B
:10276C0083F0010382F8A5300BB10C2000E00D20A2
:10277C0002F02CF817E05D2E00F0F6835B2E00F0D3
:10278C00F5835E2E01D10320F1E3562E01D102F028
:10279C0013FF039B1A78002A00F0F9836F2E40F088
:1027AC00F28306F0ABFA019B1B68580751D598F8D9
:1027BC00A530164A93B1237859070FD5029BB3F96C
:1027CC000610BAF82A31994208DD2B6813F0010380
:1027DC0002BF3221A2F8A81082F8A5302B68DA03C8
:1027EC0028D598F8AA20094B2AB993F8A32012B936
:1027FC003222A3F8A820012388F8AA3029E000BFD0
:10280C00E80900200810002084100020EC050020AE
:10281C001C000020E416002014090020E80600200B
:10282C0098160020F8160020E0060020360700203D
:10283C004807002098F8A330A54A53B1237803F039
:10284C00040303F0FF0123B9012382F8A31082F8DB
:10285C00A430D9F8006000232B6006F17B0406F14C
:10286C00CB072278637814F8010C9A420BD22146DC
:10287C0001F05CFF38B114F8022C012303FA02F2C8
:10288C002B6813432B600434BC42EAD1914B1B7868
:10289C0043B1914C914E2368914D13F0020F40F0CF
:1028AC00F682EDE206F1CA0406F5897622786378A1
:1028BC0014F8010C9A4223D2214601F037FFF8B1EB
:1028CC00A378884A013B03EB4303257913440C227C
:1028DC0002FB0582D2F8B01094F803E099427C48D0
:1028EC000ED0C2F8B0300023C2F8B43082F8ACE09D
:1028FC00012390F8DC20AB4022EA030380F8DC30A3
:10290C000634B442D2D1784A784B12681C680292D1
:10291C0098F82B20764F0392002604933A68002AED
:10292C0000F0A7821578002D00F0A3827B68029935
:10293C00CB1A002B0ADB01F5FA737B6098F8DC10DC
:10294C000123B34021EA030388F8DC30039B002BFE
:10295C0000F08F8217F8043C51780433DBB2002965
:10296C0040F04C82634931F91310BAF8283103F165
:10297C00C800814202DD92F802B014E0C83B9942D3
:10298C0004DA92F802B0CBF1000B0CE098F8DC20E2
:10299C000123B34022EA030388F8DC30029B03F5E1
:1029AC00FA737B6065E298F8DC303341DB0700F1A9
:1029BC006082BBF1000FCCBF0220012001F02CFF84
:1029CC006B1E434A132B00F24D82DFE813F0140008
:1029DC0020002F00400057005E00D3002F018B0118
:1029EC00B701E3014B0240004B005E00D3002F0106
:1029FC00A60002015E0123789B44BBF1FA0FA8BF2D
:102A0C004FF0FA0B2BEAEB7B84F800B00AE063780A
:102A1C009B44BBF1640FA8BF4FF0640B2BEAEB7B1C
:102A2C0084F801B0204601F067FE1BE2E3782046F3
:102A3C009B44BBF1640FA8BF4FF0640B2BEAEB7BFC
:102A4C0084F803B0D2F8E01001F00EFE0AE26379CC
:102A5C005B44642BA8BF642323EAE3730D2D6371DD
:102A6C0000F0008223799B44BBF1640FA8BF4FF0A8
:102A7C00640B2BEAEB7B84F804B0F3E1A3799B4461
:102A8C008BF3080B84F806B0ECE1D2F8E49099F8DB
:102A9C000020022A34D1584606F048FA164906F0AE
:102AAC004DFBD9F8241006F08DF90021059006F0A5
:102ABC002FFC40B9059A1149104606F047FC059ABF
:102ACC0010B10E4A00E00022C9F8242022E000BF19
:102ADC00EC050020FE160020E8060020E006002091
:102AEC00E40600200CD50008E41600204407002062
:102AFC009C06002014090020000020410000C84260
:102B0C0099F802205A44C82AA8BFC82222EAE272C5
:102B1C0089F802200F2D00F0A581B44BD3F8E450B6
:102B2C002B78022B1AD1584606F000FAB04906F061
:102B3C0005FB296A06F046F90021834606F0E8FBFE
:102B4C0038B95846AB4906F001FC20B1DFF8A4B205
:102B5C0001E04FF0000BC5F820B083E16B789B448B
:102B6C00BBF1C80FA8BF4FF0C80B2BEAEB7B85F865
:102B7C0001B077E1D2F8E49099F80020022A1BD139
:102B8C00584606F0D3F99B4906F0D8FAD9F830101C
:102B9C0006F018F90021059006F0BAFB40B9059A29
:102BAC009449104606F0D2FB059A10B1914A00E008
:102BBC000022C9F8302009E099F80C205A44C82AA0
:102BCC00A8BFC82222EAE27289F80C20102D00F06E
:102BDC004981864BD3F8E4502B78022B1AD15846F6
:102BEC0006F0A4F9834906F0A9FAE96A06F0EAF8B6
:102BFC000021834606F08CFB38B958467D4906F017
:102C0C00A5FB20B1DFF8ECB101E04FF0000BC5F8EB
:102C1C002CB027E1EB7A9B44BBF1C80FA8BF4FF057
:102C2C00C80B2BEAEB7B85F80BB01BE1D2F8E490D8
:102C3C0099F80020022A1BD1584606F077F96E4904
:102C4C0006F07CFAD9F83C1006F0BCF8002105908F
:102C5C0006F05EFB40B9059A6649104606F076FB15
:102C6C00059A10B1634A00E00022C9F83C2009E043
:102C7C0099F816205A44C82AA8BFC82222EAE27240
:102C8C0089F81620112D00F0ED80584BD3F8E45044
:102C9C002B78022B1AD1584606F048F9564906F003
:102CAC004DFAA96B06F08EF80021834606F030FB36
:102CBC0038B958464F4906F049FB20B1DFF834B11A
:102CCC0001E04FF0000BC5F838B0CBE06B7D9B44B6
:102CDC00BBF1C80FA8BF4FF0C80B2BEAEB7B85F8F4
:102CEC0015B0BFE0D2F8E4502B78022B1AD158461D
:102CFC0006F01CF93E4906F021FAA96A06F062F8C2
:102D0C000021834606F004FB38B95846394906F0D1
:102D1C001DFB20B1DFF8DCB001E04FF0000BC5F873
:102D2C0028B09FE0EB789B44BBF1C80FA8BF4FF0D5
:102D3C00C80B2BEAEB7B85F803B093E0D2F8E45098
:102D4C002B78022B1AD1584606F0F0F8294906F0D8
:102D5C00F5F9696B06F036F80021834606F0D8FACF
:102D6C0038B95846234906F0F1FA20B1DFF884B09F
:102D7C0001E04FF0000BC5F834B073E06B7B9B4463
:102D8C00BBF1C80FA8BF4FF0C80B2BEAEB7B85F843
:102D9C000DB067E0D2F8E4502B78022B1AD15846CC
:102DAC0006F0C4F8144906F0C9F9296C06F00AF8C3
:102DBC000021834606F0ACFA38B958460D4906F0A6
:102DCC00C5FA20B1DFF82CB001E04FF0000BC5F8CC
:102DDC0040B047E0EB7D9B44BBF1C80FA8BF4FF060
:102DEC00C80B2BEAEB7B85F817B03BE0EC05002019
:102DFC00000020410000C84200007A44012931D172
:102E0C009078844A32F913B0BBF5617F05DB40F64C
:102E1C0033039B45A8BF9B4601E04FF4617B0C2D0F
:102E2C0020D14FF4966393FBF0F0ABF5617B9BFBE9
:102E3C00F0FB794A5FFA8BFB13785B4512D0BBF140
:102E4C00040F34BF5B46022305FB03A51370049BE0
:102E5C0005F2F2451D6002F0EDF90BF10100C0B274
:102E6C0001F0DAFC98F8DC200123B340134388F816
:102E7C00DC300136042E07F10C077FF44FAD08E56A
:102E8C00019B1B68D8050FD5644BDB7863B13368A5
:102E9C00990709D52B8813F001070AD105F03EFBE1
:102EAC00012002F0DBF804E0012002F0C6F8012357
:102EBC0000E00023226852070CD55BB1012002F020
:102ECC00BCF82B889B0708D405F028FB022002F0E5
:102EDC00C5F802E0022002F0B0F82B88504A13F03B
:102EEC00030F4FF4005114BF51611161326812F09D
:102EFC000A0F23D02268D70609D55E070AD404200E
:102F0C0002F0ACF8474B1B88A8F8E83002E004202C
:102F1C0002F093F82368980606D52B88590606D438
:102F2C00402002F09BF802E0402002F086F8236873
:102F3C005A0642BF3B4B1B88A8F8EA3023684FF473
:102F4C0080701B0502D502F089F801E002F075F8DB
:102F5C009AF80530082B01D00E2B58D1402009B01F
:102F6C00BDE8F04F02F069B8012000E00220C7B2C2
:102F7C007B1E8AF8F03402F0B3F802F07FF9384681
:102F8C0001F04AFC0FE417B17E2E3FF40AAC972EE9
:102F9C0004D14FF4C873A8F8A63004E4A72E07D1C7
:102FAC0098F89A3043F0040388F89A30FFF7FBBB8B
:102FBC000022BB2E079201D1022303E0B72E04D1CD
:102FCC004FF6FE73ADF81E300AE0BE2E01D102237F
:102FDC0004E0BD2E7FF4E7AB4FF6FE73ADF81C306A
:102FEC00D9F80030BDF81C10B3F858200A44A3F8E7
:102FFC005820BDF81E10B3F85A200A44A3F85A20E2
:10300C0002F0DAFA002388F8A230FFF7CCBB09B043
:10301C00BDE8F08F14090020C0160020981600207F
:10302C00001001403607002010B5044680B205F0B0
:10303C006BFB200CBDE8104005F066BB38B50446B0
:10304C000D46242005F04EFB4D2005F04BFB002CCB
:10305C00094C14BF21203E2005F044FB23680022BC
:10306C0028469A7105F03EFB236893F84900BDE8A9
:10307C00384005F037BB00BFD806002001460020C1
:10308C00DCE746282DE9F047044600F0918500F274
:10309C0091802C2800F0DD844BD8052800F0268187
:1030AC0029D8022800F009810ED8012840F09A8511
:1030BC000320FFF7E3FF002005F014FB204605F08A
:1030CC0011FB0D2000F012BD032800F0058104282F
:1030DC0040F088850620FFF7D1FF432005F002FB66
:1030EC004A2005F0FFFA4D2005F0FCFA312005F0DE
:1030FC00F9FA00F05EBC262800F07A840CD822285D
:10310C0000F07983242840F06D850420FFF7B6FF8A
:10311C00D84B986800F061BD282800F087842A28D5
:10312C0040F060850120FFF7A9FFD24B587900F0E1
:10313C00DDBC3A2800F006821AD8342800F07D83D2
:10314C000AD8322840F04E850120FFF797FFC94B73
:10315C0093F8240100F0CABC362800F00E853828FC
:10316C0040F040850420FFF789FFC24C00F04FBCB3
:10317C00402800F0BE8411D83B2800F035833D2850
:10318C0040F03085BB4C0220FFF778FF94F87201B9
:10319C0005F0A8FA94F8710100F0A8BC422800F0E0
:1031AC00CB84452840F01E851320FFF767FF0024D1
:1031BC0000F008BD6E2800F0C98142D8652800F0E7
:1031CC00B28022D84B2800F0638408D8492840F0FC
:1031DC0009850220FFF752FFA64B9889EAE34D2898
:1031EC0000F06584642840F0FD840720FFF746FF5B
:1031FC00E72005F077FA9F4B587905F073FA002019
:10320C0005F070FA042000F0E8BC692800F0788121
:10321C000AD8662800F04281682840F0E384102028
:10322C00FFF72CFF002463E16C2800F07C816D28F3
:10323C0040F0D8840620FFF721FF0020FFF7F4FEB2
:10324C00B7E3752800F0C48215D8722800F06F839C
:10325C0007D86F2800F0A681702800F0CD8100F00F
:10326C00C1BC732800F09A83742840F0BB844FF0E3
:10327C00000801260EE3A02800F0AC830AD87728BA
:10328C0000F035837B2840F0AD843C20FFF7F6FE40
:10329C00002433E2F02800F09083FE2840F0A28452
:1032AC000820FFF7EBFE002005F02EFA002005F0B9
:1032BC002BFA002005F028FA7BE30420FFF7DEFE52
:1032CC00432005F00FFA4C2005F00CFA462005F0CF
:1032DC0009FA4C2000F00ABCFFF7D0FE012005F0E3
:1032EC0001FA0A2005F0FEF90020FFE31A20FFF78F
:1032FC00C5FE0024604B185D013405F0F3F90B2C6E
:10330C00F8D100245D4B185D013405F0EBF9082C65
:10331C00F8D100245A4B185D013405F0E3F9072C61
:10332C00F8D100F05CBC574C0B20FFF7A7FEA0882F
:10333C0005F0EAF9E08880B205F0E6F9A368C3F37A
:10334C00C000C3F38002800040EA4200C3F3400295
:10335C001043C3F3401240EAC20003F010031843B9
:10336C0005F0D2F9A289236902F0080103F4475948
:10337C0049EA010903F4804149EA010903F40041D7
:10338C0049EA010903F4803149EA010903F40031E7
:10339C0049EA010903F4802149EA010903F40021F7
:1033AC0049EA010903F4801149EA010903F00073A9
:1033BC0049EA0303DFF8D49012F0010F99F800905A
:1033CC0018BF4FF00208C9F3800908BF4FF000087E
:1033DC0043EA090312F0020F43EA080314BF4FF04B
:1033EC00040C4FF0000C12F0040F43EA0C0C14BF49
:1033FC004FF0100E4FF0000E12F0400F14BF2027AC
:10340C0000274CEA0E0E12F0100F14BF4FF400768A
:10341C0000264EEA070712F0200F14BF4FF4806508
:10342C0000253E4312F4807F14BF4FF4006000204F
:10343C00354312F4007F14BF4FF4001100212843D0
:10344C0012F4806F41EA000114BF4FF08063002337
:10345C00002019430346247DA34219D20A4A9D5CDD
:10346C00012202FA05F50D421CBF9A4010430133AC
:10347C00F2E700BFE8090020D8E50008E4E5000801
:10348C00EDE50008D8060020ED060020FD16002012
:10349C00FFF7CAFDBB4B93F8F00427E31220FFF7AC
:1034AC00EDFDB94B00251B88B3F5806F8CBF08264A
:1034BC000126B64C04F1300333F91500013590FBAD
:1034CC00F6F080B205F020F9032DF2D1E08E05F074
:1034DC001BF9208F05F018F9608F05F015F9A08FF6
:1034EC0005F012F9E08F05F00FF9B4F8400061E235
:1034FC00A74B185D013405F0F5F8102CF8D16EE3EC
:10350C00A44D00242878400000F0FE00FFF7B6FD23
:10351C002B789C4280F063839F4B33F8140005F0AA
:10352C00F3F80134F4E7994C0620FFF7A7FDB4F843
:10353C005A0005F0E9F8B4F85C0005F0E5F8B4F8C9
:10354C005E0037E20420FFF799FD45E34FF6FF7567
:10355C000720FFF793FD914B8C4C1888FF28A8BFD0
:10356C00FF20C0B205F0BEF8206EA842A8BF2846C6
:10357C0020EAE07080B205F0C7F8B4F8640005F0FA
:10358C00C3F8804BA06E93F817313BB10A23584314
:10359C00A842A8BF284620EAE07001E000F30F0023
:1035AC0080B207E2794C0B20FFF768FDE36E2546ED
:1035BC00187805F097F8E36E0026587805F092F825
:1035CC00EB6E724C33441879013605F08BF8032EF0
:1035DC00F6D1E36ED87905F085F8E36E987805F0AE
:1035EC0081F8E36ED87805F07DF8E36E588905F024
:1035FC008BF8E36E187A79E2644C1E20FFF73EFDDF
:10360C00236F00251B78022B65D1236F05F108026F
:10361C0053F82200624905F0DDFC09F0A1FA80F3B1
:10362C000800C0B205F05EF8236F5E4903EB85031A
:10363C00D86A05F0CFFC09F093FA80F30800C0B209
:10364C0005F050F8236F05F10E0253F8220056498D
:10365C0005F0C0FC09F084FA80F30800C0B2013513
:10366C0005F040F8032DD0D1072D236F21D1586CD4
:10367C004B4905F0AFFC09F073FA80F30800C0B2B7
:10368C0005F030F8236F4649986C05F0A3FC09F05F
:10369C0067FA80F30800C0B205F024F8236F93F8A2
:1036AC004C0005F03FFC09F05BFA80F30800C0B257
:1036BC000BE02B44587805F015F8236F2B44D87A7F
:1036CC0005F010F8236F2B44587D013505F00AF8EE
:1036DC000A2DC9D183E2236F2B44587805F002F8E8
:1036EC00236F2B44D87A04F0FDFF236F2B44587DB5
:1036FC00013504F0F7FF0A2DEDD170E2234D04F1F2
:10370C0008022B6F284953F8220005F063FC09F0DE
:10371C0027FA80B204F0F8FF2B6F234903EB8403E4
:10372C00D86A05F057FC09F01BFA80B204F0ECFFE4
:10373C002B6F04F10E0253F822001B4905F04AFCD2
:10374C0009F00EFA013480B204F0DEFF032CD5D15F
:10375C00072C2B6F2AD1586C134905F03BFC09F050
:10376C00FFF980B204F0D0FF2B6F0F49986C05F075
:10377C0031FC09F0F5F980B204F0C6FF2B6F93F819
:10378C004C001FE0E80900201E000020D806002095
:10379C001A070020040F002014090020C80F002075
:1037AC00000020410000C84200007A4423445878AD
:1037BC0004F0AAFF2B6F2344D87A04F0A5FF2B6FDB
:1037CC002344587D013404F09FFF0A2CC0D106E23B
:1037DC002F20FFF753FCCE4C14F8010F002800F0FB
:1037EC00FE8104F07FFFF7E70120FFF747FCC94B90
:1037FC001B6F18787AE15020FFF740FC0025C54B71
:10380C000C211C6FC44B04EB850494F87920013512
:10381C0001FB023393F8380004F064FF94F87A004B
:10382C0004F060FF94F87B0004F05CFF94F87C00DB
:10383C0004F058FF142DE2D1D1E14820FFF71EFC13
:10384C000025B44B1C6F062303FB054494F8CE00F3
:10385C0004F048FF94F8C90004F044FF94F8CA003F
:10386C0004F040FF94F8CB0004F03CFF94F8CC003B
:10387C0004F038FF013594F8CD0004F033FF0C2D23
:10388C00DFD1ACE1002E00F0AA815FFA88F0FFF7DF
:10389C00F5FB002600279F4B1A7D9742F2DA153371
:1038AC00FA5C00240C2363439B4D05F13001595CF9
:1038BC00914207D12B44586B09F037F882462EB948
:1038CC00B14605E001341C2CECD10EE080440CE038
:1038DC00D1450ADA0C2303FB04535B6B13F8090084
:1038EC0004F000FF09F10109F2E70137D3E7894D34
:1038FC000024287DFFF7C2FB2B7D9C4280F06F815A
:10390C00864B0021E65C0C2202FB01F3824800F19D
:10391C003007DA5DB24205D1034493F8380004F065
:10392C00E1FE02E001311C29EDD10134E4E77C4CCD
:10393C001620FFF7A3FBB4F8280104F0E5FEB4F859
:10394C00D40004F0E1FEB4F8D60004F0DDFEB4F8C7
:10395C00D80004F0D9FEB4F86A0104F0D5FE0020BA
:10396C0004F0C0FE002004F0BDFE002004F0BAFEFE
:10397C0094F8170104F0B6FE94F8240104F0B2FE9A
:10398C00002004F0AFFE634B0A201B6FB3F95630D6
:10399C0093FBF0F080B204F0B7FE38E00820FFF79C
:1039AC006DFB0124E0B2013404F09CFE092CF9D12A
:1039BC0015E1002004F0A8FE11E1564C0420FFF79D
:1039CC005DFB236FB3F85A0004F09EFE236FB3F82F
:1039DC005800EFE70C20FFF751FB524B1868FFF72C
:1039EC0023FB514B1868FFF71FFB504B1868F4E092
:1039FC004B4C0620FFF742FBB4F8EC0004F084FEBD
:103A0C00B4F8EE0004F080FEB4F8F000D2E794F8BD
:103A1C000C0104F067FE94F8100104F063FE94F8B6
:103A2C000F0104F05FFE94F811015FE03C4C07209D
:103A3C00FFF724FBB4F8120104F066FEB4F814018D
:103A4C0004F062FE94F8160104F04CFEB4F8180170
:103A5C00B0E7334C0C20FFF711FB94F8220104F073
:103A6C0041FEB4F82C0104F04FFEB4F8280104F028
:103A7C004BFEB4F82A0104F047FE94F8230104F03D
:103A8C0031FEB4F82E0104F03FFEB4F8300191E79A
:103A9C00234C0420FFF7F2FA94F8680104F022FE9C
:103AAC0094F8690104F01EFEB4F86A0182E7204C18
:103ABC00204D2078002600EB4000C0B2FFF7DEFA64
:103ACC00237802359E4280F08A8015F8020C04F0AF
:103ADC0009FE15F8010C013600EB800000EB8000AC
:103AEC0000F2EE2080B204F00FFEE9E704F0FAFDDC
:103AFC0075E00820FFF7C2FA0024094B234493F821
:103B0C001A01013404F0EEFD082CF6D167E000BF79
:103B1C0047D50008D806002048D50008ED0600203F
:103B2C00E8090020E8F7FF1FECF7FF1FF0F7FF1F75
:103B3C00040F00201A0B0020374C1020FFF79EFAC0
:103B4C00607904F0CFFDA068FFF76EFA94F82201BB
:103B5C0004F0C8FDB4F8EC0004F0D6FDB4F8EE00A7
:103B6C0004F0D2FDB4F8F00004F0CEFDB4F812016C
:103B7C0004F0CAFDB4F814011CE7284D264C95F846
:103B8C00740004F11006C0EBC000C0B2FFF776FA67
:103B9C0094F87C0195F9782043B29A4225D01F4ABB
:103BAC0092F984209A4220D00834B44217D0EFE71F
:103BBC000D20FFF763FA002004F094FD0020FFF7BE
:103BCC0033FA06E0164B185D013404F08BFD0B2C18
:103BDC00F8D10020FFF728FA0020FFF725FA012082
:103BEC00BDE8F0870020BDE8F08704F07BFDB4F859
:103BFC007E0104F089FD94F8800104F073FD94F8C3
:103C0C00810104F06FFD94F8830104F06BFD94F8CE
:103C1C00820104F067FDC7E7E8090020D806002000
:103C2C00D8E50008034B1A68D379591C1344D17199
:103C3C00187A7047D806002010B5FFF7F3FF84B24E
:103C4C00FFF7F0FF04EB002080B210BD70472DE9A8
:103C5C00F047054608F069FE314E0446D6F8088058
:103C6C0090B9304804F0C0FD2F4B53F8241049B1E3
:103C7C000123A34013EA080F02D02C4800F088FF60
:103C8C000134F1E72A4822E028462A49224608F066
:103C9C0055FE58B9284804F0A7FD284C54F8041FC9
:103CAC000029EFD0214800F073FFF7E72B784FF095
:103CBC0000092D2B03BF013504F1FF344FF0010A2D
:103CCC004FF0000A184B53F8297027B91C48BDE86F
:103CDC00F04704F089BD28463946224608F02EFEEE
:103CEC00D8B9012000FA09F0020601D51548EEE713
:103CFC008305FBD4BAF1000F03D001F0BFF91248D1
:103D0C0003E040EA0800B060104804F06DFD39464D
:103D1C00BDE8F0470E4800F03BBF09F10109D1E7BF
:103D2C00E8090020DAE60008D4D60008E4E600082A
:103D3C001DEB0008E8E60008EDE60008D0D6000808
:103D4C00F9E6000808E7000816E700081FE7000876
:103D5C007CE8000810B5084804F046FD074B002429
:103D6C001C701C63064B1C7002F0EEFF04F08EFFFF
:103D7C00044B1C6010BD00BF27E70008680700203B
:103D8C00FE160020E016002070B5064600240B4BF2
:103D9C00E518AA8816420AD0E158094800F0F8FE46
:103DAC002846002104F0B9FC064804F01DFD40F63D
:103DBC00C82314349C42EAD170BD00BF70D80008EF
:103DCC0053E700081DEB0008F8B504460E461746ED
:103DDC0000252046202108F09AFD0446D0B101347C
:103DEC00204608F0F7FDB0F5617F05DB40F63403A3
:103DFC009842A8BF184601E04FF46170A0F56170BD
:103E0C00192390FBF3F00DB9307000E070703B7823
:103E1C0001333B700DB90125DBE72046F8BD7FB5BA
:103E2C0004780646E4B9364B1921186800EB840077
:103E3C0090F87B5090F879204D4305F5617590F81A
:103E4C007A30009590F87C00414301F56171019145
:103E5C002C482146013400F09BFE142CE3D14CE09D
:103E6C0008F0B8FD1328054641DC254B701C1C6876
:103E7C00202100238DF80F3008F049FD1E35064631
:103E8C0070B10136304608F0A5FD1A289FBF04EB2F
:103E9C00850358709DF80F30013398BF8DF80F30A3
:103EAC003046202108F033FD064670B1013630460D
:103EBC0008F090FD0D289FBF04EB850398709DF8CA
:103ECC000F30013398BF8DF80F3004EB850430466A
:103EDC00E11C0DF10F02FFF777FF9DF80F30042B5B
:103EEC000BD0601C0021042208F0DBFC05E0064826
:103EFC0006490022132300F04BFE04B070BD00BF36
:103F0C00480700205DE7000872E7000891E7000809
:103F1C00014804F069BC00BF97E700082DE9F041A7
:103F2C00047806467CB9334D2146B5F85621B5F8D0
:103F3C0058313148013400F02BFE042C05F10405F6
:103F4C00F2D1BDE8F0812D4908F0B4FCB0B9294B91
:103F5C004FF47A714FF4FA62A3F85611A3F8582172
:103F6C00A3F85A11A3F85C21A3F85E11A3F8602101
:103F7C00A3F86211A3F86421BDE8F081304608F083
:103F8C0029FD032805462CD83046202108F0BFFC1B
:103F9C00044630B10134204608F01CFD01260746CA
:103FAC0000E006462046202108F0B1FC10B9BDE81F
:103FBC00F041ADE7013008F00DFD012EF7D140F2D4
:103FCC00DC53A7F2EE229A42F1D8A0F2EE229A42EA
:103FDC00EDD8084B543503EB8503DF801881BDE821
:103FEC00F0810748074900220323BDE8F04100F0A7
:103FFC00CFBD00BFE8090020A5E70008B8E700081E
:10400C0072E700080EEE0008F0B5047887B006469B
:10401C0014BB514B19201968062303FB041191F8AA
:10402C00CA5091F8CE20454305F5617591F8C93019
:10403C00009591F8CB50C831684300F56170019040
:10404C00087902904979454803912146013400F0E2
:10405C009FFD0C2CDDD17DE008F0BCFC0B28044648
:10406C0072DC3D4B701C1D68202100238DF817302D
:10407C0008F04DFC064680B10136304608F0AAFC2B
:10408C0003289FBF062303FB045383F8CE009DF83F
:10409C0017309CBF01338DF817303046202108F0C3
:1040AC0036FC074680B10137384608F093FC0D28E2
:1040BC009FBF062303FB045383F8C9009DF81730F8
:1040CC009CBF01338DF8173006266643A919384674
:1040DC00CA310DF11702FFF777FE202108F017FC0B
:1040EC00074670B10137384608F074FC14289FBF9E
:1040FC009DF817307619013386F8CC0098BF8DF8EF
:10410C0017303846202108F002FC78B1013008F055
:10411C0061FC0D289FBF062303FB045383F8CD00DD
:10412C009DF817309CBF01338DF817309DF8173070
:10413C00062B0FD0062202FB04500021C93008F0D8
:10414C00B0FBFFF7E5FE05E00548064900220B230E
:10415C0000F01EFD07B0F0BD48070020BEE70008C8
:10416C0072E7000891E700082DE9F3470478074649
:10417C004CB9204601A901F0BBFC0134FFF7F4FF58
:10418C00122CF6D17EE008F025FCC5B2112D73D8A7
:10419C003E4C05F1980604EB4603781C202193F85D
:1041AC00028008F0B4FB3A4F034630B9A8F1020282
:1041BC00D2F1000848EB020848E007F1580800F17A
:1041CC00010A5978404608F0A2FB68B1032D8CBF58
:1041DC0003230023C8EB0000C0B23B44184490F802
:1041EC005C90B9F1030F02D1FFF792FE4AE0A9F1FE
:1041FC000203D3F1000850464FF0200148EB0308AE
:10420C0008F085FBD8B1B8F1000FEDD0013008F003
:10421C00E1FB40F2ED2380B2984205DD40F6CA0383
:10422C009842A8BF184601E040F2EE20A0F2EE2022
:10423C00192290FBF2F004EB4603D87002E0B8F1BF
:10424C00000FD1D104EB460383F8029004EB460433
:10425C00A3781F4497F85820B8F1000F07D0E178E5
:10426C0019234B430B48294603F2EE2308E0294659
:10427C00094800F08DFC05E008480949002211238B
:10428C0000F086FC02B0BDE8F08700BFE809002012
:10429C00D4D60008DEE70008F0E7000872E7000853
:1042AC000EEE0008F7B50546124C0E4694F90000C8
:1042BC001146A8421A469DF824709DF8203004D06F
:1042CC0094F90C00A84211D10C34207A70B925B1A4
:1042DC00012D0CD10097084801E00848009702F026
:1042EC006FFE20B105712672606000E0002003B003
:1042FC00F0BD00BF500700200044004000380140D2
:10430C00074B5B6B93F90220824201D1981C7047DA
:10431C0093F90A2082420CBF03F10A000020704777
:10432C0068070020F0B5027887B08AB94B4C04F1CD
:10433C0010064B4B94F97C1193F900208A426DD0F6
:10434C0093F90C308B4269D00834B442F1D183E03C
:10435C00002204920592451C08F03CFBC4B260B2EA
:10436C00FFF7CEFF074618B18DF81040012400E08E
:10437C0004462846202108F0CAFA054638B1013512
:10438C00284608F027FB0134ADF81200E4B20026F1
:10439C002846202108F0BBFAA8B3451C284608F093
:1043AC0019FB00222F49D3B251F82210814203D0BD
:1043BC000132082AF6D100232B4A02EB8302526EFB
:1043CC00824220D1022E0FD0032E12D05A1E012E63
:1043DC00D2B204D0042A13D88DF814300EE0042A7B
:1043EC000ED88DF8153009E0052B09D88DF817304B
:1043FC0004E09A1E052A03D88DF816300134E4B275
:10440C000136042EC4D1052C03D807B0BDE8F0400A
:10441C007EE504AB03CB386079601DE094F8810134
:10442C00114B94F8805103EB8000406EB4F87E2160
:10443C00009094F8830103EB850503EB8000406E3C
:10444C00019094F8820103EB80035B6E07480293A2
:10445C006B6E00F09DFB77E707B0F0BDE80900201C
:10446C005007002038D70008D4D60008FFE7000812
:10447C002DE9FF415149044608F01CFA5049002827
:10448C0020460CBF0126072608F014FA4D490028D7
:10449C00204608BF022608F00DFA002808BF0426A3
:1044AC00F10752D5484804F09FF9002004F065F854
:1044BC00464804F099F9464F464804F095F94648A9
:1044CC0004F092F9454CD7F8088054F8041F19B140
:1044DC00434800F05DFBF8E70D46424B53F825408E
:1044EC0054B10123AB4013EA080F03D03E482146D8
:1044FC0000F04EFB0135F0E73C4804F075F921461D
:10450C007B1893F81A3104AA1344394A8A5C013196
:10451C00082903F8102CF3D10023694635488DF88F
:10452C00083000F035FB344804F05EF93348FFF7EF
:10453C00F9FE334800F02CFB4020FFF725FC3148F6
:10454C0004F052F92D48FFF70FFEB20720D52E4884
:10455C0004F04AF92D4804F047F9284804F04EF8C5
:10456C002B4804F041F92548FFF759FC294804F081
:10457C003BF92248FFF748FD274800F009FB1F488C
:10458C00FFF7CCFC1E4800F003FB8020FFF7FCFB80
:10459C0073070FD5214804F027F9214804F024F9BA
:1045AC00164804F005F8164800F0F2FA4FF4807043
:1045BC00FFF7EAFB04B0BDE8F08100BF1EE800087D
:1045CC00D1EC000825E800082BE8000839E80008C1
:1045DC00E80900204BE8000857E80008D0D600088E
:1045EC0067E80008D4D6000875E8000882E80008DF
:1045FC0014EA00088EE8000897E80008BCE40008FC
:10460C001DEB0008A6E80008B3E80008C6E800089F
:10461C00D4E80008DEE80008EDE80008FBE8000834
:10462C000CE900080B4B30B51A465C6B93F838104C
:10463C0001290BD80B464D1C04EBC303E9B29D8832
:10464C002842F5D082F83810981C30BD82F838100A
:10465C00002030BD68070020024B002283F8382070
:10466C00E0E700BF680700202DE9F047877890F855
:10467C0003C0BBB2C7F1640E03EB83065C42C3F10B
:10468C0078001C4D5FFA8EFE7600CCF16408A4B263
:10469C0080B2A3B20FFA83F9B9F1000F04DC002B3E
:1046AC0014BF3B46012300E0734609FB09F25B4350
:1046BC0002FB0CF292FBF3F3434403FB09F30A22D3
:1046CC0093FBF2F333449BB225F8023FB1F8009010
:1046DC004A880A34C9EB020A1AB202FB0AF24FF4F6
:1046EC007A7392FBF3F3A4B24B4484422B80D0D167
:1046FC00BDE8F087A007002010B5447800780022B0
:10470C0040F6C41102FB02F3193B634303F6C413D6
:10471C005343434393FBF1F3034921F81230013225
:10472C00072AEDD110BD00BFBA070020104B043092
:10473C0033F91000B0F5617F05DB40F63303984286
:10474C00A8BF184601E04FF461700A7819235A4348
:10475C0002F28332824208DA4A78534303F28333FB
:10476C008342B4BF0020012070470020704700BF77
:10477C00140900200A4B1B6813F4805F094BB3F932
:10478C00063005D0C089421A934207DD084400E088
:10479C00008A8342B4BF002001207047012070477B
:1047AC00D00F00201409002010B5064B00241C70FB
:1047BC0001F0F4FC044B83F860405C66A3F868409D
:1047CC00DC6610BDD40F00206807002030B510B98E
:1047DC00BDE83040E8E700230D4CD90004F1840219
:1047EC0012F83350854203D00133102BF4D130BD75
:1047FC00084B0A44D86E28B1214491F88540417881
:10480C008C4204D2DA660022A3F868205A6630BDC6
:10481C00D4D600086807002010B540001428A8BFA3
:10482C00142000230949022401F170029C542344F2
:10483C001A441424834202F8014CF3DB0B44FF228C
:10484C0083F870200F20BDE81040BFE768070020F8
:10485C0010B50A4A0A4B11689B6800BF1268914256
:10486C00F7D1084A4FF47A70D2F8884000FB04F272
:10487C00D31AB3FBF4F300FB013010BDE416002097
:10488C0010E000E06807002038B50446FFF7E0FFB1
:10489C000546FFF7DDFF401BA042FAD338BD10B52B
:1048AC0004462CB14FF47A70FFF7EEFF013CF8E7A9
:1048BC0010BD70B540F2DB167043114C4FF4005331
:1048CC0063614FF480432361861E0B25013D15F077
:1048DC00FF050ED0E368304683F40053E360E368D1
:1048EC0083F48043E360FFF7DAFF1920FFF7D7FF6B
:1048FC00ECE7044A044B1A60044A054BDA6070BDBD
:10490C0000100140EFBEADDEF04F00200400FA05B0
:10491C0000ED00E0024A136801331360704700BFDA
:10492C00E4160020024BD3F88C3003B118477047C3
:10493C006807002003681B69184703681B68184741
:10494C00F0B50124B0FBF4F58D4201D34C43F9E7EB
:10495C000026D4B1B0FBF4F504FB1500B4FBF1F464
:10496C001EB9002D01DC002CF3D1092D03F1010E31
:10497C00EFB204DD002A14BF3725572500E030259F
:10498C003D441D7001367346E3E71C70F0BDF0B575
:10499C000124B0FBF4F58D4201D34C43F9E700261A
:1049AC00D4B1B0FBF4F504FB1500B4FBF1F41EB963
:1049BC00002D01DC002CF3D1092D03F1010EEFB217
:1049CC0004DD002A14BF3725572500E030253D446F
:1049DC001D7001367346E3E71C70F0BD2DE9F843FA
:1049EC00089E002B074688461446334614BF4FF0EA
:1049FC0030094FF0200913F8012B0AB9254603E0C2
:104A0C00002CFBDD013CF6E7002D04DD3846494661
:104A1C00C047013DF8E7354624EAE474A01B28445E
:104A2C0015F8011B11B13846C047F7E7BDE8F8830C
:104A3C00014B1868FFF781BFCC020020F8B5074680
:104A4C000C464868002115461E4604F057FC58B128
:104A5C00284604F06BFA104904F0BCFA01464FF0FA
:104A6C007E5004F06BFB60606168304604F0AAF97C
:104A7C000146304604F062FB256806462946384656
:104A8C0004F09EF90146304604F0A4FA014628468B
:104A9C0004F098F92060F8BDDB0FC94030B505462D
:104AAC0087B00C4603A800210C2207F0FAFE28461A
:104ABC00002104F04BFC20B12846284904F082F96F
:104ACC0003E02846254904F07BF9254904F082FAD5
:104ADC0004F046FC054680EAE0706946A0EBE57000
:104AEC0001F006F8002DACBF20232D2368468DF86D
:104AFC000C3007F01AFF012807D130238DF80D3048
:104B0C008DF80E308DF80F300CE0022805D13023D3
:104B1C008DF80D308DF80E3004E0032804BF3023DF
:104B2C008DF80D30694603A807F0E2FE03A807F0E4
:104B3C00FCFE0338C5B22A4603A9204607F020FF25
:104B4C00002363552046074907F0D2FE03AB2046ED
:104B5C00591907F0CDFE204607B030BD6F12033A4D
:104B6C0000007A44EDE9000870B50646B6FBF2F495
:104B7C000846154614B12046FFF7F6FF05FB1464F2
:104B8C00024B1B5D00F8013B70BD00BFEFE9000854
:104B9C000FB42DE9F04F7B4B89B012ACD3F80080E9
:104BAC00794B54F8046BD3F80090049400253178B9
:104BBC00002900F08580252902D00136404673E09B
:104BCC0072784FF0000A302A0CBFB278B71CA2F1F1
:104BDC00300312BF4FF0000BF71C4FF0010B092BE9
:104BEC0019D8A2F13003D9B2092905D80A2202FB3F
:104BFC000A3A17F8012BF4E7A2F16103052B02D84E
:104C0C00A2F1570305E0A2F14103052B03D8A2F151
:104C1C0037030A2BEADD6C2A2FD13A787E1C642AE2
:104C2C0000F088800AD8252A3CD002D8002A47D028
:104C3C00BDE7582A0CD0632A19D0B8E7732A22D0C2
:104C4C0002D86E2A37D0B2E7752A62D0782AAED154
:104C5C00271D2068A2F1580462424FF010016241F6
:104C6C005BE02CD9582A38D0632A34D13E464046D2
:104C7C002178271DC84701350FE0642A69D00ED969
:104C8C00732A14D13E462368404600934946524647
:104C9C000023FFF7A3FE271D05443C4687E7252A82
:104CAC00DFD13E4640462521C84701357FE70ED867
:104CBC006E2A10D13E46236804341D6077E752B942
:104CCC00324B1868FFF736FE0028F9D053E0752AEE
:104CDC0028D0782A01D03E4669E7A2F1580304F1A6
:104CEC00040C5A422068CDF80CC04FF010015A4108
:104CFC0005ABFFF725FEDDF80CC03E46644605AB60
:104D0C0000934046494652465B46FFF767FE054412
:104D1C004DE72068271D0A21002205ABFFF737FE5F
:104D2C003C46ECE704F1040CCDF80CC020680A21D9
:104D3C000022DDE72068271D002808DA2D238DF8D6
:104D4C00143040420DF115030A210022E6E705ABB1
:104D5C00FAE7206804F1040C00280ADA2D238DF8F8
:104D6C00143040420DF11503CDF80CC00A2100227D
:104D7C00BFE705ABF8E7284609B0BDE8F04F04B033
:104D8C00704700BFAC030020A8030020CC02002019
:104D9C0080EAE073A3EBE0738B4206DB002801DDB5
:104DAC00401A704702D0084470470020704770B515
:104DBC00044604F0D5FA2030402857D820462C4918
:104DCC0004F0C4FA28B120462A4903F0F9FF04463E
:104DDC00F4E72046284904F09BFA28B120462549DF
:104DEC0003F0F0FF0446F4E72046244904F0AEFA41
:104DFC0030B12249204603F0E3FF01461F480AE088
:104E0C0020461F4904F084FA40B11C49204603F0A7
:104E1C00D9FF01461A4803F0D3FF04462146204629
:104E2C0004F0D8F805462046294604F0D3F8154975
:104E3C000646284604F0CEF8134903F0C1FF01469C
:104E4C00284604F0C7F8114903F0BCFF0146284678
:104E5C0004F0C0F80E4903F0B3FF0146304604F0ED
:104E6C00B9F80146204603F0ADFF70BD002070BDBF
:104E7C00DB0F4940DB0FC940DB0F49C0DB0FC93FDB
:104E8C00DB0FC9BF9A7C2E36FAAF4F393587083CF9
:104E9C00A4AA2A3E2DE9F04F056885B00C46814640
:104EAC003B49284603F08EFFFFF781FF80462846DA
:104EBC00FFF77DFFD9F8045006463549284603F024
:104ECC0081FFFFF774FF07462846FFF770FFD9F8FC
:104EDC00089005462E49484603F074FFFFF767FF1C
:104EEC0082464846FFF763FF41468146504604F030
:104EFC0071F841468346484604F06CF851460190DF
:104F0C00304604F067F849460290304604F062F8E7
:104F1C0039460390504604F05DF84946206007F18D
:104F2C00004004F057F829466060A560029804F030
:104F3C0051F80146019803F045FF2946E0600398BB
:104F4C0004F048F80146584603F03AFF3946206110
:104F5C0006F1004004F03EF829466061584604F022
:104F6C0039F80146039803F02BFF2946A0610198FC
:104F7C0004F030F80146029803F024FF4146E0614A
:104F8C00384604F027F8206205B0BDE8F08F00BF6A
:104F9C00DB0FC93F2DE9F04107688AB04668856888
:104FAC000446084601A9FFF775FF0199384604F03D
:104FBC0011F804998046304604F00CF8014640463E
:104FCC0003F000FF07998046284604F003F80146D9
:104FDC00404603F0F7FE02992060384603F0FAFFD2
:104FEC0005998046304603F0F5FF0146404603F034
:104FFC00E9FE08998046284603F0ECFF014640463E
:10500C0003F0E0FE03996060384603F0E3FF069975
:10501C000746304603F0DEFF0146384603F0D2FE69
:10502C0009990646284603F0D5FF0146304603F0A1
:10503C00C9FEA0600AB0BDE8F081074B10B51A8814
:10504C001C4622EA00009042188002D00120FFF793
:10505C00E3FB208810BD00BFE4060020064B10B512
:10506C001A881C4610439042188002D00120FFF78A
:10507C00D3FB208810BD00BFE4060020024A9368D1
:10508C0023EA000090607047E809002008B5104B37
:10509C001A780023D9B2914207D20E49002051F858
:1050AC002310013309680880F4E73220FFF7F7FB7F
:1050BC00094B1B685A0309D5084B9B685B0305D445
:1050CC00BDE8084040F2DC50FFF7E9BB08BD00BF6B
:1050DC007B100020A0100020D00F0020E809002039
:1050EC002DE9F7434D4F4E4A4B233B706923137008
:1050FC004FF4A3635380BE231371EF2382F816354C
:10510C0000231946164682F81735F25C0133B3F5C5
:10511C00A36F81EA0201F8D1414B424A83F817157B
:10512C00414B4FF004085A6002F188325A6000205B
:10513C0008F1FF3818F0FF085ED03B4B34223B4C93
:10514C00DA6004F17849A9F57849C9F3090353B138
:10515C0000234FF4005056F80990019300F0E0FD45
:10516C000428E5D11CE04FF4302000F0D9FD0428D0
:10517C00DED12D4D4FF430202B6943F002032B610F
:10518C006C612B6943F040032B6100F0C9FD41F6C3
:10519C00FD732A69042803EA02032B61D8D0C7E700
:1051AC00214D4FF400502B6943F001032B611FFA82
:1051BC0089F3238000F0B4FD042813D1A31C0193C0
:1051CC00019B4FEA1949A3F800904FF4005000F0EE
:1051DC00A7FD41F6FE732A69042803EA02032B613A
:1051EC0006D0A5E741F6FE732A6913402B619FE7B1
:1051FC000F4B04349C42A4D10B4A0428136943F08E
:10520C008003136102D102F0E9F910B90A20FFF70B
:10521C0050FB02233B7003B0BDE8F083F105002086
:10522C00E8090020230167450020024000F800082F
:10523C0018FD000810B50E4C2068FFF75DFA2068C9
:10524C000022047A02FB02F3193B634303F6C413F6
:10525C005343192193FBF1F3064921F81230013223
:10526C00072AEFD1BDE810400349FFF7FDB900BF95
:10527C004407002000020020BC0A00202DE9F8435E
:10528C0002F0ACF910B90A20FFF713FBAD4CAE4E8F
:10529C004B23AE494FF4A3622046337007F0F6FA65
:1052AC0094F8F0344FF48E71022B84BF002384F8F1
:1052BC00F03494F8F024A64D01FB02F3E01800F54D
:1052CC00CE702344286093F8F00101FB02420228BF
:1052DC0003F5F47384BF0020187292F8F0319D4AE4
:1052EC0013700C2202FB03439B4A03F2F24313603C
:1052FC0046F20902A3681A401AB9924A43F40053C1
:10530C009360A368D80703D54FF40050FFF7B6FE9F
:10531C00A368590409D50820FFF7B0FE4FF40050DC
:10532C00FFF7ACFE0120FFF7A9FEA3681A0706D50C
:10533C004FF40050FFF7A2FE0120FFF79FFEA36879
:10534C009B0413D54FF40040FFF798FE7D4B93F868
:10535C001631012B03D14FF40060FFF78FFE4FF491
:10536C008030FFF78BFE4020FFF788FE94F8702109
:10537C00744B2AB193F8742112B1002283F8742172
:10538C004FF00008C646754F754B1F6004EB0803C1
:10539C00B3F87EC14FEA5C0101F077314FEA9C0310
:1053AC0003F03333C1EB0C00C11A4FEADC0303F0FA
:1053BC001133CB1A03EB231303F00F32FF2392FBB1
:1053CC00F3F31CF00109C3EB032318BF0EF1010E1C
:1053DC00A2EB030318BF5FFA8EFE012B0ADD022B32
:1053EC0040F0AD80B9F1000F00F0A9801CF0BC0FAB
:1053FC0000F0A58008F10808B8F1100FC6D10EF125
:10540C00FF3EBEF1010F00F29A80FFF713FF00215F
:10541C003022544807F045FADFF89491524BD5F8F6
:10542C000080C3F80090514B08F17900C3F800805C
:10543C0000F032FB4E4B80F0010018704D4B09F11F
:10544C0026021A6098F8000001F00EFD4A4B94F801
:10545C00681109F194021A6064224A43474BC8321E
:10546C005A6000229A60DA601A615A619A61DA61B4
:10547C0083F8202083F82120414B09F12C021A607B
:10548C00404B09F108021A603F4BDFF82881C3F842
:10549C0000903E4B09F1A0021A6009F1A403C8F870
:1054AC0000303B4BB4F8F6001F6003F03BFDC8F82E
:1054BC000800B4F8F80003F035FD2D6808F104027B
:1054CC0095F85C30C8F80C0088F8043095F8783002
:1054DC00286E88F8053094F87331C8F8145088F8A1
:1054EC0010302C4B2C491A602C4B05F164021A60BD
:1054FC0003F070FD01464FF07C5003F01FFEB5F831
:10550C001641274B1860204603F010FD0146254834
:10551C0003F014FE244903F05DFD244BC8F8185029
:10552C00186005F16803C8F81C30022305F2111548
:10553C003370C8F82050C8F82490BDE8F88300F008
:10554C0089FA62E7E8090020F105002000F800085C
:10555C0048070020C016002044070020020B002042
:10556C00CC0F002098060020CC060020D00600208E
:10557C001C000020D8000020BC160020981600202B
:10558C00400100207011002074110020D80200206E
:10559C009C03002070010020DB0F4940A801002073
:1055AC00A4010020000061444C3D0F44D4020020B3
:1055BC00BC0A0020F807002008B5FFF791FDFFF7A3
:1055CC005DFEBDE808400120FFF726B9084BDA68FC
:1055DC00D10709D4DA68520708D4DB6813F0100F2E
:1055EC0014BF03200420704701207047022070472D
:1055FC000020024003788B4286BF024B33F8110027
:10560C0000207047200800200022134670B5234963
:10561C0014180C44247E83EA0423082413F4004F4A
:10562C004FEA430318BF83F4815304F1FF3418BFCE
:10563C0083F0010314F0FF049BB2EFD10132192A5D
:10564C00E5D100F1190200F11A050A440D44167E49
:10565C002A7E02EB062292B29A421ED10F4B93F88D
:10566C003950E2B2AA4215D2431C03EB4203DBB21F
:10567C00CA1801330B44127E1B7E03EB02239BB230
:10568C004FF4AF6253431B1303F5487321F81430E6
:10569C000134E6E7012381F83A3070BD2008002080
:1056AC0003788B420BD9074B890093F83B201944A4
:1056BC00C86B02B1400800F5777080B270470020CB
:1056CC00704700BF2008002007299DBF034B03EB48
:1056DC008101B1F86C000020704700BF2008002049
:1056EC00034B03EB4101B1F88C00C008704700BFBD
:1056FC002008002008B5084B03EB8101D1F8AC0061
:10570C0003F010FC054903F065FC054903F05AFB56
:10571C0003F04CFE80B208BD200800200000203FA2
:10572C0000005C44024B03EB4101B1F8F4007047FC
:10573C0020080020024B03EB4101B1F8180170471F
:10574C0020080020024B03EB4101B1F8180170470F
:10575C00200800200020704710B50446FFF778F8A9
:10576C0041F288310E4BE4B2D3F83021C3F830014A
:10577C00821A8A42C3F8342184BF002283F838216C
:10578C0093F8382106490F2A134418BF013283F8C5
:10579C00394112BF81F83821012381F8493110BDFC
:1057AC002008002070B50546FFF752F8314CD4F8AC
:1057BC004C31C4F84C01C31AB3F5FA5FC4F850313C
:1057CC0082BF002384F8543184F8553194F8543155
:1057DC002BB9A12D02BF274A012182F8551194F84B
:1057EC005511244A29B1D118EDB201330D7682F846
:1057FC00543194F8545194F85631AB4239D11D4B75
:10580C0093F85731052B02D0062B03D02CE0002047
:10581C00FFF7FAFE637E1E2B26D100200246C1B292
:10582C006B1E994219DA21440B7E0821DBB283EA04
:10583C000206F60744BF83F01803C3F3460301F1D5
:10584C00FF3154BF5B0843F0800311F0FF01C2F33A
:10585C004702ECD101301A46E1E723441B7E9A4201
:10586C0002D10320FFF7D0FE002384F8553184F8D1
:10587C00543170BD2008002010B50446FEF7E8FF37
:10588C0041F288310E4BD3F85821C3F85801821AD3
:10589C008A42C3F85C2184BF002283F8602193F80C
:1058AC0060210749142A134418BF013283F861415F
:1058BC0012BF81F86021012381F8763110BD00BF41
:1058CC002008002038B50446FEF7C2FF274A2749B6
:1058DC00D2F87831C2F87801C31AB3F57A6F84BF65
:1058EC00002382F87C3192F87C3133B9A82C3BD15F
:1058FC0081F87D31A1F87E3106E0022B02D181F8CE
:10590C00804101E0242B02D8D11881F8814192F812
:10591C00801101330231DBB249008B42134D82F806
:10592C007C3118DAB5F87E31E0B283EA0020082326
:10593C0010F4004F4FEA400018BF80F4815003F17F
:10594C00FF3318BF80F0010013F0FF0380B2EFD1DA
:10595C00A2F87E0138BD01318B4201BF002385F8CE
:10596C007C31012385F87D3138BD00BF2008002033
:10597C0010B50446FEF76CFF40F6AC510F4AD2F856
:10598C00A831C31A8B42C4BF002382F8AC3192F801
:10599C00AC31D11881F8AD4123B90F2C0DD1074989
:1059AC00C1F8A8010133DBB2192B044982F8AC31E0
:1059BC000CBF0123002381F8C63110BD2008002044
:1059CC000C4B0D49DA684378D243C2F30222C2F180
:1059DC000402934002781B01DBB20A4482F80033C4
:1059EC0003780122580903F01F0302FA03F341F86C
:1059FC002030704700ED00E000E100E073B5054693
:105A0C0000210068012202F005F82A68012413889D
:105A1C0000269BB243F001031380EB7A01A88DF8AA
:105A2C0004308DF805408DF806608DF80740FFF7BF
:105A3C00C7FFEB7A1B2B0BD1192301A88DF804306F
:105A4C008DF805408DF806608DF80740FFF7B8FF1C
:105A5C0002B070BD10B50F4C0021122204F242307E
:105A6C0006F01FFF0523042184F8483384F84A33D9
:105A7C0084F8503384F852335223012284F84913AA
:105A8C0084F8511384F8423384F84C23A4F8462349
:105A9C0010BD00BF2008002000F1500302781AB995
:105AAC008178C278914204D304309842F6D1002018
:105ABC0070470120704770B50646441E14F8011F4C
:105ACC0089B1094D284606F022FF0028F6D005F1D1
:105ADC00080398423FBF054B401BC018A31B38BF9F
:105AEC0080F8E232EAE770BD14EA000820080020D2
:105AFC00031EB8BF2D2210B5B8BF58420C46B8BF14
:105B0C0001F8012B0A22FFF72FF80023037020461F
:105B1C0010BD07B51B4B03F2E462C3F8E02693F803
:105B2C00EA225AB1012A14D1032183F8E61607217F
:105B3C0083F83B2083F8E7160C2208E0022183F857
:105B4C00E616032183F83B2083F8E716072283F837
:105B5C00E4260D4A0D4B40201A60FEF77DFD70B116
:105B6C000122002390F9000040218DE80C00084A26
:105B7C004FF4E133FEF796FB003018BF012003B061
:105B8C005DF804FB20080020AD5600082000002022
:105B9C006557000801200021FDF750BA4FF6FE733F
:105BAC000268134003600023036043608360C3609A
:105BBC00284B984201D1284A27E0284B984201D122
:105BCC00254A2AE0264B984201D1234A2DE0254B49
:105BDC00984201D1204A30E0234B984201D11E4A11
:105BEC0033E0224B984204D11B4A536843F47003B0
:105BFC002EE01F4B984204D1174A536843F0706350
:105C0C0026E01C4B984204D11B4A536843F00F0307
:105C1C001EE01A4B984204D1174A536843F0F00324
:105C2C0016E0174B984204D1134A536843F470633F
:105C3C000EE0144B984204D10F4A536843F470435E
:105C4C0006E0114B984204D10B4A536843F470237D
:105C5C005360704708000240000002401C000240E4
:105C6C003000024044000240580002406C000240E8
:105C7C008000024008040240000402401C04024060
:105C8C003004024044040240580402401F4A10B53C
:105C9C00536803F00C03042B03D0082B04D01C4BCB
:105CAC0014E01C4B5B6811E053685168C3F38343E9
:105CBC00C90303F1020301D4174906E0516811F43A
:105CCC00003F1449496818BF49084B4303605368A7
:105CDC001249C3F30313CC5C0368E340436054687C
:105CEC00C4F302240C5D23FA04F484605468C4F3F6
:105CFC00C2240C5DE340C3605268C2F381320A4493
:105D0C00127CB3FBF2F3036110BD00BF0010024024
:105D1C0000127A002000002000093D0034D8000851
:105D2C0010B50446FFF752FC012806D11CB1FFF751
:105D3C004DFC013CF8E7052010BD002C08BF0520E8
:105D4C0010BD0F4B1A6842F001021A6059680D4AD7
:105D5C000A405A601A6822F0847222F480321A6067
:105D6C001A6822F480221A605A6822F4FE025A60E1
:105D7C004FF41F029A60044B4FF000629A60704718
:105D8C00001002400000FFF800ED00E02DE9F843A0
:105D9C005B4C0368013AC4F8E83683880D46A4F8D6
:105DAC00EC36072A42D8DFE802F0040A1018222940
:105DBC002F35B4F8E8360B80B4F8EA3613E0B4F8B3
:105DCC00EA360B80B4F8E83605E0B4F8E8365B4206
:105DDC000B80B4F8EA365B4205E0B4F8EA365B4275
:105DEC000B80B4F8E8366B80B4F8EC361DE0B4F8F0
:105DFC00E8365B420B80B4F8EA3612E0B4F8EA36C7
:105E0C000B80B4F8E8360CE0B4F8E8360B80B4F844
:105E1C00EA3605E0B4F8EA365B420B80B4F8E836B3
:105E2C005B426B80B4F8EC365B42AB80354B1B7A33
:105E3C00002B62D1B5F9000003F078F88046B5F973
:105E4C00020003F073F80746B5F9040003F06EF88E
:105E5C00D4F8F0160646404603F0BCF8D4F8FC160D
:105E6C008146384603F0B6F80146484602F0AAFFD0
:105E7C00D4F808178146304603F0ACF80146484682
:105E8C0002F0A0FF06F06CFED4F8F4162880404611
:105E9C0003F0A0F8D4F800178146384603F09AF8BE
:105EAC000146484602F08EFFD4F80C178146304666
:105EBC0003F090F80146484602F084FF06F050FECD
:105ECC00D4F8F8166880404603F084F8D4F8041728
:105EDC008046384603F07EF80146404602F072FFD9
:105EEC00D4F810170746304603F074F801463846CC
:105EFC0002F068FF06F034FEA880BDE8F88300BF0E
:105F0C00200800202000002044F6FB71084BD3F839
:105F1C001427137803EB431300FB03135078C0EBE7
:105F2C000030B3FBF0F39078B3FBF0F080B2704725
:105F3C00200800202DE9F84F774C0023B4F92227D4
:105F4C00A4F818370A2A18BF84F8203794F8206769
:105F5C00714B002E66D1714A03F5E465C3F8242712
:105F6C00C3F82C274FF07E52C3F830276C4AA84652
:105F7C00C3F834276B4A6C49C3F8382740F2DC521B
:105F8C00C3F874271022A3F872271822C3F8281715
:105F9C00A3F8702708EB06074FF09741386903F018
:105FAC0019F80021814603F0B3F928B148464FF0A7
:105FBC007C5102F005FF04E048464FF07C5102F0A2
:105FCC0001FF03F02FFAC5E90E0178684FF09741F5
:105FDC0003F000F80021074603F09AF928B138467F
:105FEC004FF07C5102F0ECFE04E038464FF07C514F
:105FFC0002F0E8FE03F016FA04360C2EC5E908018F
:10600C0005F10805C6D10A23A4F82237474BC4F87A
:10601C009037C4F89C37C4F89437C4F8A0370123E0
:10602C0084F82037DFF808C1D4F87487B4F97257B4
:10603C00DCF82430C8F10006AE407343DCF8207065
:10604C004FEAE67BD4F890E707FB0B33C4F8906774
:10605C00A7FB0667D4F89C271F44DCF84430DCF817
:10606C0040A053434FEAE27BD4F8A0070AFB0B395C
:10607C00C4F8A027AAFB02234B44B61A67EB03070C
:10608C00DCF82C30DCF828200EFB03F34FEAEE7B17
:10609C0002FB0B39A2FB0E23B6184B445F41DCF814
:1060AC004C30DCF8482043434FEAE07B02FB0B39D1
:1060BC00A2FB0023D4F89417B21ADCF83460C4F8AD
:1060CC00A40701FB06F6DCF830004B4467EB030336
:1060DC00CF17C4F8981700FB0766A0FB01018018C6
:1060EC003144C4F894E75941B4F9702702F056FED4
:1060FC006A1E01239340C4F89C07C01841EBE3715E
:10610C002A4602F04BFE10EB080080B2FFF7FCFEB3
:10611C00A4F8A807BDE8F88F2008002056157D3993
:10612C006350FABF0CE0743F5615FD39000024FA99
:10613C00400F002070B512494300D1F8AC270E4631
:10614C00D418257E15B1022D10D00BE0022805D9EC
:10615C00032807D1D1F8B037DB0401D5D08970BD45
:10616C00908A70BD3344B3F8F40070BD607E00EBD0
:10617C00800000EB800000F2EE2080B270BD00BF0A
:10618C002008002042F20102034BD3F8B0371A4228
:10619C000CBF01200020704720080020104B10B5C8
:1061AC0093F8B4271C46012A0DD007D3022A0ED12E
:1061BC000C4AD36883F48043D36008E0094B4FF456
:1061CC0080421A6103E0074B4FF480425A61FEF79C
:1061DC003FFB00F5F42000F59070C4F8B80710BD33
:1061EC0020080020001001402DE9F04F87B00393E8
:1061FC00904B07461B8893469B0736D540F2E632F8
:10620C00109B8D48DC89B0F900301B1B03F2F31591
:10621C00954203D8002BB8BF5B4201E04FF4FA73F0
:10622C00B0F9022040F2E630121B02F2F314844261
:10623C0003D8002AB8BF524201E04FF4FA729342DD
:10624C00B8BF13460522C3F5FA7393FBF2F30A2287
:10625C00643B53433A7FD2105343642293FBF2F3D3
:10626C00134423EAE373DBB200E06423B8460093E3
:10627C00CB1C02930025029B022D13F8010F4FEA51
:10628C00450A02936D4B06D1B3F9046000F11B046F
:10629C00744362112EE033F91510CBF100024C005F
:1062AC00944203DB5C452246A8BF5A46644C34F941
:1062BC000A40121B039C34F9156016445D4AB2F86F
:1062CC0000E01EF0010F12D100F11B044C431EF034
:1062DC00020F4FEA24120DD0BC7C9DF900007443D0
:1062EC004443642194FBF1F102EB211202E03A7A6F
:1062FC00724312115349042431F90A1098F801C061
:10630C0091FBF4F44D4E141B0CFB04FC06F108023B
:10631C00AA5C97F8519002FB0CFC019264229CFB46
:10632C00F2FC4FEAEC1CB9F1000F20D0022D10D179
:10633C006046049302F0FAFD5FEA5901049B04D015
:10634C0049450A46A8BF4A4600E001223E495B6A1D
:10635C0008E0604602F0EAFD4A4606F10C01736A59
:10636C0001EBC501FEF76AFB02F0FAFF8446374BDE
:10637C0098F80B601988314B01FB04F203F1280EDD
:10638C005EF82500D21206FB0206314AB6F5001F54
:10639C00A8BF4FF40016964203F13400B8BF16465E
:1063AC0050F8252040F825404FF6FF700909B0FB46
:1063BC00F1F1A21A4A4303F1400103F14C044EF8E7
:1063CC00256051F825E054F8250044F825E097F8AD
:1063DC005040921170447613104441F825208CB132
:1063EC00CDF810C0059302F0A1FD059B224603F1E8
:1063FC00580101EBC5015B6AFEF720FB02F0B0FF10
:10640C00DDF810C098F8153066445843019B4FF0E6
:10641C00640C434393FBFCF001350E4B06EB202040
:10642C00032D23F80A0008F101087FF424AF07B00C
:10643C00BDE8F08FE406002014090020E00F0020D6
:10644C00320700200E070020FC0F0020DC06002085
:10645C000000E0FF501000202DE9F04F89B00593AB
:10646C00B74B0026B3F90290B3F90030B9F1000F25
:10647C00B8BFC9F10009002BB8BF5B429945B8BF42
:10648C0099460746B2463446B9F5FA7F0491039211
:10649C00A8BF4FF4FA79019000960296A94B188880
:1064AC0010F003053AD0A64B610033F91420039B7E
:1064BC0052005B429A4203DB039B9342A8BF1346F4
:1064CC00A14A6FF0040A895E059A5B1A32F914101E
:1064DC00642219443B7A4B4393FBF2F33A7F0AFB59
:1064EC0002FA534504DB02EB820A9A45A8BF9A468E
:1064FC00964A52F82430194442F210739942A8BFBC
:10650C001946934B9942B8BF1946BB7C42F82410EC
:10651C005943012D4FEA2133029338D08849A60004
:10652C0031F9143028310093019B51F824E093F891
:10653C0001C0884B33F9145085EAE573A3EBE5737E
:10654C00B3F5206F16DC009A50235A4392FBFCF3F0
:10655C00042295FBF2F55D1BAE44BEF57A5F7E4BD3
:10656C00A8BF4FF47A5E9E45ACBF41F824E041F8D9
:10657C00243002E0002341F824308B597D2693FB14
:10658C00F6F6019BDB7A7343402693FBF6F6820703
:10659C0012D5009A09FB06F509FB02F80298C9F519
:1065AC00FA7303FB0A8803FB00534FF4FA7198FB50
:1065BC00F1F293FBF1F505E0C30755BF35465246A2
:1065CC00009A029D634B4FF0040833F914304FEAE4
:1065DC00440B93FBF8F85A4B03F18001615C01FB0F
:1065EC0008F86FF04F0198FBF1F8904497F85120A0
:1065FC0082B140460793069202F098FC079B069ADC
:10660C0003F10C0101EBC4015B6AFEF717FA02F00F
:10661C00A7FE80464F4B3BF80300494B02B203F1F7
:10662C0084013BF901E02BF80100CEEB02024FF0A4
:10663C00040E92FBFEF203F1880103F1900E51F867
:10664C0024C05EF8240041F824206044104497F8DC
:10665C0050204EF824C072B10793069202F066FCEB
:10666C00079B069A03F1580101EBC4015B6AFEF724
:10667C00E5F902F075FE324A454402F1980111F831
:10668C00048002F1700308FB00F04FF0200890FB2F
:10669C00F8F02D1A2BF80350019B013301930CB920
:1066AC000124FBE6049BB2F904109B7904200F3300
:1066BC005B004B4327495B11B1F90410002B91FB94
:1066CC00F0F0A3EB0000B8BF5B42322B146B797B6C
:1066DC000BDC01FB0041214B8B42A8BF0B46204930
:1066EC008B42ACBF1363116301E000231363F97891
:1066FC0001FB00F392F89B109B1103290CD9B7F8FE
:10670C004E10B1F5FA7F07D24842834203DB8B422D
:10671C00A8BF0B4600E00346116B6FF0FF0041F37E
:10672C004F31B1F5807FA8BF4FF480718142ACBF6F
:10673C005B181B18A2F8743009B0BDE8F08F00BFCD
:10674C00E00F0020E4060020320700205810002043
:10675C00F0D8FFFF0E07002080C1FFFFFEFFFF0FE8
:10676C00020000F02DE9F04F054690F850008DB076
:10677C000A9107920B9318B13228A8BF322000E07F
:10678C00012002F0D3FB01469B4802F0D7FC9B4B47
:10679C0004461888002808BF012002F0C7FB98495E
:1067AC00089002F017FC01900199204602F00AFBB8
:1067BC000146019802F0C2FC924B09901B88980785
:1067CC0024D59149B1F90030B1F9020083EAE372A2
:1067DC0080EAE071A2EBE372A1EBE07191420C460E
:1067EC00B8BF1446B4F5E17F12DA914203DD0028FC
:1067FC00D8BF404203E0002BCCBF1846584202F0F1
:10680C0095FB824902F09AFC064603E0002601E063
:10681C004FF07E564FF0000904950024CDF80890F7
:10682C00630006937A4B33F814800FFA88F002F069
:10683C007DFB784902F0CEFB02F092FD02F076FB74
:10684C00754902F0C7FB704B039033F9140002F04A
:10685C006DFB6C4B07461B889907059362D001466C
:10686C0002F0B0FA02F07CFD079B5B42984203DB1E
:10687C00079B8342A8BF03460699684A885E0B9A19
:10688C001B1A32F91400184402F050FB8246287F80
:10689C0002F048FB624902F09DFB8346287A02F025
:1068AC0041FB0146504602F095FB5E4902F092FB1B
:1068BC0002F056FD81460BF1004002F051FD81457E
:1068CC0005DB584602F04CFD4845A8BF484602F08F
:1068DC002DFBDFF8749102900199504602F07AFB7F
:1068EC0059F8241002F06EFA4F494FEA840B824695
:1068FC0002F00EFD38B950464C4902F027FD20B18C
:10690C00DFF828A101E0DFF820A149F80BA0A87C52
:10691C0002F008FB0146504602F05CFB444902F0D1
:10692C0059FB8146059BDA0700F190800FFA88F835
:10693C00B8F1000FB8BFC8F10008B8F5206FDFF848
:10694C0000A14FEA840803DD00234AF8243028E034
:10695C003849384602F03EFB049B8346587802F0D7
:10696C00E1FA0146584602F0E9FB039902F028FAD5
:10697C00019902F02FFB5AF8241002F023FA2E4949
:10698C00824602F0C5FC38B950462C4902F0DEFCB8
:10699C0020B1DFF8A8A001E0DFF89CA0284B43F859
:1069AC0008A0049BD87A02F0BDFA254B53F82410AA
:1069BC0002F010FB234902F00DFB059B80469B0760
:1069CC0046D53846029902F0FBF90146304602F0F2
:1069DC0001FB0146029802F0F5F94946074640468C
:1069EC0002F0EEF90146304602F0F4FA0146484650
:1069FC0002F0E8F980462BE083F9223EDC06002009
:106A0C00BD378635E4060020E00F00200000E1438E
:106A1C000E0700200000A03ECDCC4C4032070020D9
:106A2C000000A0406F12033C0000F0C10000F041D8
:106A3C000AD7A33D0000A043000040C30000404320
:106A4C00841000200AD7233C7C100020C846029FEB
:106A5C00DFF8E8A10AF18003185D02F067FA01463D
:106A6C00039802F0B7FA744902F0B4FA01463846BA
:106A7C0002F0A6F995F85120834642B10AF10C01B7
:106A8C0001EBC401DAF82430FDF7D8FF83466B4FD5
:106A9C00039807F1B00A5AF8241002F091F9019901
:106AAC0002F04CFB039B4AF8243007F1B80353F86F
:106ABC0024A00393514602F083F90146099802F091
:106ACC0089FA0146504602F07DF9039B414643F892
:106ADC0024008246584602F075F907F19803804667
:106AEC00185D02F023FA0146504602F073FA54493D
:106AFC0002F070FA0146404602F062F906F030F8F6
:106B0C00069A07F170039852049B013304930CB955
:106B1C00012485E60A9AB7F9043094796400283484
:106B2C005C43484B6411B3F9040002F0FFF94FF0D9
:106B3C007A5102F04FFA06F013F8201A02F0F6F927
:106B4C00002CB8BF6442322C064602DD00233B63A6
:106B5C0024E0089802F004FC20F0030002F0E6F9AF
:106B6C008046687B02F0DEF90146304602F032FACC
:106B7C0035490446404602F0E1FA0146204602F04F
:106B8C0029FA02F0EDFB3B6B1844304B9842A8BF3E
:106B9C0018462F4B9842ACBF38633B633B6B6FF08E
:106BAC00FF005B13B3F5807FA8BF4FF4807398424E
:106BBC00B8BF184602F0BAF90446304602F0D0FBD2
:106BCC00EB785843801102F0B1F997F89B200346FB
:106BDC00032A11D9B5F84E60B6F5FA7F0CD202F043
:106BEC00BFFB7342984203DBB0420346A8BF334657
:106BFC00184602F09BF9034695F8512062B15108F2
:106C0C0003D08A42A8BF0A4600E001221846114967
:106C1C007B6AFDF713FF03461846214602F0D2F8B3
:106C2C0002F09EFB00B202F081F905F099FFA7F883
:106C3C0074000DB0BDE8F08FA69B443BE00F002024
:106C4C00F7CC92380E07002000803B45FEFFFF0F6B
:106C5C00020000F0FC0F00202DE9F8430024254B26
:106C6C00E0B293F89B60B0420DD203EB8003224A52
:106C7C00D3F8C03032F810101BB10B2801D8DB68E8
:106C8C0098470134EBE71D4B1B685B032FD50024A1
:106C9C002346E2B2B2422AD2DFF858904FEA840877
:106CAC0009F1C00757F8242055689D4217D0284693
:106CBC0000F004FFEFF31283502282F31288282194
:106CCC00AA8C01FB009092B20132C0F81421AA8A5E
:106CDC00DBB292B242F00102AA8283F3118857F818
:106CEC00083000221B6801341A802B46D1E7BDE81E
:106CFC00F88300BFE00F00201A070020D00F0020FF
:106D0C0008B50E4B1B6813F4805F0D4B14BFD3F802
:106D1C009021D3F8942193F89B1092880023D8B239
:106D2C00884204D2074820F813200133F7E7FFF715
:106D3C0093FFBDE808403220FDF7B1BDD00F002015
:106D4C00E00F00201A0700200A4B30B51A680A4BD6
:106D5C0002F48052D3F89041D3F8945100230AB135
:106D6C00A18800E0A988054820F8131001330C2BEA
:106D7C00F5D130BDD00F0020E00F0020C21600204E
:106D8C002DE9F74F334C0546D4F898713249384603
:106D9C0002F018F8FEF70BF806463846FEF707F82F
:106DAC00D4F89C7181462C49384602F00BF8FDF75B
:106DBC00FEFF01903846FDF7FAFFD5F804A0074610
:106DCC003146504602F006F9D5F80880834649460C
:106DDC00404602F0FFF80146584601F0F1FF019BD6
:106DEC0029688346184602F0F5F849460546504690
:106DFC0002F0F0F8394602F0EDF80146284601F0B1
:106E0C00E1FF39460546404602F0E4F8314602F00F
:106E1C00E1F80146284601F0D5FF0146584605F039
:106E2C002BFF0E4902F0D6F80D4902F087F9D4F881
:106E3C00A01101F0C7FF0B4902F080F905F090FE9C
:106E4C0083B21A0444BF00F5B47083B218B203B015
:106E5C00BDE8F08FE00F0020DB0FC93F0000E144DC
:106E6C00DB0F49400000204101380A4B042804D8AC
:106E7C00DFE800F00507090B0D00074A08E0074A98
:106E8C0006E0074A04E0074A02E0074A00E0074A26
:106E9C001A60704730000020C17E0008F5610008C0
:106EAC0071810008017C00086564000871670008A6
:106EBC00F0B5046D8279A389467923F4005312F05E
:106ECC00020F4FEA03434FEA13430CBF00214FF468
:106EDC00005112F0040FA38114BF4FF4806E4FF0D9
:106EEC00000E16F0010F8768054614BF0420002021
:106EFC00B307238A48BF40F008029BB223F44053E7
:106F0C0043EA01032382A18948BF90B289B221F4DC
:106F1C00B05121F00C014EEA010140EA0102A281BC
:106F2C00A38A87B023F440731B041B0CA38201A813
:106F3C00FEF7ACFE049E039B204A944218BF1E46EB
:106F4C00A389192272431BB2002BB4BF7E00BE0072
:106F5C00B2FBF6F66427B6FBF7F00001010907FB5C
:106F6C001163A28912B2002AADBF1A01D9003231C5
:106F7C003232ABBFB2FBF7F3B1FBF7F203F00F0306
:106F8C0002F00702B4BF104318432A6DAB7980B2EC
:106F9C00208113F0080F938A0BBF23F008039BB2D8
:106FAC001B0443F0080308BF1B0C938293899BB20C
:106FBC0043F40053938107B0F0BD00BF003801408B
:106FCC002DE9F3411D468C4B8846984217469DF897
:106FDC00206051D1894B8A4A8A491A608A4A59637E
:106FEC005A6102F580729A614FF48072DA601A610C
:106FFC00864A9F601A63A2F54842543ADA649A644E
:10700C001865834B31079A6942F480429A615A6938
:10701C0042F001025A614FF002038DF803304FF435
:10702C000073ADF8003001D51C230FE0AA0706D57C
:10703C001823784869468DF80230FAF719FBEB07EC
:10704C000AD54FF48063ADF8003048237148694687
:10705C008DF80230FAF70CFB0E238DF80430002269
:10706C00012301A88DF805308DF806208DF8073026
:10707C00624CFEF7A5FC4DE0674B984240F0B8809F
:10708C00664B5F4A9F601A604FF48072DA601A6137
:10709C00634A18655A6102F580729A61614A340735
:1070AC009A64DA645A4BDA6942F40032DA615A694A
:1070BC0042F001025A614FF002038DF803304FF099
:1070CC000403ADF8003001D51C230EE0A80706D54B
:1070DC001823504869468DF80230FAF7C9FAE907C7
:1070EC0009D50823ADF8003048234A4869468DF885
:1070FC000230FAF7BDFA26238DF804300022012362
:10710C0001A88DF805308DF806208DF80730FEF7B4
:10711C0057FC424C012384F8443000232362E36182
:10712C00A3626362C4F82C806571A760A6712046C7
:10713C00FFF7BEFEEA072AD5206B00B3E76CD4F844
:10714C000C806669FEF72AFD236B216D1A6822F408
:10715C00FF4222F0700242F485521A60C3F8048098
:10716C009F60DE601A6842F001021A608A8A92B24D
:10717C0042F040028A825B689BB2236407E04FF6C0
:10718C00DF72236D1A80DA6842F02002DA60AB07F6
:10719C0026D5606BF8B1A56C2669FEF7FFFC636B16
:1071AC001A6822F4FF4222F0700242F4845242F038
:1071BC0010021A6000225E609D60DA60196841F06E
:1071CC00020119605A605A60226D938A9BB243F097
:1071DC008003938204E0226DD36843F08003D36074
:1071EC00226D204693899BB243F40053938100E0B7
:1071FC00002002B0BDE8F08100380140D815002015
:10720C0048D8000844000240841100205800024075
:10721C00001002400008014000440040841500208A
:10722C0084130020044400407B4B10B51B78012BC9
:10723C0014BF00240324038C91BB23F001031B0413
:10724C001B0C0384018B038C89B221F0F30141F0F8
:10725C00010141EA0411714C9BB2A04212D004F519
:10726C000064A0420ED0B0F1804F0BD0A4F598343E
:10727C00A04207D004F58064A04203D004F58064DA
:10728C00A04202D123F0020301E023F00A0343F0F1
:10729C0001031A4301830284038B23F00C0339E0AE
:1072AC0004293ED123F010031B041B0C0384038B15
:1072BC00018C23F440731B051B0D43F4807343EACC
:1072CC000434564B89B2984212D003F500639842AD
:1072DC000ED0B0F1804F0BD0A3F59833984207D065
:1072EC0003F58063984203D003F58063984207D17D
:1072FC0021F0200141F0100141EA021292B204E0A7
:10730C0021F0A00141F010010A4304830284038B95
:10731C0023F440631B041B0C0383038B9BB203837A
:10732C0010BD082937D123F480731B041B0C038474
:10733C00818B038C89B221F0F30141F0010141EA08
:10734C000411364C9BB2A04212D004F50064A0424A
:10735C000ED0B0F1804F0BD0A4F59834A04207D0DA
:10736C0004F58064A04203D004F58064A04207D1E8
:10737C0023F4007343F4807343EA022292B204E0D4
:10738C0023F4206343F480731A4381830284838B38
:10739C0023F00C0338E023F480531B041B0C0384F0
:1073AC00818B038C21F440710905090D41F4807126
:1073BC0041EA0431194C9BB2A04212D004F500648E
:1073CC00A0420ED0B0F1804F0BD0A4F59834A0425F
:1073DC0007D004F58064A04203D004F58064A04279
:1073EC0007D123F4005343F4805343EA023292B2A0
:1073FC0005E047F6FF541C4044F48054224381833B
:10740C000284838B23F440631B041B0C8383838BC8
:10741C009BB2838310BD00BFCC030020002C014025
:10742C00026D70B515880446ADB2A90613D5036B71
:10743C008BB9C36A1BB1908880B298470BE0E169A5
:10744C00928840694E1CD2B2E6614254E169E2680E
:10745C00914228BFE3612B0613D5636AA26A9A4254
:10746C00236D0AD0511CA069A162825C9A802369A9
:10747C00994206D30023A36270BDDA6822F0800221
:10748C00DA6070BD026B0346C16810B5406942B149
:10749C001A6C8C1A013A08BF0A46005D1A64C0B215
:1074AC0010BD1A6A805C01328A4228BF0022C0B229
:1074BC001A6210BD436B13B190F844007047836A95
:1074CC00406A1B1A584258417047036B13B15B68F2
:1074DC00016C01E0C369016A8B423CBFC2689B1816
:1074EC00581AC0B27047836A8169426B1944D160E3
:1074FC00416A994297BF0169CB1ACB1A536096BF68
:10750C000023536083624FF0000380F8443013680B
:10751C0088BF816243F0010313607047436A82693C
:10752C00D154436A02690133934228BF002343625A
:10753C00436B1BB11B68DB0705D4D4E7026DD36822
:10754C0043F08003D36070472DE9F04105460E46A9
:10755C00078A83899BB21F40002F37D0B7FA87F276
:10756C004FF00043D340DB4399B21F40A2F11B0301
:10757C002982042BF0D8DFE803F0221F1C1903002A
:10758C00746A24B1013C0023A4B2736201E0AC8D97
:10759C00A4B2D6F82080B8F1000FDDD0D8F80030B6
:1075AC00404621469847D8F80480F4E73068A98E05
:1075BC0008E07068298F05E0B068A98F02E0F068D8
:1075CC00B5F84010036889B29847C5E7BDE8F0816B
:1075DC004171FFF76DBC8160FFF76ABC0E4B1A78E6
:1075EC00692A15D15A88B2F5A36F11D11A79BE2A1E
:1075FC000ED193F816250020EF2A0BD113F8012B8E
:10760C005040064A9342F9D1B0FA80F040097047D5
:10761C0000207047704700BF00F8000818FD0008F4
:10762C002DE9F74FDB4C00214FF4A362204605F007
:10763C0038F9D94B04F5CE721A60D84B00221A7067
:10764C00D74B04F2F2411960692323700323637151
:10765C0040F20113A3604FF41673A4F8F630FA232A
:10766C00A4F8F830BC23A4F8F4304FF4FA73A4F85F
:10767C00FE30012384F8F23084F80E3184F8163190
:10768C00052384F89B3140F2DC53A4F8283140F2F6
:10769C004C43A4F82A3140F26C73A4F82C3140F21C
:1076AC007533A4F82E3140F64303A4F83031234649
:1076BC00202184F8FA106E2184F80C110A2184F828
:1076CC000D112B2184F80F11212184F81011232185
:1076DC0084F811114FF4C871A4F81211032ACCBF0D
:1076EC000121002102F1010283F8321114BF1E2185
:1076FC007521122A83F8331103F10203EED14FF4F2
:10770C00FA63A4F85831A4F85C31A4F86031A4F8F9
:10771C006431052384F87231C823A4F8763140F221
:10772C007E43A4F8D43040F23A73A4F8D63040F239
:10773C007E53A4F8DC3040F2EA53A4F8DE3040F279
:10774C00B45340F2DC5001264FF47A784FF0320AF1
:10775C004FF01E094FF0190BA4F8E0304FF47A5398
:10776C0084F8259184F873B1A4F8DA000190A4F898
:10777C00E2A0A4F8E430A4F8E6A0A4F85681A4F89A
:10778C005A81A4F85E81A4F8628184F8716184F84E
:10779C00746184F8756184F87861A4F8D880FEF778
:1077AC0059F97D4A002513684FF00F0E2674E673C5
:1077BC00A573A58183F805E04FF0220E83F806E04F
:1077CC004FF00E0E83F810E04FF0350E172183F8B2
:1077DC001AE04FF0210E5975997583F811E0552177
:1077EC004FF0530E2827D97083F807B02D2183F85A
:1077FC001BE000924FF05A0E64224FF00A0B4FF030
:10780C00780C83F80B9083F80C90597383F804A0D0
:10781C0083F808E01A7783F80AC01D705F709F70B8
:10782C00DD759D731D76DD735D7683F812B05F7226
:10783C0019754FF4FA71A3F84E10082183F8501003
:10784C005849DFF87CC19963D9635749C3F82CC0F8
:10785C00C3F830C09962DFF86CC14FF07E515963A8
:10786C004FF07F595149C3F82090C3F82490C3F8C6
:10787C0048C001984FF04B0C4FF0000959649E77AB
:10788C0083F8525083F85170C3F8409083F84CC081
:10789C0084F8F2E44FF0410E84F8F3E484F8F4A495
:1078AC00A4F8FC0484F8F55484F8F95484F8FA54D8
:1078BC0084F8F65484F8F75484F8F85404201966C4
:1078CC00152183F85C00A3F85850A3F85A50A3F87C
:1078DC00565083F8647083F86810354983F86570E6
:1078EC00D966344983F87860196733493348596746
:1078FC00FEF7E1F8009A4FF44873D2F800A0AAF80A
:10790C001631C8238AF811518AF812518AF813716A
:10791C008AF814618AF8185184F86931642384F860
:10792C0068B1A4F86A8184F86C51A4F86E31194CD2
:10793C002B191035C02DC3F81490F8D1514604F50D
:10794C002E704FF48E7204F0A1FF04F57570514641
:10795C004FF48E7204F09AFF114B1B681A68C4F82E
:10796C00FE245A68C4F802259A68C4F806251A68D9
:10797C00C4F80A255A68C4F80E259A68012384F8BD
:10798C000C330223C4F8122584F8283403B0BDE864
:10799C00F08F00BFE809002048070020C016002027
:1079AC00440700208FC2F53C000060400000A0405E
:1079BC009A99193FF6287C3F3D0A773F29EA00083F
:1079CC00CDCCCC3E0000404001480249BCE500BF94
:1079DC00000800404811002001480249B4E500BFEE
:1079EC0000040040201100204FF080400049ABE51E
:1079FC00F810002001480249A6E500BF002C014008
:107A0C00D0100020014802499EE500BF002C014027
:107A1C00D0100020254B10B55A43254B254C1B6824
:107A2C000139B3FBF2F20388013AA04289B292B257
:107A3C009BB212D004F50064A0420ED0B0F1804F7E
:107A4C000BD0A4F59834A04207D004F58064A04272
:107A5C0003D004F58064A04202D123F070039BB2E2
:107A6C00154CA04206D004F58064A0421CBF23F440
:107A7C0040739BB203800F4B8185984202850FD0D7
:107A8C0003F5006398420BD003F54063984207D08E
:107A9C0003F58063984203D003F58063984201D1CB
:107AAC00002303860123838210BD00BF40420F00D8
:107ABC0038000020002C0140001000400C4B800AC4
:107ACC0098420CD004D8B0F5801F0CD1012070471F
:107ADC00084B984205D04933984206D003E0022067
:107AEC00704703207047FE2070470020704700BF8E
:107AFC0001001000020010002DE9F843046807464D
:107B0C00204688469146FFF7D9FF03284BD8BA7A0E
:107B1C009108B8F1000F06D1A589AEB202258D40AF
:107B2C0026EA0505A5810A2303FB00131F4A42F828
:107B3C002380043342F82390B8F1000F07D0BD7AAC
:107B4C00A189AD080223AB400B439BB2A381282330
:107B5C00434303F120011144EFF31286502585F3C2
:107B6C00128803F10C051C331544134455F8047F9B
:107B7C0017B10F60296804319D42F7D100230B60C7
:107B8C00F3B283F31188282303FB0020036A23B18B
:107B9C00A3899BB243F0010304E0A38923F0010302
:107BAC001B041B0CA381BDE8F88300BFD010002080
:107BBC00004835E484150020004831E4D815002035
:107BCC000A4B4FF400525A604FF6FE730848D0F837
:107BDC00882011680B401360826FC36F9A4201D0EA
:107BEC00543080E4012380F8983070470000024044
:107BFC00841500202DE9F04F85B002939B4B8046F5
:107C0C001C88019104F00204A4B2009294B1984B28
:107C1C00B3F90240B3F90030002CB8BF6442002B1A
:107C2C00B8BF5B429C42B8BF1C46B4F5007FA8BFEE
:107C3C004FF40074C34600278D4B4FF0040E33F9FC
:107C4C0017208C4B8C4933F917304FEA470A002B1D
:107C5C0093FBFEFEB8BF5B42B3F5206F4FEA4202C6
:107C6C004FEA870951F827000FDCCEEB02030344DF
:107C7C00B3F57A5F8148A8BF4FF47A538342ACBF07
:107C8C0041F8273041F8270002E0002341F8273063
:107C9C0051F809509BF80B309BF80160ED117349BA
:107CAC005D4356430988AD1189074FEAA6133BD0B3
:107CBC00009949428A4203DB00999142A8BF1146C0
:107CCC0042F210766E4A6F483AF90220891A029AEB
:107CDC0032F91720114459F800200A44B242A8BFC7
:107CEC003246694EB242B8BF324649F8002098F885
:107CFC000800414398F81C00C91100EB8000C0F14A
:107D0C00000C614503DB8142A8BF01468C4698F804
:107D1C001210CCEB03064A431213AD1A65436643AB
:107D2C0002EB65250CEB6623584AD65D98F851207A
:107D3C0006FB0EF6A3EBA61672B13046039201F0C9
:107D4C00F5F85349534B01EBC701039A1B68FCF739
:107D5C0075FE01F005FB064646494F4B3AF801000B
:107D6C003AF903E002B2CEEB02024FF0040E92FBA2
:107D7C00FEF22AF803009E440C3359F80EC059F851
:107D8C00030049F80E206044104498F8502049F83C
:107D9C0003C0894662B1039201F0C8F83F493D4BDC
:107DAC0001EBC701039A1B68FCF748FE01F0D8FAF7
:107DBC003B4B3C4ADB5D35445843A5EB60102AF83D
:107DCC0002000BF1010B0FB9012735E7284B0424F6
:107DDC00B3F90410019B28489B7985680F335B002D
:107DEC004B43B9F904105B1191FBF4F4002BA3EB9A
:107DFC000404B8BF5B42322B98F80D100BDC01FB6E
:107E0C000451294B8B42A8BF0B4628498B42ACBF6F
:107E1C008360816001E00023836098F8031001FB0C
:107E2C0004F323499B11097803290CD9B8F84E1097
:107E3C00B1F5FA7F07D24C42A34203DB8B42A8BFB9
:107E4C000B4600E0234681686FF0FF0041F34F3191
:107E5C00B1F5807FA8BF4FF480718142ACBF5B1835
:107E6C001B18938005B0BDE8F08F00BFE40600201E
:107E7C00E00F00200E0700200810002080C1FFFF3B
:107E8C003207002058100020F0D8FFFF60100020AF
:107E9C00EC0F0020041000202C16002038100020BD
:107EAC007810002050100020FEFFFF0F020000F0A1
:107EBC007B1000202DE9F04F87B00493994B4FF0C5
:107ECC00000BB3F90270B3F90030002FB8BF7F423A
:107EDC00002BB8BF5B429F42B8BF1F468246D946B3
:107EEC00D8465C46B7F5FA7F0392A8BF4FF4FA77F1
:107EFC000190CDF808B08C4B198811F0030040D0DC
:107F0C00022C3ED0874B650033F91420039B5200A2
:107F1C005B429A4203DB039B9342A8BF1346834AFE
:107F2C006FF00408AD5E049A5B1B32F914506422A6
:107F3C001D449AF808306B4393FBF2F39AF81C201B
:107F4C0008FB02F8434504DB02EB82089845A8BF06
:107F5C009846774A52F824302B4442F21075AB42C3
:107F6C00A8BF2B46734DAB42B8BF2B4642F824300A
:107F7C009AF81220012802FB03F34FEA23330293F1
:107F8C0041D0684B6C4D33F91490019BA00093F8D1
:107F9C0001C06A4B55F824E033F9146086EAE673A5
:107FAC00A3EBE673B3F5206F1DDC022C15D0502328
:107FBC0003FB09F292FBFCF3042296FBF2F69E1BE8
:107FCC00B644BEF57A5F5E4BA8BF4FF47A5E9E4511
:107FDC00ACBF45F800E02B5007E089EAE973A3EB4E
:107FEC00E973642BE3DD00232B50534B4FF07D0CD6
:107FFC00C35893FBFCFC019BDB7A03FB0CF34FF0A7
:10800C00400C93FBFCFB8A0713D5022C11D007FB09
:10801C000BF607FB09F30299C7F5FA7202FB08335A
:10802C0002FB01624FF4FA7593FBF5F392FBF5F644
:10803C0008E0CB0704D5022C02D0029E434601E097
:10804C005E464B46620000923C4A042532F91420ED
:10805C0092FBF5F53B4AA25C55436FF04F0295FB42
:10806C00F2F59AF851201D44E2B1022C05922846F3
:10807C000BD100F05BFF059A530803D09A42A8BFBE
:10808C001A4600E00122304905E000F04FFF2F496D
:10809C00059A01EBC4012E4B1B68FCF7CFFC01F0D9
:1080AC005FF90546254B009A0098D15A294B0AB224
:1080BC00C05E121A042092FBF0F20098C15203F138
:1080CC000801143351F824E053F8240041F824201B
:1080DC00704410449AF8502043F824E062B10592A1
:1080EC0000F024FF1C491A4B01EBC401059A1B68D4
:1080FC00FCF7A4FC01F034F9184B35441B5D202629
:10810C00584390FBF6F0164B009A281AD052019B5C
:10811C0001340133032C01937FF4EDAE07B0BDE8BD
:10812C00F08F00BFE00F0020E40600203207002093
:10813C0058100020F0D8FFFF081000200E07002078
:10814C0080C1FFFF60100020FC0F0020EC0F00200E
:10815C000410002040160020381000207810002059
:10816C00501000202DE9F04F89B00593934B074632
:10817C001B880C469B0702924DD540F2E631129BB0
:10818C008F4AD889B2F900301B1A03F2F3158D42CD
:10819C0003D8002BB8BF5B4201E04FF4FA73B2F97D
:1081AC000220101A40F2E63200F2F311914203D889
:1081BC000028B8BF404201E04FF4FA7097F84C50D9
:1081CC003DB39842B8BF1846C0F5FA7000F0AEFE49
:1081DC007C4900F0B3FF4FF07E5100F0F1FD0646F4
:1081EC00642090FBF5F000F0A1FE0146304600F053
:1081FC00F1FE4FF07E5100F0E5FD0021064601F046
:10820C0087F830B930464FF07E5101F09FF820B11D
:10821C0001E0002601E04FF07E56E31C049300972A
:10822C000024049B620013F8015F022C0493039258
:10823C00654B09D1B3F904000A35684300F076FEAA
:10824C00624900F07BFF5DE033F91490484600F082
:10825C006DFE8046029800F065FE5A4900F06EFFF4
:10826C000146404600F0B6FE029B8046584200F0A4
:10827C005DFE82464046514601F04AF848B90298E4
:10828C0000F054FE82464046514601F05FF800B9BA
:10829C00C246039A4E4B985E00F048FE014650468B
:1082AC0000F08EFD059B804633F9140000F03EFE75
:1082BC000146404600F086FD464900F03FFF3F4B2B
:1082CC008246B3F8008018F0010F03D0796C00F0EF
:1082DC0081FE17E005F1140009FB00F000F026FE0A
:1082EC003A4900F02BFF18F0020F05460BD0B96C81
:1082FC00504600F06FFE314600F06CFE01462846F9
:10830C0000F060FD0546039A334BDFF8EC80985E75
:10831C0000F00CFE314B596C00F05CFE0146284617
:10832C0000F04EFD009B8246196A00F053FE2C4B68
:10833C000546185D00F0FAFD0146284600F04AFE9D
:10834C00284900F0FBFE97F8512081469AB1022C87
:10835C0009D1530803D09A42A8BF1A4600E0012263
:10836C004846214902E0214901EBC401D8F800300C
:10837C00FCF764FB8146D8F800305046194601934F
:10838C0000F028FE009BDFF874B0D96A00F022FEE2
:10839C00104900F01FFE5BF8241000F013FD144987
:1083AC00A500804600F0B4FF50BB4046114900F0D8
:1083BC00CDFF38B3DFF83C8024E000BFE40600209A
:1083CC00140900200000FA43E00F0020000048428E
:1083DC0032070020000020410E0700202C16002040
:1083EC00E80F00200000C842FC0F0020EC0F00201A
:1083FC0000007AC300007A4304100020841000208F
:10840C00DFF810814BF80580DFF80CB1504655F8B9
:10841C000B1000F0D5FC45F80BA0069001994FF01D
:10842C007E5000F08BFE069B0146184600F0D2FDF4
:10843C0082460BF10C03EA580BF1180B104655F859
:10844C000B100793069200F0BDFC514600F0BAFCED
:10845C00069A079B45F80B2097F85020014645F8E3
:10846C0003A032B12349019B01EBC401FCF7E6FAEE
:10847C0001460846204900F061FE009B996B00F014
:10848C00A9FD1E4B0546185D00F050FD014628461F
:10849C0000F0A0FD1A4900F051FE1A49054600F003
:1084AC0037FF30B92846184900F050FF10B1164D6F
:1084BC0000E0144D4146484600F084FC294600F08B
:1084CC0081FC04F04DFB114BB0F57A7FA8BF4FF443
:1084DC007A709842B8BF1846039A0D4B01349852E3
:1084EC00009B032C03F1040300937FF49AAE09B0B4
:1084FC00BDE8F08F3810002000004040E80F00204D
:10850C000000C842000096C30000964318FCFFFF11
:10851C005010002000007AC374160020044B002277
:10852C001A605A60034B00221A605A60704700BFF1
:10853C00581000207C10002010B50D4C012384F83D
:10854C006F304FF48060022384F88C30FCF786FD8A
:10855C00084BD4F890201B685278642101FB02333D
:10856C00C4F88030B4F86C300133A4F86C3010BD12
:10857C002C160020E4160020704707B5064B07495F
:10858C000093074B074A01930748084BFCF700FB85
:10859C0003B05DF804FB00BFE4E5000852EA0008F4
:1085AC00EDE5000858EA000832EA0008D8E50008B2
:1085BC0008B5037833B90C4B0C481978BDE8084062
:1085CC00FCF7E6BA04F006FA02280CD8064B0C228B
:1085DC001870074B02FB0030064B02301860FCF79A
:1085EC0029FE0548E5E708BDC01600205FEA000833
:1085FC00D80E002044070020BCE4000808B503781E
:10860C003BB90B4B0B4893F8F014BDE80840FCF752
:10861C00BFBA04F0DFF9022808D8054B83F8F00440
:10862C00FCF75EFDFCF72AFE0348E8E708BD00BF37
:10863C00E809002063EA0008BCE4000873B503787D
:10864C0013B9FBF765FC3FE001AA204904F0F1F9EE
:10865C0000240246264625469AB134B1012C08D195
:10866C00104604F0B7F9064603E0104604F0B2F9E0
:10867C00054601AA0020154904F0DBF90134024635
:10868C00EAE70B2D03D9124812490C230CE0022CFB
:10869C0011D1A6F57A73B3F57A7F08D90C480E4937
:1086AC004FF47A724FF4FA63FCF772FA0CE00B4B4E
:1086BC0003EB45035E80094B094803EB4503294650
:1086CC00B3F90220FCF764FA02B070BD90E4000824
:1086DC0072E7000891E7000849EC0008C01600207A
:1086EC0070EA000810B50446054B2146D869FCF722
:1086FC0024F9044B1B6898796040987110BD00BF39
:10870C00C0160020D806002010B50446C0B2FFF7F2
:10871C00E9FF200ABDE81040E4E737B5828883689A
:10872C00044610060D4641BF29494FF48E7091F84E
:10873C00F01400FB0133D10542BF26490C20097807
:10874C0002F03F0248BF00FB0133042A12D006D8C6
:10875C00012A0DD0022A2FD193F900102DE0102AF6
:10876C000AD0202A0AD0082A26D1B3F9001024E016
:10877C00197822E0198820E019681EE0694618680B
:10878C00FCF78CF901461448FCF702FAF5B1E068E5
:10879C0000F0CCFB6946FCF781F901460F48FCF769
:1087AC00F7F9206900F0C2FB6946FCF777F901463E
:1087BC000A48FCF7EDF909E000210948FCF7E8F953
:1087CC0025B10848E1682269FCF7E2F903B030BD35
:1087DC00E8090020C01600205AEB000853EB0008F3
:1087EC0083EA00087FEA000810B5441E14F8011F44
:1087FC0021B1034B186AFCF7A0F8F7E710BD00BFD6
:10880C00C016002013B51548154B446A154990F84D
:10881C0028001A8851F82010134B14481B7800912B
:10882C004FF47A71B4FBF1F1FCF7B2F9104B11482B
:10883C001968114BB1FBF3F1FCF7AAF90F48FFF7DC
:10884C00D3FF0F4B0F481A880F4B92B219884FF475
:10885C00A36302B0BDE81040FCF79AB9C016002023
:10886C00C80F002060D800083400002086EA0008F9
:10887C0038000020C9EA000840420F001DEB000838
:10888C00DE060020D9EA0008DC0600202DE9F041C4
:10889C000024804625460F4E4146A759384604F021
:1088AC0081F858B139460C48FCF772F9301900219F
:1088BC00FFF733FF0948FFF797FF013540F6C82350
:1088CC0014349C42E7D11DB9BDE8F04104488BE754
:1088DC00BDE8F08170D8000857E700081DEB0008D0
:1088EC00F9E600082DE9F04F85B0054604F01DF8B7
:1088FC00064620B1012818D12B782A2B15D19C487B
:10890C00FFF772FF00249B4D9B486159FCF740F91F
:10891C0028193146FFF701FF9848FFF765FF40F62D
:10892C00C82314349C42EED11EE128463D2103F0AD
:10893C00EEFF002800F0138103461A4613F8011DC0
:10894C002029FAD0441C531B2046019304F042F812
:10895C008346204602780346202A00F10100F9D014
:10896C00092AF7D02D2A03D10346DFF8349204E00C
:10897C002B2A08BF03464FF07E591E460024324670
:10898C0016F8011BA1F13007FBB2092B0DD87C495D
:10899C00204600F01FFB0446384600F0C7FA01469B
:1089AC00204600F00FFA0446E9E72E29134617D1AA
:1089BC00734F334616F8010B3038C2B2092A0FD860
:1089CC0000F0B4FA394600F0B9FB0146204600F03D
:1089DC00F9F96B490446384600F0FCFA0746E8E71B
:1089EC001A7802F0DF02452A39D15A782D2A02D1A1
:1089FC000233012704E02B2A14BF01330233002772
:108A0C00013B002613F8012F303AD1B2092903D8C3
:108A1C000A2101FB0626F5E7B6F59A7F28BF4FF42D
:108A2C009A76B0464FF07E53B8F1070F07D9184627
:108A3C00544900F0CFFAA8F108080346F4E706F011
:108A4C00070636B118464E4900F0C4FA013E0346FB
:108A5C00F7E719462FB1204600F070FB04E04FF009
:108A6C007E51204600F0B6FA0346002614247443C7
:108A7C00454F039307F1100854F808A0504603F033
:108A8C0054FF8446514662462846CDF808C003F090
:108A9C0055FFDDF808C0039B002858D19DF8042031
:108AAC00624554D11946484600F094FAA0443C441F
:108ABC000546E06900F03AFA0146284600F03CFC15
:108ACC00002842D0206A00F031FA0146284600F016
:108ADC0029FC002839D0A38A9A0658BF5D46142277
:108AEC0002FB06761C0648BF2848B26942BF90F8C4
:108AFC00F0044FF48E7404FB0022D80542BF2448C6
:108B0C000C24007803F03F0348BF04FB0022042B25
:108B1C0029460BD004D8013B012B0CD815700AE068
:108B2C00102B05D0202B05D0082B04D1118002E08E
:108B3C00156000E0156051461648FCF729F84046D0
:108B4C00002105B0BDE8F04FE7E5134803E001361E
:108B5C008A2E8BD1114805B0BDE8F04F44E628466B
:108B6C0005B0BDE8F04F91E605B0BDE8F08F00BF51
:108B7C000BEB000870D8000857E700081DEB000845
:108B8C000000204120BCBE4C60D80008E809002041
:108B9C00C016002020EB00082BEB0008F9E60008BB
:108BAC00000080BFF0B585B0044603F0BEFE082877
:108BBC0026D1621EE01D1F4912F8013F09681944B5
:108BCC00497801F00301022908BF203B824213704F
:108BDC00F1D1254604F1080715F8016B164831460A
:108BEC0003F095FE20B12846314603F090FE10B1FB
:108BFC00FBF78EF91CE0BD42EED12046FCF75BFF83
:108C0C000E48FFF7F1FD00230D4A04A91A4492F80F
:108C1C001A210A440849595C0133082B02F80C1C30
:108C2C00F2D10023074801A98DF80C30FBF7B0FFF7
:108C3C0005B0F0BD3C00002014EA00084BEB000826
:108C4C00E80900207DE8000838B500240B4D605978
:108C5C002544FFF7C9FD696811B10948FBF798FF76
:108C6C00A96811B10748FBF793FF07481034FFF7C9
:108C7C00BBFDB4F5A87FE9D138BD00BF38E30008CF
:108C8C0051EB000857EB00081DEB000810B50A4823
:108C9C00FFF7AAFD094B1C6A2046FBF74BFE18B9DF
:108CAC000A20FBF7FCFDF7E7FEF72AF8FCF7EEF9D4
:108CBC00034A044BDA6010BD5DEB0008C0160020BF
:108CCC000400FA0500ED00E008B50548FFF78CFD3F
:108CDC00FEF7A6FCFCF704FABDE80840D6E700BF97
:108CEC0069EB000808B50448FFF77EFDFCF7F8F9BE
:108CFC00BDE80840CAE700BF7FEB000813490B78BA
:108D0C0013F0010F03F004021BD0F2B910480068F5
:108D1C0040011AD4980714D443F004030B700D4B84
:108D2C004FF47A711A880C4B05201A800B4B0C4AA5
:108D3C001B6892F8722101FB02330A4A1360FBF79D
:108D4C0045BD12B90120FBF767BD7047FD16002029
:108D5C00E806002036070020D6060020E416002086
:108D6C00E809002088060020054A1378590705D524
:108D7C0023F0040304201370FBF728BD704700BFD9
:108D8C00FD16002008B5044B1B7803F00503052BDA
:108D9C0001D1FDF7B5FFFEE7EC160020D0400B1C0F
:108DAC001141203A03D49C46134118436346524266
:108DBC0093401843704700BF80F0004002E000BFB2
:108DCC0081F0004142001FBF5FEA410392EA030FAA
:108DDC007FEA226C7FEA236C6AD04FEA1262D2EBF4
:108DEC001363C1BFD218414048404140B8BF5B42F9
:108DFC00192B88BF704710F0004F40F4000020F092
:108E0C007F4018BF404211F0004F41F4000121F0A7
:108E1C007F4118BF494292EA030F3FD0A2F10102F1
:108E2C0041FA03FC10EB0C00C3F1200301FA03F12F
:108E3C0000F0004302D5494260EB4000B0F5000F52
:108E4C0013D3B0F1807F06D340084FEA310102F111
:108E5C000102FE2A51D2B1F1004F40EBC25008BFC3
:108E6C0020F0010040EA03007047490040EB00008D
:108E7C0010F4000FA2F10102EDD1B0FA80FCACF1BC
:108E8C00080CB2EB0C0200FA0CF0AABF00EBC250BB
:108E9C0052421843BCBFD0401843704792F0000FA9
:108EAC0081F4000106BF80F400000132013BB5E7FC
:108EBC004FEA41037FEA226C18BF7FEA236C21D072
:108ECC0092EA030F04D092F0000F08BF08467047D7
:108EDC0090EA010F1CBF0020704712F07F4F04D1A5
:108EEC00400028BF40F00040704712F100723CBFB8
:108EFC0000F50000704700F0004343F0FE4040F4E2
:108F0C00000070477FEA226216BF08467FEA23639F
:108F1C000146420206BF5FEA412390EA010F40F48A
:108F2C00800070474FF0000304E000BF10F00043D6
:108F3C0048BF40425FEA000C08BF704743F09643BD
:108F4C0001464FF000001CE050EA010208BF7047D8
:108F5C004FF000030AE000BF50EA010208BF70475F
:108F6C0011F0004302D5404261EB41015FEA010C74
:108F7C0002BF84460146002043F0B64308BFA3F16C
:108F8C008053A3F50003BCFA8CF2083AA3EBC2534E
:108F9C0010DB01FA02FC634400FA02FCC2F120026D
:108FAC00BCF1004F20FA02F243EB020008BF20F0A4
:108FBC000100704702F1200201FA02FCC2F120020A
:108FCC0050EA4C0021FA02F243EB020008BF20EAFF
:108FDC00DC7070474FF0FF0C1CEAD0521EBF1CEA2D
:108FEC00D15392EA0C0F93EA0C0F6FD01A4480EA1B
:108FFC00010C400218BF5FEA41211ED04FF0006304
:10900C0043EA501043EA5111A0FB01310CF000402F
:10901C00B1F5000F3EBF490041EAD3715B0040EA55
:10902C00010062F17F02FD2A1DD8B3F1004F40EB25
:10903C00C25008BF20F00100704790F0000F0CF0F8
:10904C00004C08BF49024CEA502040EA51207F3ABC
:10905C00C2BFD2F1FF0340EAC250704740F4000097
:10906C004FF00003013A5DDC12F1190FDCBF00F088
:10907C0000407047C2F10002410021FA02F1C2F136
:10908C00200200FA02FC5FEA310040F1000053EAD2
:10909C004C0308BF20EADC70704792F0000F00F020
:1090AC00004C02BF400010F4000F013AF9D040EA26
:1090BC000C0093F0000F01F0004C02BF490011F4BA
:1090CC00000F013BF9D041EA0C018FE70CEAD153B8
:1090DC0092EA0C0F18BF93EA0C0F0AD030F0004C38
:1090EC0018BF31F0004CD8D180EA010000F00040EC
:1090FC00704790F0000F17BF90F0004F084691F0AA
:10910C00000F91F0004F14D092EA0C0F01D14202E3
:10911C000FD193EA0C0F03D14B0218BF084608D1AC
:10912C0080EA010000F0004040F0FE4040F40000F6
:10913C00704740F0FE4040F4400070474FF0FF0C89
:10914C001CEAD0521EBF1CEAD15392EA0C0F93EAD0
:10915C000C0F69D0A2EB030280EA010C49024FEA22
:10916C00402037D04FF0805343EA111143EA1013DB
:10917C000CF000408B4238BF5B0042F17D024FF493
:10918C00000C8B4224BF5B1A40EA0C00B3EB510F6E
:10919C0024BFA3EB510340EA5C00B3EB910F24BF57
:1091AC00A3EB910340EA9C00B3EBD10F24BFA3EBDC
:1091BC00D10340EADC001B0118BF5FEA1C1CE0D1A4
:1091CC00FD2A3FF650AF8B4240EBC25008BF20F057
:1091DC00010070470CF0004C4CEA50207F32C2BFAB
:1091EC00D2F1FF0340EAC250704740F400004FF048
:1091FC000003013A37E792F0000F00F0004C02BF79
:10920C00400010F4000F013AF9D040EA0C0093F042
:10921C00000F01F0004C02BF490011F4000F013B9C
:10922C00F9D041EA0C0195E70CEAD15392EA0C0F04
:10923C0008D142027FF47DAF93EA0C0F7FF470AF3C
:10924C00084676E793EA0C0F04D14B023FF44CAF7F
:10925C0008466EE730F0004C18BF31F0004CCAD114
:10926C0030F000427FF45CAF31F000437FF43CAF50
:10927C005FE700BF4FF0FF3C06E000BF4FF0010C72
:10928C0002E000BF4FF0010C4DF804CD4FEA400254
:10929C004FEA41037FEA226C18BF7FEA236C11D09E
:1092AC0001B052EA530C18BF90EA010F58BFB2EB51
:1092BC00030088BFC81738BF6FEAE17018BF40F0D1
:1092CC00010070477FEA226C02D15FEA402C05D185
:1092DC007FEA236CE4D15FEA412CE1D05DF8040B0A
:1092EC00704700BF844608466146FFE70FB5FFF79D
:1092FC00C9FF002848BF10F1000F0FBD4DF808ED55
:10930C00FFF7F4FF0CBF012000205DF808FB00BF45
:10931C004DF808EDFFF7EAFF34BF012000205DF89F
:10932C0008FB00BF4DF808EDFFF7E0FF94BF0120EC
:10933C0000205DF808FB00BF4DF808EDFFF7D2FFE9
:10934C0094BF012000205DF808FB00BF4DF808ED2C
:10935C00FFF7C8FF34BF012000205DF808FB00BFF9
:10936C004FEA4002B2F1FE4F0FD34FF09E03B3EB26
:10937C0012620DD94FEA002343F0004310F0004F66
:10938C0023FA02F018BF404270474FF000007047BC
:10939C0012F1610F01D1420205D110F0004008BF5B
:1093AC006FF0004070474FF00000704742000ED243
:1093BC00B2F1FE4F0BD34FF09E03B3EB126209D404
:1093CC004FEA002343F0004323FA02F070474FF0BA
:1093DC000000704712F1610F01D1420202D14FF02F
:1093EC00FF3070474FF00000704700BF7BB972B977
:1093FC000029BEBF00204FF0004106E008BF002846
:10940C001CBF6FF000414FF0FF3000F075B882B018
:10941C00EC462DE9005000F03FF8DDF804E002B016
:10942C000CBC704710B500210446FFF771FF20B942
:10943C002046BDE8104000F009B804F1004000F0EF
:10944C0005F8404261EB410110BD00BFD0B500F002
:10945C00B9F900220E4B06460F4600F007FA00F051
:10946C0017FC044600F08CF900220A4B00F0FEF9C0
:10947C0002460B463046394600F044F800F008FC32
:10948C002346002242EA000210461946D0BD00BF16
:10949C000000F03D0000F0412DE9F041069C9046A3
:1094AC0006460F461D4600F013FC08FB01FCA8FB0A
:1094BC00002300FB05C5B21A2B4467EB0303864659
:1094CC00C4E90023BDE8F0812DE9F843089E174656
:1094DC00804689461D4600F051FD00FB05F3A0FBBC
:1094EC00074507FB0137B8EB04043D4469EB050560
:1094FC00C6E90045BDE8F883704700BF81F0004124
:10950C0002E000BF83F0004330B54FEA41044FEA5C
:10951C00430594EA050F08BF90EA020F1FBF54EAF7
:10952C00000C55EA020C7FEA645C7FEA655C00F093
:10953C00E2804FEA5454D4EB5555B8BF6D420CDD64
:10954C002C4480EA020281EA030382EA000083EAE7
:10955C00010180EA020281EA0303362D88BF30BD87
:10956C0011F0004F4FEA01314FF4801C4CEA1131DD
:10957C0002D0404261EB410113F0004F4FEA03333C
:10958C004CEA133302D0524263EB430394EA050FC7
:10959C0000F0A780A4F10104D5F1200E0DDB02FA36
:1095AC000EFC22FA05F2801841F1000103FA0EF2CA
:1095BC00801843FA05F359410EE0A5F120050EF190
:1095CC00200E012A03FA0EFC28BF4CF0020C43FAC1
:1095DC0005F3C01851EBE37101F0004507D54FF0CE
:1095EC00000EDCF1000C7EEB00006EEB0101B1F51E
:1095FC00801F1BD3B1F5001F0CD349085FEA300064
:10960C004FEA3C0C04F101044FEA445212F5800F6E
:10961C0080F09A80BCF1004F08BF5FEA500C50F10B
:10962C00000041EB045141EA050130BD5FEA4C0CEE
:10963C00404141EB010111F4801FA4F10104E9D177
:10964C0091F0000F04BF01460020B1FA81F308BF6E
:10965C002033A3F10B03B3F120020CDA0C3208DD3A
:10966C0002F1140CC2F10C0201FA0CF021FA02F115
:10967C000CE002F11402D8BFC2F1200C01FA02F185
:10968C0020FA0CFCDCBF41EA0C019040E41AA2BFAA
:10969C0001EB0451294330BD6FEA04041F3C1CDA72
:1096AC000C340EDC04F11404C4F1200220FA04F092
:1096BC0001FA02F340EA030021FA04F345EA03013C
:1096CC0030BDC4F10C04C4F1200220FA02F001FAFE
:1096DC0004F340EA0300294630BD21FA04F0294680
:1096EC0030BD94F0000F83F4801306BF81F4801119
:1096FC000134013D4EE77FEA645C18BF7FEA655C8C
:10970C0029D094EA050F08BF90EA020F05D054EA5D
:10971C00000C04BF1946104630BD91EA030F1EBF62
:10972C000021002030BD5FEA545C05D14000494166
:10973C0028BF41F0004130BD14F580043CBF01F559
:10974C00801130BD01F0004545F0FE4141F470013F
:10975C004FF0000030BD7FEA645C1ABF194610461A
:10976C007FEA655C1CBF0B46024650EA013406BF1B
:10977C0052EA033591EA030F41F4002130BD00BFDA
:10978C0090F0000F04BF0021704730B54FF4806497
:10979C0004F132044FF000054FF0000150E700BF18
:1097AC0090F0000F04BF0021704730B54FF4806477
:1097BC0004F1320410F0004548BF40424FF0000164
:1097CC003EE700BF42004FEAE2014FEA31014FEAA7
:1097DC0002701FBF12F07F4393F07F4F81F06051F6
:1097EC00704792F0000F14BF93F07F4F704730B565
:1097FC004FF4607401F0004521F0004120E700BFF8
:10980C0050EA010208BF704730B54FF000050AE07E
:10981C0050EA010208BF704730B511F0004502D57F
:10982C00404261EB41014FF4806404F132045FEA81
:10983C00915C3FF4DCAE4FF003025FEADC0C18BF26
:10984C0003325FEADC0C18BF033202EBDC02C2F11C
:10985C00200300FA03FC20FA02F001FA03FE40EAAE
:10986C000E0021FA02F11444C1E600BF70B54FF0AE
:10987C00FF0C4CF4E06C1CEA11541DBF1CEA135590
:10988C0094EA0C0F95EA0C0F00F0DEF82C4481EAF8
:10989C00030621EA4C5123EA4C5350EA013518BF18
:1098AC0052EA033541F4801143F4801338D0A0FB05
:1098BC0002CE4FF00005E1FB02E506F00042E0FBB2
:1098CC0003E54FF00006E1FB03569CF0000F18BFB8
:1098DC004EF0010EA4F1FF04B6F5007F64F5407460
:1098EC0004D25FEA4E0E6D4146EB060642EAC621F3
:1098FC0041EA55514FEAC52040EA5E504FEACE2E60
:10990C00B4F1FD0C88BFBCF5E06F1ED8BEF1004F62
:10991C0008BF5FEA500E50F1000041EB045170BDDE
:10992C0006F0004646EA010140EA020081EA030122
:10993C00B4EB5C04C2BFD4EB0C0541EA045170BD1E
:10994C0041F480114FF0000E013C00F3AB8014F198
:10995C00360FDEBF002001F0004170BDC4F10004E1
:10996C00203C35DA0C341BDC04F11404C4F1200562
:10997C0000FA05F320FA04F001FA05F240EA0200BD
:10998C0001F0004221F0004110EBD37021FA04F6F3
:10999C0042EB06015EEA430E08BF20EAD37070BDAD
:1099AC00C4F10C04C4F1200500FA04F320FA05F00C
:1099BC0001FA04F240EA020001F0004110EBD3700E
:1099CC0041F100015EEA430E08BF20EAD37070BD7E
:1099DC00C4F1200500FA05F24EEA020E20FA04F357
:1099EC0001FA05F243EA020321FA04F001F0004106
:1099FC0021FA04F220EA020000EBD3705EEA430E77
:109A0C0008BF20EAD37070BD94F0000F0FD101F0A5
:109A1C000046400041EB010111F4801F08BF013CDE
:109A2C00F7D041EA060195F0000F18BF704703F01C
:109A3C000046520043EB030313F4801F08BF013DA3
:109A4C00F7D043EA0603704794EA0C0F0CEA13555F
:109A5C0018BF95EA0C0F0CD050EA410618BF52EA19
:109A6C004306D1D181EA030101F000414FF000001F
:109A7C0070BD50EA410606BF1046194652EA43062D
:109A8C0019D094EA0C0F02D150EA013613D195EAA1
:109A9C000C0F05D152EA03361CBF104619460AD1E9
:109AAC0081EA030101F0004141F0FE4141F47001F3
:109ABC004FF0000070BD41F0FE4141F4780170BDE3
:109ACC0070B54FF0FF0C4CF4E06C1CEA11541DBF48
:109ADC001CEA135594EA0C0F95EA0C0F00F0A7F84A
:109AEC00A4EB050481EA030E52EA03354FEA013177
:109AFC0000F088804FEA03334FF0805545EA13138A
:109B0C0043EA12634FEA022245EA111545EA106551
:109B1C004FEA00260EF000419D4208BF964244F1E8
:109B2C00FD0404F5407402D25B084FEA3202B61A07
:109B3C0065EB03055B084FEA32024FF480104FF4DB
:109B4C00002CB6EB020E75EB030E22BFB61A75464F
:109B5C0040EA0C005B084FEA3202B6EB020E75EBE2
:109B6C00030E22BFB61A754640EA5C005B084FEA4A
:109B7C003202B6EB020E75EB030E22BFB61A754617
:109B8C0040EA9C005B084FEA3202B6EB020E75EB22
:109B9C00030E22BFB61A754640EADC0055EA060EE3
:109BAC0018D04FEA051545EA16754FEA06164FEA26
:109BBC00C30343EA52734FEAC2025FEA1C1CC0D1D2
:109BCC0011F4801F0BD141EA00014FF000004FF05F
:109BDC00004CB6E711F4801F04BF01430020B4F120
:109BEC00FD0C88BFBCF5E06F3FF6AFAEB5EB030CD8
:109BFC0004BFB6EB020C5FEA500C50F1000041EBD5
:109C0C00045170BD0EF0004E4EEA113114EB5C04A1
:109C1C00C2BFD4EB0C0541EA045170BD41F4801174
:109C2C004FF0000E013C90E645EA060E8DE60CEA7C
:109C3C00135594EA0C0F08BF95EA0C0F3FF43BAF99
:109C4C0094EA0C0F0AD150EA01347FF434AF95EA50
:109C5C000C0F7FF425AF104619462CE795EA0C0F34
:109C6C0006D152EA03353FF4FDAE1046194622E701
:109C7C0050EA410618BF52EA43067FF4C5AE50EADB
:109C8C0041047FF40DAF52EA43057FF4EBAE12E7CB
:109C9C004A0011D212F5001211D20DD56FF478735F
:109CAC00B3EB62520ED44FEAC12343F0004343EAB4
:109CBC00505323FA02F070474FF00000704750EAFF
:109CCC00013002D14FF0FF3070474FF00000704769
:109CDC0000292DE9F043C0F2A8800026002BC0F229
:109CEC009E8081468E4690469C46174604460D46FD
:109CFC00002B3DD18A4259D9B2FA82F33BB1C3F160
:109D0C0020029D4020FA02F29F4015439C40390CE2
:109D1C00B5FBF1F01FFA87FE01FB10550EFB00F3AB
:109D2C00220C42EA0545AB4209D9ED1900F1FF328C
:109D3C0080F00B81AB4240F2088102383D44ED1AB1
:109D4C00B5FBF1F301FB13550EFB03FEA4B244EA81
:109D5C000545AE4508D9ED1903F1FF3280F0F780C7
:109D6C00AE4540F2F480023B43EA0043002203E09C
:109D7C008B420FD900221346341C18BF01246042B9
:109D8C004FF0000565EB4501584051400019694101
:109D9C00BDE8F083B3FA83F2002A40F089808B424D
:109DAC0002D3804500F2E2800123E5E712B90123DA
:109DBC00B3FBF2F7B7FA87F8B8F1000F3BD1ED1B04
:109DCC004FEA174C1FFA87FE0122B5FBFCF00CFB87
:109DDC0010550EFB00F3210C41EA0545AB4207D9A7
:109DEC00ED1900F1FF3102D2AB4200F2C3800846FC
:109DFC00ED1AB5FBFCF30CFB13550EFB03FEA4B2E2
:109E0C0044EA0545AE4507D9ED1903F1FF3102D2FD
:109E1C00AE4500F2AD800B4643EA0043ACE752423C
:109E2C006FEA060663EB43035BE7404261EB4101DB
:109E3C004FF0FF3652E707FA08F7C8F1200225FA6F
:109E4C0002F34FEA174CB3FBFCF11FFA87FE0CFB35
:109E5C00113324FA02F205FA08F50EFB01F92A4334
:109E6C00100C40EA0343994504FA08F407D9DB19AE
:109E7C0001F1FF3078D2994576D902393B44C9EBD0
:109E8C000303B3FBFCF00CFB10330EFB00F592B29A
:109E9C0042EA03439D4207D9DB1900F1FF325FD23E
:109EAC009D425DD902383B445D1B40EA01428CE780
:109EBC00C2F1200328FA03F10CFA02FC41EA0C0C63
:109ECC004FEA1C402EFA03F1B1FBF0F51FFA8CF7A8
:109EDC0000FB151129FA03F30EFA02FE07FB05F934
:109EEC0043EA0E0E4FEA1E4343EA0141894508FA44
:109EFC0002F808D911EB0C0105F1FF3332D2894578
:109F0C0030D9023D6144C9EB0101B1FBF0F300FB18
:109F1C00131107FB03F71FFA8EFE4EEA014E77452D
:109F2C0008D91EEB0C0E03F1FF3117D2774515D96A
:109F3C00023BE64443EA0543A3FB0889C7EB0E0E3C
:109F4C00CE4509D305D0002216E71046F7E6134696
:109F5C000AE794404445F6D2013BF4E70B46E9E7A7
:109F6C001046A1E71D46CEE7014688E7134603E7F6
:109F7C00023B51E702383D443AE700BF2DE9F0437C
:109F8C00002B44D18A42154604464FD9B2FA82F7C7
:109F9C000E464FB1C7F12003B94020FA03F602FA7E
:109FAC0007F50E4300FA07F42F0CB6FBF7F01FFA77
:109FBC0085FE07FB10620EFB00F1260C46EA0243FD
:109FCC00994209D95B1900F1FF3280F0EE80994279
:109FDC0040F2EB8002382B44591AB1FBF7F307FB24
:109FEC0013110EFB03FEA4B244EA01418E4508D9BD
:109FFC00491903F1FF3280F0DA808E4540F2D780A8
:10A00C00023B43EA004000263146BDE8F0838B4218
:10A01C0047D8B3FA83F6002E48D18B4202D3824242
:10A02C0000F2CF8001203146BDE8F08312B9012542
:10A03C00B5FBF2F5B5FA85FCBCF1000F78D1491BE4
:10A04C002F0C1FFA85FE0126B1FBF7F007FB101150
:10A05C000EFB00F2230C43EA01418A4207D949194D
:10A06C0000F1FF3302D28A4200F2BC801846891AF2
:10A07C00B1FBF7F307FB13110EFB03FEA4B244EA8A
:10A08C000142964508D9521903F1FF3180F09180B5
:10A09C00964540F28E80023B43EA00403146BDE8D3
:10A0AC00F083002630463146BDE8F083C6F120042B
:10A0BC0022FA04F5B3402B4321FA04F74FEA134874
:10A0CC00B7FBF8FC1FFA83F908FB1C7720FA04FE97
:10A0DC0001FA06F509FB0CF44EEA05054FEA154E9C
:10A0EC004EEA0747BC4202FA06F204D9FF180CF1FB
:10A0FC00FF3168D38C463F1BB7FBF8F408FB147791
:10A10C0009FB04F9ADB245EA0741894504D9C918E0
:10A11C0004F1FF355DD32C4644EA0C44A4FB022326
:10A12C00C9EB0101994249D345D0204600266BE783
:10A13C00CCF1200405FA0CF521FA04F32A0CB3FB3C
:10A14C00F2F61FFA85FE02FB163820FA04F701FA24
:10A15C000CF10EFB06F90F433C0C44EA08439945FD
:10A16C0000FA0CF407D95B1906F1FF3138D2994586
:10A17C0036D9023E2B44C9EB0303B3FBF2F002FBCE
:10A18C0010330EFB00F1BFB247EA0343994207D9E3
:10A19C005B1900F1FF3721D299421FD902382B44A9
:10A1AC001746591A40EA06464EE7104614E713467E
:10A1BC0027E70B4670E7B0409042B6D2601E0026EF
:10A1CC0022E7304620E7BC4294D9ACF1020C1F4484
:10A1DC0091E789459FD9023C19449DE73846DFE752
:10A1EC000E46C8E70238294441E700BF4FEA410256
:10A1FC00B2F1E04324BFB3F5001CDCF1FE5C0DD9D9
:10A20C0001F0004C4FEAC0024CEA5070B2F1004F22
:10A21C0040EB830008BF20F00100704711F0804F25
:10A22C0021D113F13872BCBF01F00040704741F4EA
:10A23C0080114FEA5252C2F11802C2F1200C10FAEE
:10A24C000CF320FA02F018BF40F001004FEAC123D2
:10A25C004FEAD32303FA0CFC40EA0C0023FA02F376
:10A26C004FEA4303CCE77FEA625307D150EA01334C
:10A27C001EBF4FF0FE4040F44000704701F000401C
:10A28C0040F0FE4040F40000704700BF19481A49E6
:10A29C00026800608A4217D0002103E0174B5B581C
:10A2AC00435004311648174B42189A42F6D3164ABB
:10A2BC0002E0002342F8043B144B9A42F9D3FBF71B
:10A2CC0040FD00F035F8FEE7114E124830601248A0
:10A2DC00016821F070610160410201600F4C18208F
:10A2EC0020600F490F4808600F48D0F800D0406834
:10A2FC0000470000F04F0020EFBEADDE8CF60008EA
:10A30C0000000020A8000020A8000020001700205A
:10A31C00181002400900000004000140140C014018
:10A32C00000C01404434434400F0FF1FFEE70000E2
:10A33C002DE9804893B0F5F7E3FEAF4CAF4E237890
:10A34C00356833B1AE4B1B68EB1A002BA4BF00234E
:10A35C002370FBF717FF10B1AA4B00221A70AA4BFF
:10A36C001F683B0740F18A81A84B1B681B7A062BA0
:10A37C0000F27881DFE813F0070007003400D40006
:10A38C00100138013801A24B1A78002A00F06A81BA
:10A39C0000221A709F4B022293F800E09E4B1B6820
:10A3AC0093F800C09D4B93F800809D4802F1010981
:10A3BC00835C43FA0EF303F00F0363450CD20B2BB3
:10A3CC009FBF815C10F8090001EA080100EB012134
:10A3DC009CBF944840F823100232102AE5D108E1C2
:10A3EC00914B1A78002A00F03D8100221A708F4B95
:10A3FC008F4A93F802C093F803E059780CF00700E9
:10A40C0041EA00210EF03F00400140EADC001160FF
:10A41C00197950605879890093F806C041EA9E1169
:10A42C0000F0010E41EA8E21916093F807E00CF0E8
:10A43C000F01C90141EA50010EF07F00D16000010B
:10A44C00197A40EA1C1093F809C04900106141EADE
:10A45C00DE110CF0030093F80AE041EA402151614F
:10A46C00D97A0EF01F008001C90040EA9C0041EA35
:10A47C005E1193F80DC093F80EE0D161197B9061D9
:10A48C000CF0070041EA00210EF03F00400140EAC9
:10A49C00DC001162D97B5062187C890093F811C0E2
:10A4AC0041EA9E1100F0010E41EA8E21916293F86F
:10A4BC0012E00CF00F01C90141EA50010EF07F00CF
:10A4CC00000140EA1C10D162D97C106393F814C0CF
:10A4DC00490041EADE110CF0030093F815E041EA63
:10A4EC00402151630EF01F00997D8001DB7D40EA15
:10A4FC009C00C90041EA5E119063D807D1634CBF40
:10A50C0040F21471AD21116499074CBF40F21471E3
:10A51C00AD2113F0080F516414BF03230123A2E0F3
:10A52C00444A1378002B00F09D8000231370424A9C
:10A53C00DFF828E1107841490EEB400CB1F80080AF
:10A54C009CF803909CF8041041EA0921884540F0DE
:10A55C0089809EF80110012904D0812940F0838064
:10A56C00032300E00B46102884BF102111703449DE
:10A57C0092F800E00022D0B2704501F1020172D2D3
:10A58C0011F802CC11F8010C40EA0C20DFF8D0C015
:10A59C002CF812000132EEE72A4B1A78002A61D00F
:10A5AC0000221A70284B1A789946A82A5AD1DB7CBB
:10A5BC00002B57D1984609EB4803D8781B7903EB4D
:10A5CC000020FEF7AFFC2149FEF7B8FD2049FEF74D
:10A5DC00F7FBFEF7EBFE1F4B43F8280008F10108D0
:10A5EC00B8F1080FE7D104E01B4B1A78D2B3002264
:10A5FC001A70012337E000BF17060020F416002064
:10A60C00A800002018060020D00F0020CC0F00203E
:10A61C0069090020060F0020000F0020070F002002
:10A62C00590900205C080020E6090020CD09002013
:10A63C00CC0800209D090020A00900209E090020C4
:10A64C00A40900209609002081090020CDCCCC4023
:10A65C000080BB438C0800205A080020A109002070
:10A66C00AC0800200023DA0741BF83F00203944AB0
:10A67C000121C3F3400344BF11702370780406D545
:10A68C00904A13790BB1002111718D4A137044F269
:10A69C0008033B403BB18A4B1B7823B105F5C33310
:10A6AC00884AA0331360F9070CD5864B9A795979EF
:10A6BC008A421FBF0122227005F5C332A0321CBF93
:10A6CC001A609971BA0409D500237F4A32F8132015
:10A6DC00002A40F0B18001330C2BF6D1784B794C29
:10A6EC001B7823B9794B1B68EB1A002B04DBF7F7AB
:10A6FC0003FD0123E37187E0A7687B1CA360002F97
:10A70C007CD1734B1B681B0778D5E368EB1A002BC5
:10A71C0074DB05F5C335A03563696E48E560984771
:10A72C006C486D4B01461A78FBF730FB6B4802788E
:10A73C00550713D5E368A3613B46694900251944C5
:10A74C00A1F8065163495D5A66495D5206315D5266
:10A75C000233062BF1D122F00402027094F8283057
:10A76C0083B15C4B5E491A88B1F80601121A1A8043
:10A77C00B1F808015A88B1F80A11121A5A809A884D
:10A78C00521A9A80A1694F4A002937D0D36802F136
:10A79C001C005B1A54498B4202F122011CD8534A0B
:10A7AC00D36883F48043D36000234A4A30F913E022
:10A7BC0032F813205D0017B2BE45C4BFDFF824E1A8
:10A7CC002EF8132031F905E00133BE45BCBF484FCC
:10A7DC00EA53032BE9D111E00023464D936130F984
:10A7EC00137031F9132001333A44022792FBF7F22C
:10A7FC00032B25F8022FF2D1FAF7DEFEA368012B0A
:10A80C00C2BF304B00229A60FAF722F8344B30600A
:10A81C00DB7BE56A63B1384B0FA8DB6898479DF882
:10A82C003C308BB9354B1868401B96280CD584E509
:10A83C00401B002808DA80E501232370214A05F526
:10A84C00C333A033136049E7D4F81C2133682C4878
:10A85C001344E3622B4B1B4D1E68274B5B689847D8
:10A86C00274894F8F9220146FBF790FA264B1B88EF
:10A87C00002B00F0A1802B6B05F134071B784035C1
:10A88C0003934FF00008204B4FEA4809B3F800A09F
:10A89C00BAF57A7F02BF00233B602B61184B33F96A
:10A8AC0018003B6803443B60FEF740FB2B69013307
:10A8BC00012B2B612AD1002368602860AB6050E02B
:10A8CC0018060020A800002038090020EC05002004
:10A8DC00E006002014070020FB160020860600204E
:10A8EC00E8090020C40000207FC3C901001001400A
:10A8FC00CA000020EC0A002060160020F41600208C
:10A90C000E07002048070020F8160020D5F800C0DC
:10A91C0006936146CDF810C00590FEF751FA069BE0
:10A92C0083461846FEF702FB01465846FEF706FC26
:10A93C00DDF810C001466046FEF744FA0346059A5E
:10A94C001946686010460493FEF73AFA01465846D9
:10A95C00FEF740FBA968FEF735FA049BE8602B6014
:10A96C00A860684ADFF8C0B10023BAF1010F29F8DA
:10A97C00023029F80B30DFF8B4A128D1286901285E
:10A98C0007DD0138FEF7D2FA0146E868FEF7D6FB80
:10A99C0000E0002002F072F9039A7AB1049010469C
:10A9AC00FEF7C4FA049B01461846FEF7CFFC28B10B
:10A9BC004FF47A73AAF8003000231CE03B684FF484
:10A9CC007A7203F5FA7393FBF2F32BF8093008F162
:10A9DC000108B8F1030F07F1040705F114057FF422
:10A9EC0052AFBAF80000012801D1F9F7EFFEBAF81E
:10A9FC000030013BDEE7444D424905F17C0031F863
:10AA0C00132030F81300121A21F813200133032BF2
:10AA1C00F1D13E4B1B6813F0020300F01A83D5F8FA
:10AA2C00883005F190009847394B05F19000394F6B
:10AA3C001A780146FBF7AAF93B8805F19008BE4647
:10AA4C00002B40D0D5F898000023BEF800203249E6
:10AA5C00B2F5C87F04BF002241F823204FEA8309D6
:10AA6C0038F913C051F80920274D624441F80920E8
:10AA7C00002128F8131020F813100133032BE4D114
:10AA8C003B88012B1CD1D5F89C304FF4C87EC833C1
:10AA9C0093FBFEF30380D5F8A020C83292FBFEF2A4
:10AAAC004280D5F8A4301D4AC83393FBFEF31288BC
:10AABC009B1A8380A6F85810A6F85A10FAF77CFD5A
:10AACC003B88013B3B80164B1B68590740F191803A
:10AADC00144D2B88AE46322B2AD1D4F898301A88D4
:10AAEC00A4F8A8205A889B88A4F8AA20A4F8AC3013
:10AAFC00B6F85830A4F8AE30B6F85A30A4F8B030E6
:10AB0C0018E000BF0E070020A8000020E00600207F
:10AB1C00FA16002092060020440100201E0000209E
:10AB2C00D00F00209406002024010020F8160020ED
:10AB3C00002B3ED0D4F898900023BEF800208E490C
:10AB4C00322A04BF002241F823204FEA830C38F943
:10AB5C00130051F80C20894F024441F80C200022BC
:10AB6C0028F8132029F813200133032B1146E4D1C4
:10AB7C002B88012B1AD1824A0C201170814A137038
:10AB8C00F9F724FEB7F8A830A9F80030B7F8AA30C6
:10AB9C00A9F80230B7F8AC30A9F80430B7F8AE30E9
:10ABAC00A6F85830B7F8B030A6F85A302B88013BCD
:10ABBC002B80754B1A78E2B100221A70D4F8B4309D
:10ABCC00322093FBF0F3D4F898100B80D4F8B83003
:10ABDC0093FBF0F34B80D4F8BC3093FBF0F36B4851
:10ABEC0000881B1A8B80A6F85820A6F85A20FAF772
:10ABFC00E3FCD4F89820B4F89030118800265B1A46
:10AC0C00A4F890305188B4F892305B1AA4F89230C2
:10AC1C009288B4F894309B1AA4F89430F9F718FE83
:10AC2C00D4F8C0700546C31B18460393FEF77AF997
:10AC3C00D4F8C4100490FEF7CDF9C4F8C0503546D2
:10AC4C00D4F8C880524F98F800B00590514A0DF1D5
:10AC5C00240932F91500FEF769F90599FEF7BAF9DE
:10AC6C0049F82500BBF1000F2BD05846FEF75EF9D2
:10AC7C0001464FF07E50FEF761FA0246DFF828A13C
:10AC8C0011464FF07E500792FEF79AF85AF82510AD
:10AC9C00FEF7A0F9AAF13C01069031F91500FEF778
:10ACAC0045F9079A1146FEF795F9DDF818C00146EB
:10ACBC006046FEF787F84AF82500FEF751FB7880CE
:10ACCC0003E0354A32F815207A8037F9022F013526
:10ACDC00032D02FB0266B9D1DFF8B0A064235E43FA
:10ACEC00BAF800302D485B4396FBF3F6493E09A9B0
:10ACFC00B6B2FAF74FF93B2ED8F8045011D91F4EC3
:10AD0C00B6F9E400FEF712F9D6F8E05001462846F1
:10AD1C00FEF71CFB224B002848D01A7842F00802A0
:10AD2C0047E04FF07E512846FEF74CF801464FF0B5
:10AD3C007E50FEF703FA06464FF0000B174B2846E1
:10AD4C0053F82B100693FEF745F91649059031F987
:10AD5C001B00FEF7EBF8059A01461046FEF732F899
:10AD6C003146FEF737F9069B43F82B000BF1010B2C
:10AD7C00BBF1030FE2D1C2E75C010020A800002068
:10AD8C00960600208F060020900600201E00002052
:10AD9C00060700200E07002038010020800100204B
:10ADAC008606002008070020740100201A7822F083
:10ADBC0008022946D4F8DC001A7001F05DFFBA4D88
:10ADCC00D4F8D8302860D4F8DC00D4F8E020014660
:10ADDC0003F1004B0692FEF7FDF8069A059011461A
:10ADEC001046FEF7F7F8059B01461846FDF7EAFFFB
:10ADFC0001F044FF0146584601F03EFFAB49686044
:10AE0C002868FEF7E7F801F0ABFEDFF8E0B2A749DF
:10AE1C00ABF800006868FEF7DDF801F0A1FEA44B6A
:10AE2C00ABF802001B681A0732D5A24809A9FAF739
:10AE3C00B1F8D8F808904FF07E514846FDF7C2FFA4
:10AE4C0001464FF07E50FEF779F907464FF0000BA4
:10AE5C00984A484652F82B100692FEF7BBF89649D2
:10AE6C00059031F91B00FEF761F8DDF814C00146BE
:10AE7C006046FDF7A7FF3946FEF7ACF8069A42F894
:10AE8C002B000BF1010BBBF1030FE1D1104641E09C
:10AE9C00DFF828B249465846FAF77CF8DBF8000090
:10AEAC00DBF80830DBF80420014605930692FEF728
:10AEBC0091F8069A814611461046FEF78BF801462A
:10AECC004846FDF77FFF059B814619461846FEF75D
:10AEDC0081F801464846FDF775FF01F0CFFE0021D1
:10AEEC008146FEF70BFAA0B9DBF800004946FEF7E5
:10AEFC0025F94946CBF80000DBF80400FEF71EF9F3
:10AF0C004946CBF80400DBF80800FEF717F9CBF83C
:10AF1C0008006A48FBF734FF694B6A4918800498AB
:10AF2C00FEF758F82B68814603F100430C936B68CD
:10AF3C00654D03F100430D93614BB3F90000FDF730
:10AF4C00F5FF624900F10040FEF744F80E90B5F9A8
:10AF5C000000FDF7EBFF0F90B5F90200FDF7E6FFDF
:10AF6C001090B5F90400FDF7E1FF0CA911900FA8A2
:10AF7C00FAF710F898F80130012B18D1544B1B78C4
:10AF8C005B070ED4D6F8F400402390FBF3F3C01A01
:10AF9C00FDF7CCFF1199FDF715FFFEF7E1F9C6F8A7
:10AFAC00F400D6F8F400402390FBF3F001E0BAF87B
:10AFBC000000FDF7BBFF01461198FDF701FFD4F827
:10AFCC00FC1011904846FDF7FDFE01464846FEF781
:10AFDC00B5F8D4F8F850064629461198FDF7F0FE5E
:10AFEC0001463046FDF7F6FF01462846FDF7EAFE1E
:10AFFC000646C4F8F8000F9801F0B2FDD4F80051E1
:10B00C002978F9F7C5FED4F804311844C4F80401C2
:10B01C00109801F0A5FD2978F9F7BAFED4F808319B
:10B02C001844C4F80801304601F09AFD6978F9F724
:10B03C00AFFED4F80C31274A184403991368C4F8AE
:10B04C000C011944D4F8103111600133C4F81031DB
:10B05C0005E0A5F89030A5F89230A5F89430F9F7F2
:10B06C00F7FB1D4D1D4BDFF888801860D5F81431A7
:10B07C00C5F81401C31A9BB2A8F800301846FDF7A6
:10B08C0051FF1049FDF7A6FF154C164F2368386089
:10B09C0093F85230AA46A34663BB134B1B7C002B80
:10B0AC0000F0AE804FE000BF781100204C3D0F4403
:10B0BC00E006002090010020140700200000002072
:10B0CC0036070020BD3786350807002035FA8E3C40
:10B0DC00FD160020F0160020A8000020F416002019
:10B0EC004807002004100020E80900203207002047
:10B0FC00DC060020D5F818010021FEF7FFF840B15E
:10B10C00D5F81C01FDF70EFFA949FDF763FFC5F843
:10B11C0018010026DFF8D09239F91600FDF706FF6A
:10B12C00DBF80030A34993F8522001EBC601DAF8A2
:10B13C001831F9F783FCFEF713F929F816000136DC
:10B14C00032EE7D1A9E79C4EB8F80000FDF7EAFE04
:10B15C003B6806F59E710122B5F83891F9F76EFC43
:10B16C00FEF724F980B2B9FBF0F0EB79471CBFB2C3
:10B17C00A5F8447113B3B6F9469100238E4E8F4A4D
:10B18C0006F5A47838F9131006F5A87E09FB01F131
:10B19C0032F813C03EF813202EF813C0C2EB0C0A81
:10B1AC003AB291FBF2F2524428F813200133042BEB
:10B1BC00E4D10023F371A6F8460104E0B6F8463159
:10B1CC00013BA6F84631B5F946017B4A00284FF001
:10B1DC00000313DDB2F944517949A1F1080232F9A7
:10B1EC00132031F81310424392FBF5F28A1A73497B
:10B1FC0021F813200133042BEED101E0A2F84631E3
:10B20C006E4BB3F906106F4BD3F800E00493BEF805
:10B21C000A2091420FDBB1F5FA6F9EF80750BFBFC1
:10B22C008B1A6B43A2F5FA6593FBF5F5ACBFC5F130
:10B23C006405643500E06425634B2268B3F828C1CB
:10B24C0093F9F23005929BB216460693002240F217
:10B25C00E6305A4B4FEA420933F91280CCEB080323
:10B26C0003F2F314844203D8002BB8BF5B4201E015
:10B27C004FF4FA73022A03934FF06400059B2ED00F
:10B28C0093F811412CB1039BA342CCBF1B1B002391
:10B29C000393039B4D4C93FBF0F76FF0630B34F867
:10B2AC0017A00BFB073B013734F917400FFA8AF74D
:10B2BC00E41B04FB0BF494FBF0F4454B544423F8CF
:10B2CC0009400EEB02042479039B6343414C93FB2E
:10B2DC00F4F364339BB26B4393FBF0F030E093F8E0
:10B2EC0012412CB1039BA342CCBF1B1B0023039325
:10B2FC00039B314C93FBF0F06FF0630A0AFB003BAD
:10B30C0004EB400704EB4000B7F95871B0F95A014F
:10B31C00069BC01B00FB0BFB9BFBFAFBC7EB0B0B51
:10B32C000BFB03FB2A4BA3F804B0039B9EF806000F
:10B33C00002BB8BF5B424343264893FBF0F06430CC
:10B34C0073786427434393FBF7F3234C022AA354EB
:10B35C00F37A224C00FB03F393FBF7F3A354737DB6
:10B36C001B4C00FB03F090FBF7F01D4B98541D4B4E
:10B37C000FD1E0459F700FDBDFF84CB0BBF82A21F2
:10B38C005D46914232DBB1F5FA6FA8BF4FF4FA611A
:10B39C002DE0E0459D5404DA34F809305B4224F882
:10B3AC0009300132032A06F101067FF450AFE3E7BE
:10B3BC00BD378635C8010020A800002014090020E4
:10B3CC00F801002044070020E8090020BA070020FB
:10B3DC00E00F00200CFEFFFF601000200E0200208A
:10B3EC0078100020E80F00200E0700201146891A63
:10B3FC004FF47A735943C2F5FA62B1FBF2F1642748
:10B40C0091FBF7F2DFF8B0E26FF063033EF8120045
:10B41C0003FB021101323EF9122003B2D21A51433E
:10B42C0091FBF7F30344E380934B944E1B885F0628
:10B43C003FD5934A934B10881B88181A00B2FDF71E
:10B44C0075FD9149FDF7C6FD90490746FDF7BAFC1D
:10B45C00F9F7ADFC80463846F9F7A9FC0746B6F972
:10B46C000200FDF763FD8146B6F90000FDF75EFDB5
:10B47C0041468246FDF7AEFD394603904846FDF73E
:10B48C00A9FD039B01461846FDF79AFCFDF768FFE2
:10B49C00414630804846FDF79DFD39468046504672
:10B4AC00FDF798FD01464046FDF78CFCFDF758FF73
:10B4BC007080774B1B689E0772D545F20721754B40
:10B4CC00754E1A68D6F86C31D31A8B4268DDDFF8EA
:10B4DC00DC81C6F86C21FAF72DFD98F800306F4F1F
:10B4EC00032B3B8822D10A2B2CD90023282088F847
:10B4FC000030F9F7D4F9FAF71DFD694B1888FAF703
:10B50C0003FD684B1A68D37890FBF3F001300828E0
:10B51C00654BA8BF08201870537980B24343A6F836
:10B52C00703113795843A6F872010BE00A2B09D835
:10B53C0003235D4A88F8003000231370A6F870319D
:10B54C00A6F8723198F80030584A012B0CD002D36F
:10B55C00022B1CD024E0B6F870213B889A421FDDE8
:10B56C00012388F8003010E03988B6F872318B422C
:10B57C0002DD0223137010E0474BB3F87031013336
:10B58C00994202DD002313700AE0082006E0B6F8A9
:10B59C0072313A8801339A42E2DC0720F9F716F946
:10B5AC003B4B434E1A6812F4006F00F0A580394BE8
:10B5BC0039481968D0F87431C3EB010845F20723F8
:10B5CC00984540F39980DFF8DCE0B4F90670DEF8BA
:10B5DC0000A04FF47A739AF80AE0C0F87411BEF127
:10B5EC00010F98FBF3F8BBF8E210A7F57A77DFF8B8
:10B5FC00CC9004D064D3BEF1020F1BD063E0D0F822
:10B60C007821082792FBF7F1521AC0F8782192FBA7
:10B61C00F7F240F6E44792B27A430021A0F87C118D
:10B62C00BAF80810C1EB12325343BAF9062093FB57
:10B63C00F2F346E03078BAF808304007C9F8003029
:10B64C0041D51C4805930392F9F794F8039A059B8E
:10B65C0018B912F0100F18BF002707FB07F23221A0
:10B66C0092FBF1F21744BAF9062057434FF47A7261
:10B67C0097FBF2F73B4424E0E4060020E00F0020A7
:10B68C00D60600203607002035FA8E3CDB0FC93F6A
:10B69C00D00F0020F4160020A8000020C80F0020B6
:10B6AC00380F0020340F002034000020E816002052
:10B6BC00FD160020020B0020A207002040070020EE
:10B6CC000023C9F80030D9F80020984F02FB08F885
:10B6DC00D7E900014FF47A7298FBF2F810EB0802EC
:10B6EC0041EBE87310461946914A0023C7E9000163
:10B6FC00FDF77CFE8F4B1860DFF88892D9F800308C
:10B70C00DB0402D50A20F9F761F8DFF87C82D8F85F
:10B71C000020002A45D0DFF874A28749DAF80030FF
:10B72C00096899423DD8854B854F18785168B0B956
:10B73C0001221A703B88CB5CD3B1824B1A70FAF79A
:10B74C002DFD3B88A3B9D8F800301B78053B012BA5
:10B75C000ED8F9F77DF87C4BC3F8880108E000227D
:10B76C001A703B88CB5C1BB1764B1A70FAF716FD3E
:10B77C00D8F800303A885B6871499B5CFE2B02D18B
:10B78C0000230B800DE0FF2B02D1F9F70DF808E038
:10B79C00DAF800000A2707FB03036748013203604D
:10B7AC000A8033785F0704D5684B4FF480425A61A6
:10B7BC0035E0D9F80020D0075EBF654943F001039E
:10B7CC000B70644B1B7819075EBF337823F00103B1
:10B7DC003370D30242BF337823F0010333705E4BD6
:10B7EC001A88584B1AB15D4A1268970702D45C4A02
:10B7FC00128832B102221A70337823F001033370AD
:10B80C0004E03178C80758BF02221A70F9F720F803
:10B81C00544B1B68C01A002801DBFAF7BFFC524BD3
:10B82C001F780393002F00F0F380504B1A68049399
:10B83C00002A00F0BE85049B186803685B68984773
:10B84C00002800F0B685494B494D186803689B6881
:10B85C0098470928014601D03F285BD14FF00008DA
:10B86C002F684546DFF8289137B14248D9F80010C7
:10B87C003A4601F063F810B9C84605B94D463E4B3F
:10B88C0009F110099945EFD3EDB1D5F80090D8F82E
:10B89C0000A0374A136819F803E01AF80300704542
:10B8AC0011D1344950B92D2B08D803F1010EC2F82F
:10B8BC0000E02022CA5401F80E0004E001F803E075
:10B8CC0001331360E5E72A4BDFF8A0A01A6899460C
:10B8DC000AB1454512D02948FCF786FF454509D8E1
:10B8EC0055F8100BFCF780FFDAF800000921F9F786
:10B8FC0024F8F3E72248FCF777FF0027D9F800304B
:10B90C009F4298D21B4BDAF80000D95DF9F715F875
:10B91C000137F3E72B68002B40F02B85042840F00F
:10B92C0016871448F8F716FA00F043BD28020020D9
:10B93C00407E050038070020CC070020C8070020F7
:10B94C00D0070020D40F0020A800002000100140D8
:10B95C00FD1600208606002092060020E00600203E
:10B96C00F8160020D80F0020FE160020E01600204C
:10B97C00980700206807002088E4000888E4000885
:10B98C008DE40008E8060020D4070020E41600200F
:10B99C0038E30008059BDFF844A3186803685B686C
:10B9AC00984758B3DAF8000003689B689847C84B6F
:10B9BC0081461B6893F84810002938D124286FD190
:10B9CC00012283F84820DFF80893D9F8003093F867
:10B9DC004820062ADED193F84900F7F752FB0028DD
:10B9EC0000F08780DFF8E882D8F800309879FCF70F
:10B9FC0079FED8F80030002283F84820B54B93F834
:10BA0C002832002B40F0A3844C37982F00F0D184BF
:10BA1C00B14AD31993F84A100129F5D1DFF8B08255
:10BA2C00BA58C8F80030AD4B1A600593B2E701293B
:10BA3C0004D14D2814BF00220222C2E7022904D1EE
:10BA4C003C2814BF00220322BBE703290AD140285B
:10BA5C004FF000029FBF1A71DA715871987198BF3C
:10BA6C000422AEE7042908D19A7983F8490080EAC8
:10BA7C00020983F806900522A3E70529A3D1597979
:10BA8C001A799142997906D941409971511C1971D1
:10BA9C001344187297E781420CBF0622002290E7EC
:10BAAC0033788F495B078ED42328DAF8003013D112
:10BABC000691039901220A708A4A8B481360854AC1
:10BACC00C2F82432FCF790FE8848FCF78DFE0699EC
:10BADC000B7843F002030B70854B1B681B784B45AE
:10BAEC0001BF844A844B1A60844A04BF844BDA60D9
:10BAFC0069E7D9F8002092F849304C2B00F09A8372
:10BB0C0059D8372B00F0E28317D8292B00F05C832F
:10BB1C0009D8252B00F02E83272B00F03783232BFD
:10BB2C0040F011862DE2332B00F0BE83352B00F054
:10BB3C0060822D2B40F0078657E3412B00F0B98330
:10BB4C0009D83C2B00F010813E2B00F00081392BE2
:10BB5C0040F0F98527E3442B00F0F0834A2B00F0EA
:10BB6C00FF80432B40F0EF85F8F75CF80023AB60C7
:10BB7C00F8F762F88046F8F75FF8AB6808EB00401E
:10BB8C000343AB60F8F74EF885F82201F8F754F848
:10BB9C00A5F8EC00F8F750F8A5F8EE00F8F74CF81B
:10BBAC00A5F8F000F8F748F8A5F81201F8F744F8F2
:10BBBC00A5F81401C6E3D02B00F0BA8247D8CC2BE1
:10BBCC0000F0568208D8C82B77D0CA2B00F0DA8048
:10BBDC004E2B40F0B8853AE3CE2B00F0BD8240F2FC
:10BBEC00B282F8F729F86FF4AF6E00EB0E039BB23C
:10BBFC00C62B98BFA5F82801F8F71EF8A5F8D400B5
:10BC0C00F8F71AF8A5F8D600F8F716F8A5F8D80042
:10BC1C00F8F712F8A5F86A01F8F704F8F8F702F843
:10BC2C00F8F700F8F7F7FEFF85F81701F7F7FAFFBA
:10BC3C0085F82401F7F7F6FF324BD3F80080F7F7BD
:10BC4C00FBFF00EB80004000A8F85600ABE2D62BBF
:10BC5C0000F0628208D8D32B2AD0D42B00F0728348
:10BC6C00D22B12D000F06FBDEF2B61D005D8D82BA2
:10BC7C0040F069854FF0000816E1F22B00F062836A
:10BC8C00FA2B00F0738200F05EBD337803F00403EE
:10BC9C0003F0FF08002B40F05583F7F7C3FF022891
:10BCAC0085F8F00440F24A82174B83F8F08445E2A1
:10BCBC00F7F7C2FF154B188044E392F805804FEA62
:10BCCC005808B8F1120F23D9F9F764FF3AE300BF13
:10BCDC00D8060020A800002034020020DC1600202A
:10BCEC00FD160020E0160020BDE400088DE40008DD
:10BCFC009C070020EFBEADDEF04F00200400FA05DB
:10BD0C0000ED00E048070020E8090020D4060020E0
:10BD1C004FF00009C14507D2F7F78EFFC94B23F846
:10BD2C00190009F10109F5E7C74B01221A7109E362
:10BD3C00DFF81883D8F80090F7F77EFFA9F85A00BF
:10BD4C00D8F80080F7F778FFA8F85800FAE2F7F770
:10BD5C0069FF85F87201F7F765FF85F87101F1E26B
:10BD6C00F7F76AFFA881EDE2DFF8E082D8F80090DF
:10BD7C00F7F758FF89F80000D8F800301878FBF76F
:10BD8C0073F8DFE2B14B1A6898461278022A6ED12A
:10BD9C004FF00008DFF8B49208F1080AD9F8003027
:10BDAC000593F7F73FFFFDF7BDF8A949FDF7C6F975
:10BDBC00059B43F82A00D9F800A0F7F733FF08F1E8
:10BDCC000A030AEB830AFDF7ADF8A249FDF7B6F9B1
:10BDDC00D9F80030CAF804000593F7F723FFFDF7F4
:10BDEC00A1F89D49FDF7AAF908F10E0A059B08F187
:10BDFC000108B8F1030F43F82A00CBD1B8F1070FB3
:10BE0C00D9F800A01AD1F7F70DFFFDF78BF8904980
:10BE1C00FDF794F9CAF84400D9F800A0F7F702FF2F
:10BE2C00FDF780F88A49FDF789F9CAF84800D9F876
:10BE3C0000A0F7F7F7FE8AF84C0012E0F7F7F2FED5
:10BE4C00C2448AF80100D9F800A0F7F7EBFEC2440F
:10BE5C008AF80B00D9F800A0F7F7E4FEC2448AF880
:10BE6C00150008F10108B8F10A0FC7D16AE24FF0CA
:10BE7C000009D8F800A0F7F7D5FECA448AF80100EB
:10BE8C00D8F800A0F7F7CEFECA448AF80B00D8F811
:10BE9C0000A0F7F7C7FECA4409F10109B9F10A0F6E
:10BEAC008AF81500E5D14DE2DFF8A09108F1080AF7
:10BEBC00D9F800300593F7F7BFFEFDF733F8664964
:10BECC00FDF73CF9059B43F82A00D9F800A0F7F7D9
:10BEDC00B3FE08F10A030AEB830AFDF723F85E4967
:10BEEC00FDF72CF9D9F80030CAF804000593F7F7E0
:10BEFC00A3FEFDF717F85849FDF720F908F10E0AD3
:10BF0C00059B08F10108B8F1030F43F82A00CBD1C7
:10BF1C00B8F1070FD9F800A01AD1F7F78DFEFDF78D
:10BF2C0001F84D49FDF70AF9CAF84400D9F800A008
:10BF3C00F7F782FEFCF7F6FF4749FDF7FFF8CAF862
:10BF4C004800D9F800A0F7F777FE8AF84C0012E009
:10BF5C00F7F772FEC2448AF80100D9F800A0F7F78F
:10BF6C006BFEC2448AF80B00D9F800A0F7F764FE08
:10BF7C00C2448AF8150008F10108B8F10A0FC7D1BC
:10BF8C00E0E1F7F74FFE132882463FF69DAEDFF84F
:10BF9C00BC90D9F80080F7F745FE00232F490C22FE
:10BFAC0002FB0312117A81421FD1137808EB8A0825
:10BFBC0088F87930F7F736FE88F87A00F7F732FE12
:10BFCC0088F87B00F7F72EFE254A264B88F87C0074
:10BFDC001A60D9F80000244B18607930F9F75CFD31
:10BFEC00224B80F001001870ACE101331C2BD5D131
:10BFFC006AE6F7F717FE0B2881463FF665AE134B42
:10C00C00D3F80080F7F70EFE03283FF65DAE06234B
:10C01C0003FB098888F8CE00F7F704FE88F8C900FE
:10C02C00F7F700FE88F8CA00F7F7FCFD88F8CB009C
:10C03C00F7F7F8FD88F8CC00F7F7F4FD88F8CD0099
:10C04C0080E100BF14090020A80000204807002050
:10C05C00000020410000C84200007A4478D5000856
:10C06C00BC0A0020CC060020D00600201C000020BA
:10C07C005379092B7FF628AE049BD3F80080F7F791
:10C08C00D1FD049B88F80000D3F80080F7F7CAFDB7
:10C09C0088F80100F7F7C6FD049B64281B68A8BF4D
:10C0AC0064201871F7F7BEFD049B64281B68A8BFB9
:10C0BC0064205871F7F7B6FD049BFF281B68A8BFD6
:10C0CC00FF209871F7F7AEFD049B6428D3F800802D
:10C0DC0028BF642088F80700F7F7A4FD049B88F8B4
:10C0EC000200D3F80080F7F79DFD049B88F803004D
:10C0FC00D3F80080F7F7A0FDD9F80030A8F80A00B3
:10C10C005B790A2B40F21E81C84BD3F80080F7F7FD
:10C11C0089FD88F8080015E18046F7F78DFDC44BC2
:10C12C0023F8180008F10108B8F1080FF5D109E15E
:10C13C003378580700F10681FBF772FAF8F7D0FF55
:10C14C00F9F79CF8FEE03378590700F1FB80B94B06
:10C15C004FF4C8721A80F5E033785A0700F1F28078
:10C16C00B54A137843F004031370EBE033785B07A4
:10C17C00E4D5E8E2A860F7F75FFD8046F7F75CFDD1
:10C18C00AB6808EB00400343AB60DBE0F7F754FD12
:10C19C00A5F8EC00F7F750FDA5F8EE00F7F74CFD0D
:10C1AC00A5F8F000CEE0F7F73DFD85F80C01F7F7A8
:10C1BC0039FD85F81001F7F735FD85F80F01F7F714
:10C1CC0031FD85F81101BDE0F7F736FDA5F8120138
:10C1DC00F7F732FDA5F81401F7F724FD85F81601E1
:10C1EC00F7F72AFDA5F81801ACE0F7F71BFD85F869
:10C1FC002201F7F721FDA5F82C01F7F71DFDA5F895
:10C20C002801F7F719FDA5F82A01F7F70BFDD8F867
:10C21C00003085F823015B79DFF85492082B40F24B
:10C22C009180F7F709FDA9F82E01F7F705FDA9F89C
:10C23C00300187E0F7F7F6FC85F86801F7F7F2FCB8
:10C24C0085F86901F7F7F8FCA5F86A017AE092F82D
:10C25C0005800323B8FBF3F8B8F1120F3FF634ADA9
:10C26C00DFF80C924FF0000AC2456BD2F7F7DAFCFC
:10C27C0089F83201F7F7E0FC40F2ED23984205DD36
:10C28C0040F6CA039842A8BF184601E040F2EE20DF
:10C29C00A0F2EE20192390FBF3F00AF1010A89F8C1
:10C2AC00330109F10209DFE7F7F7BCFC85F824013B
:10C2BC0048E08046F7F7B6FC05EB080308F10108E7
:10C2CC00B8F1080F83F81A01F4D13BE053794FF021
:10C2DC000709B3FBF9F9C9EBC9029B1A13F0FF0F5D
:10C2EC007FF4F2AC5FFA89F909F1FF395FFA89F949
:10C2FC00B9F1FF0F26D0F7F795FC5FFA80FA4FFAE9
:10C30C008AF0F7F7FDFF804600283FF4DDAC80F89B
:10C31C0000A0F7F791FCA8F80200F7F783FC88F867
:10C32C000400F7F77FFC88F80500F7F77BFC88F82A
:10C33C000700F7F777FC88F80600D5E73F4B01229A
:10C34C0083F828220020F6F799FEFFF74BBB3C4BF5
:10C35C00F858F8F7EFFA18B93220F8F7A0FAF6E720
:10C36C00FAF7CEFCF8F792FE364A374BDA60FFF755
:10C37C004BBB0C2800F0ED810A2940F01B82334F97
:10C38C003348FCF731FA3846232100F0C0FA08B1E3
:10C39C00C01B28602B68002B40F032822B602B488E
:10C3AC000021302200F07DFA039B1B78002B40F01B
:10C3BC00D381284B9B680BB127489847274B284DB6
:10C3CC001B6813F0080F56D0A188264A01F14503CB
:10C3DC009BB28A2B1288244B4CD8244800884707E0
:10C3EC0048D51B88D21A92B293B218B2B330BCBFE4
:10C3FC0002F5B4739BB210481AB2B32A0078C4BFCA
:10C40C00A3F5B4739BB200079BF8F22033D552B25C
:10C41C00524253432A681BB2527A53436FF01D02A7
:10C42C0093FBF2F30B44A38025E000BF44070020EC
:10C43C00C21600209206002086060020A8000020CC
:10C44C00340200200400FA0500ED00E0680700202B
:10C45C001DEB000860160020D2020020E006002030
:10C46C004807002036070020D4060020E4060020F0
:10C47C00E80900201A80BB4B1B7843B1BA4BB3F9C7
:10C48C000620BBF82A319A42DCBF0023A3802B681C
:10C49C00B64F93F81881B8F1000F4FD0B44B1B88EE
:10C4AC009B074BD0D7F8D800D7F8DC300146039364
:10C4BC00FCF790FD039B824619461846FCF78AFD53
:10C4CC0001465046FCF77EFCD7F8E0908246494680
:10C4DC004846FCF77FFD01465046FCF773FC00F024
:10C4EC00CDFB01464846FCF729FEA2498146FCF7E4
:10C4FC0019FFF8B9484600F06FFBD7F82C12FCF77F
:10C50C0069FD00F02DFBB0F5617FA8BF4FF46170A1
:10C51C00FCF70CFD9849FCF711FEF8F748FC814636
:10C52C004046FCF703FD4946FCF754FD00F018FBB0
:10C53C0080B200E00020E3881844E0808F4B28682C
:10C54C00BBF8FE2000938E4B1D688E4B196800F1D2
:10C55C005803A8478C4B8D491D78032D1AD9D7F851
:10C56C003032B3F802E0BEF5FA7F13D2B4F904000E
:10C57C00B1F904C080EAE078A8EBE078CEF10002D3
:10C58C00C8EB02039C4504DB0EEB08036345A8BF14
:10C59C0063468B80B4F806B0B1F80280B1F8009015
:10C5AC00D7F83072B1F904A0794C0023AB4204F1F6
:10C5BC0010043DD20FFA8BF00493FCF7B7FC54F83F
:10C5CC00181CFCF707FD03900FFA88F0FCF7AEFC83
:10C5DC0054F8101CFCF7FEFC039A01461046FCF7BD
:10C5EC00F1FB03900FFA89F0FCF7A0FC54F8141C33
:10C5FC00FCF7F0FC039A01461046FCF7E3FB0390B2
:10C60C0097F9010040420AFB00F0FCF78FFC54F84C
:10C61C000C1CFCF7DFFC039A01461046FCF7D2FB1E
:10C62C00FCF79EFE049B5B4A22F813000133BDE726
:10C63C00327802F0040202F0FF03002A79D0564B44
:10C64C00012193F80380534B1A88A94214B207D2E4
:10C65C0033F9112001319442B8BF1446A2B2F4E769
:10C66C004E49DFF84CE10968DEF800E0488803EB3E
:10C67C0045058442C8BF101A494AC8BF80B2146825
:10C68C00394A04F48059B2F90660384AD8BF002000
:10C69C00D2F8F472D2F830C23E4A04F01004AA4226
:10C6AC003DD013881B1A9BB222F8023B1BB2B9F186
:10C6BC00000F0CD0B7F80EA05645C7BFBEF802A0AD
:10C6CC00B1F802B0B1F804A0BEF800B006E0B1F8C1
:10C6DC0002B0B8F1000F0AD0B1F804A0534503DB47
:10C6EC005B45A8BF5B469A4622F802ACD7E7B1F887
:10C6FC0000A0534503DB5B45A8BF5B469A4622F876
:10C70C0002AC3B8A9E42CADA0CB18B8804E09CF8DE
:10C71C000030002BC3D10B8822F8023CBFE7134B2F
:10C72C0093F8F832002B3DF408AEFAF795FAFDF7C2
:10C73C0004BEAB42F3D21B4A32F81310154A22F84E
:10C74C0013100133F5E7F9F725FAFFF74BB90C286D
:10C75C0004D11548FCF748F8144836E07F293BD142
:10C76C00FFF769B81C00002014090020A800002065
:10C77C00E40600208FC2753CEFB6B044020B0020DB
:10C78C0030000020440700207B10002050100020B7
:10C79C00E40200201A0700209816002074110020D3
:10C7AC00D00F0020C216002092E400088DE400088F
:10C7BC00701100200D293FF4E2AD7F2909D12B4ADD
:10C7CC00013B00212A482B60D154FCF70DF8FFF7F0
:10C7DC0032B82F2B3FF62FA8A1F12002D2B25E2A3D
:10C7EC003FF629A813B920293FF425A85A1C2A6022
:10C7FC001E4AD1541F4B1868F8F79FF8FFF71BB867
:10C80C005A1EB95C202901D11346C4E5174A0021F0
:10C81C002B60D154184B194DD3F800902968DFF8D0
:10C82C004CA00846059100F080F8074605993A4659
:10C83C00504600F083F8124A28B91AF807304B44D6
:10C84C005B78590703D010359542E7D306E0954243
:10C85C0004D2781CEB685044984702E00948FBF777
:10C86C00C3FF094B00221A6099E500BF680700203E
:10C87C00B9E40008E01600203C00002038E3000872
:10C88C0088E400089DE400089807002010B5431EBA
:10C89C000A44914204D011F8014B03F8014FF8E718
:10C8AC0010BD03460244934202D003F8011BFAE781
:10C8BC00704700000D4B30B51D6810F8013BEA18AD
:10C8CC00527802F00302012A11F8012B08BF203321
:10C8DC00AC18647804F00304012C08BF20329B1AB6
:10C8EC0001D1002AE9D1184630BD00BF3C00002020
:10C8FC00024610B513461C780132002CFAD1013BCC
:10C90C0011F8012B03F8012F002AF9D110BDC9B27F
:10C91C00034610F8012B1AB18A42F9D11846704718
:10C92C0000290CBF184600207047034613F8012B52
:10C93C00002AFBD1181A0138704700000F4B70B554
:10C94C001E680A44914216D010F8013BF418647822
:10C95C0004F00304012C11F8014B08BF20333519E6
:10C96C006D7805F00305012D08BF20341B1B03D186
:10C97C00002CE7D100E00023184670BD3C000020DD
:10C98C00034610B532B111F8014B013A03F8014BD3
:10C99C00002CF7D11A44934203D0002103F8011B59
:10C9AC00F9E710BD30B5037823B90B78002B18BF0D
:10C9BC00002030BD03461A7801303AB100228C5C5D
:10C9CC0034B19D5CA542F5D10132F8E7104630BD7B
:10C9DC00184630BD00210A2200F0B4B8F0B548B9B1
:10C9EC00106838B9F0BD17F8016B5EB1B542FAD1D9
:10C9FC002BB1204604460F4614F8015BF3E7146094
:10CA0C000370F0BD4DB915602846F0BD17F8016BE9
:10CA1C00AE4207D0002EF9D11C4623460F4613F820
:10CA2C00015BF3E715B10021217000E02B46136088
:10CA3C00F0BD0123FFF7D2BF2DE9F0470F46404C64
:10CA4C00D4F800903D4615F801EB09EB0E0466781E
:10CA5C0006F0080404F0FF060CB12F46F2E774460A
:10CA6C002D2C03D1BD1C7C78012603E02B2C04BF9C
:10CA7C007C78BD1C13B1102B0AD15AE0302C56D146
:10CA8C002C7804F0DF04582C4CD16C781023023530
:10CA9C00002E14BF4FF000486FF00048B8FBF3FABB
:10CAAC000027BE4603FB1A8809EB040C9CF801C056
:10CABC001CF0040F01D0303C0BE01CF0030C1BD01D
:10CACC00BCF1010F0CBF4FF0370C4FF0570CCCEBF7
:10CADC0004049C4210DAB7F1FF3F0AD0D64506D8C1
:10CAEC0001D1444503DC03FB0E4E012701E04FF05E
:10CAFC00FF3715F8014BD7E77C1C73460AD1002E83
:10CB0C004FF0220114BF4FF000436FF0004301605F
:10CB1C002AB911E00EB1CEF100036AB107B1691E5A
:10CB2C00116009E03024002BB2D10823B0E70A23AE
:10CB3C00AEE7302CACD1A3E71846BDE8F08700BFB8
:10CB4C003C00002030B505460C461346034A2946E6
:10CB5C0010682246BDE83040FFF76EBFA0000020F1
:10CB6C0030B5C0F3C755A5F17F021E2A83B001462C
:10CB7C0021DC501C1CDB162A4FEAD1740ADDC1F3F0
:10CB8C00160343F40003963DAB4060424340181932
:10CB9C0003B030BD0F4B53F824502846FCF712F964
:10CBAC00019001982946FCF70BF920F0004333B9AA
:10CBBC00002003B030BDFCF7D3FB03B030BDC0F395
:10CBCC001603C0F3C75043F40003C0F19600C340F2
:10CBDC00DBE700BF48F6000870B58AB0064600F0E7
:10CBEC009BF8224D044695F90030013303D03046B2
:10CBFC0000F000FC10B920460AB070BD304600F0C1
:10CC0C00F5FB4FF07E51FCF7A1FB0028F3D018493F
:10CC1C00012200233046009208930191FCF7D2FDCB
:10CC2C0002460B461348CDE90423CDE9022300F05C
:10CC3C00C1FA95F90030CDE90601022B0BD06846FC
:10CC4C0000F0B6FA38B1089B53B9DDE90601FDF7DF
:10CC5C00CDFA0AB070BD00F0E7FB21230360F2E7C8
:10CC6C0000F0E2FB089B0360EFE700BFA40000208C
:10CC7C0050F6000858F6000800F0B6B970B58AB046
:10CC8C00064600F041FA224D044695F90030013376
:10CC9C0008D0304600F0AEFB20B130460021FCF746
:10CCAC0037FB10B920460AB070BD1A490122002387
:10CCBC003046019100920893FCF784FD2C78CDE965
:10CCCC000401CDE902017CB900220023CDE9062341
:10CCDC00684600F06DFA88B1089BA3B9DDE906013E
:10CCEC00FDF784FA0AB070BD0020002102460B4605
:10CCFC00FCF7E6FE022CCDE90601E9D100F094FB2D
:10CD0C0021230360E8E700F08FFB089B0360E5E755
:10CD1C00A40000205CF60008F8B520F00043B3F145
:10CD2C007E5F044610D008DCB3F17C5F11DAB3F1FE
:10CD3C000C5F00F384809D48F8BD0146FCF740F879
:10CD4C000146FCF7FBF9F8BD002840F3CD8000202C
:10CD5C00F8BD0028C0F2CA8001464FF07E50FCF7A7
:10CD6C002FF84FF07C51FCF735F9044600F0CCF964
:10CD7C008F4906462046FCF72DF98E49FCF722F820
:10CD8C002146FCF727F98C49FCF71AF82146FCF7E9
:10CD9C0021F98A49FCF716F82146FCF71BF988495A
:10CDAC00FCF70EF82146FCF715F98649FCF70AF852
:10CDBC002146FCF70FF9844905462046FCF70AF991
:10CDCC008249FBF7FDFF2146FCF704F98049FBF78C
:10CDDC00F9FF2146FCF7FEF87E49FBF7F1FF2146EF
:10CDEC00FCF7F8F84FF07E51FBF7ECFF01462846B4
:10CDFC00FCF7A4F93146FCF7EDF826F47F6525F035
:10CE0C000F05074629462846FCF7E4F8014620465C
:10CE1C00FBF7D6FF294604463046FBF7D3FF014605
:10CE2C002046FCF78BF901463846FBF7CBFF014651
:10CE3C002846FBF7C7FF0146FBF7C4FFF8BD0146C8
:10CE4C00FCF7C8F805465A49FCF7C4F85949FBF7F2
:10CE5C00B9FF2946FCF7BEF85749FBF7B1FF294645
:10CE6C00FCF7B8F85549FBF7ADFF2946FCF7B2F8CB
:10CE7C005349FBF7A5FF2946FCF7ACF85149FBF7E2
:10CE8C00A1FF2946FCF7A6F84F4906462846FCF7B1
:10CE9C00A1F84E49FBF794FF2946FCF79BF84C4947
:10CEAC00FBF790FF2946FCF795F84A49FBF788FFFA
:10CEBC002946FCF78FF84FF07E51FBF783FF0146B4
:10CECC003046FCF73BF901462046FCF783F8014657
:10CEDC004148FBF775FF01462046FBF771FF014601
:10CEEC003E48FBF76DFFF8BD3D48F8BD4FF07E5155
:10CEFC00FBF768FF4FF07C51FCF76CF804462C49AB
:10CF0C00FCF768F82B49FBF75DFF2146FCF762F84C
:10CF1C002949FBF755FF2146FCF75CF82749FBF73D
:10CF2C0051FF2146FCF756F82549FBF749FF2146EE
:10CF3C00FCF750F82349FBF745FF2146FCF74AF86C
:10CF4C000646204600F0E0F81F4905462046FCF74F
:10CF5C0041F81E49FBF734FF2146FCF73BF81C490E
:10CF6C00FBF730FF2146FCF735F81A49FBF728FF91
:10CF7C002146FCF72FF84FF07E51FBF723FF0146BB
:10CF8C003046FCF7DBF82946FCF724F81249FBF78E
:10CF9C0017FF01462846FBF715FF0146FBF712FF6A
:10CFAC0001461048FBF70CFFF8BD00BFDB0FC93F73
:10CFBC0008EF1138047F4F3A4611243DA80A4E3E23
:10CFCC0090B0A63EABAA2A3E2EC69D3D6133303FA3
:10CFDC002D57014039D119406821A233DA0FC93FCE
:10CFEC00DB0F4940DA0F4940F8B521F00044B4F1A9
:10CFFC00FF4F034614DC20F00046B6F1FF4F074606
:10D00C000EDCB1F17E5F3AD08D1705F0020545EAD2
:10D01C00D07556B9022D30D0032D2BD13148F8BD27
:10D02C0008461946FBF7CEFEF8BDFCB1B4F1FF4F34
:10D03C0029D0B6F1FF4F19D0341BE4153C2C1ADC67
:10D04C00002938DB1846FCF779F800F0CFF900F02E
:10D05C00B7F8012D2CD0022D22D0002D2FD0224933
:10D06C00FBF7B0FE2149FBF7ABFEF8BD002F15DB3B
:10D07C001F48F8BDF8BD1E48EBE71C48F8BDBDE8DD
:10D08C00F84000F09DB8B6F1FF4F19D0022DF4D046
:10D09C00032DC3D0012D1BD00020F8BD1548F8BDC1
:10D0AC001149FBF78FFE01461048FBF789FEF8BDCE
:10D0BC0000F10040F8BD3C34C4DA0020C9E7F8BDEB
:10D0CC00022D0CD0032D08D0012D04D00A48F8BD38
:10D0DC004FF00040F8BD0948F8BD0948F8BD0948B3
:10D0EC00F8BD00BFDB0F49C02EBDBB33DB0F494081
:10D0FC00DB0FC93FDB0FC9BFDB0F493FDB0F49BF5C
:10D10C00E4CB16C0E4CB164020F00042B2F1FF4F46
:10D11C0070B5034604462DD25AB300283DDBB2F558
:10D12C00000F4FEAE0502CD3002631467F38C3F372
:10D13C001603C20743F4000348BF5B0040105B00BA
:10D14C0019244FF080728D189D4202DC5B1BA918CC
:10D15C001644013C4FEA43034FEA5202F3D113B198
:10D16C0006F001031E44761006F17C5606EBC05007
:10D17C0070BD70BD0146FBF72DFF2146FBF722FE6B
:10D18C0070BD14F400020FD15B00190202F1010210
:10D19C00FAD5C2F101021044C6E70146FBF710FEB6
:10D1AC000146FBF7CBFF70BD01221044BCE700BF6A
:10D1BC000020704700200149704700BF0000F87F35
:10D1CC002DE9F04120F00045B5F1A14F044606468B
:10D1DC0008DBB5F1FF4F6FDC002840F3A0806F48EF
:10D1EC00BDE8F0816E4B9D4277DCB5F1445F68DBA6
:10D1FC004FF0FF3721462046FBF7ECFE01468046F8
:10D20C00FBF7E8FE05466749FBF7E4FE6649FBF7CA
:10D21C00D9FD2946FBF7DEFE6449FBF7D3FD294611
:10D22C00FBF7D8FE6249FBF7CDFD2946FBF7D2FE92
:10D23C006049FBF7C7FD2946FBF7CCFE5E49FBF7BF
:10D24C00C1FD4146FBF7C6FE5C4980462846FBF70C
:10D25C00C1FE5B49FBF7B4FD2946FBF7BBFE594900
:10D26C00FBF7AEFD2946FBF7B5FE5749FBF7A8FDCA
:10D27C002946FBF7AFFE5549FBF7A2FD2946FBF704
:10D28C00A9FE7B1C014640464CD0FBF79BFD21467A
:10D29C00FBF7A0FE4E4B4F4D53F82710FBF790FDBC
:10D2AC002146FBF78DFD014655F82700FBF788FD5D
:10D2BC00002E30DBBDE8F0810146FBF783FDBDE8B5
:10D2CC00F0814549FBF77EFD4FF07E51FCF73EF8AF
:10D2DC0000288DD02046BDE8F08100F087F83F4B48
:10D2EC0004469D4229DCA3F5D0039D4244DC014653
:10D2FC00FBF768FD4FF07E51FBF762FD4FF080416C
:10D30C0005462046FBF75EFD01462846FBF716FF57
:10D31C00002704466EE700F10040BDE8F08130487C
:10D32C00BDE8F081FBF74EFD2146FBF753FE0146AD
:10D33C002046FBF745FDBDE8F0812A4B9D4214DCED
:10D34C004FF07F51FBF73CFD4FF07F5105462046D7
:10D35C00FBF740FE4FF07E51FBF734FD01462846AB
:10D36C00FBF7ECFE0227044644E701461E48FBF798
:10D37C00E5FE032704463DE74FF07E51FBF720FD09
:10D38C004FF07E5105462046FBF71CFD0146284612
:10D39C00FBF7D4FE012704462CE700BFDB0FC93F87
:10D3AC00FFFFDF3ED769853C59DA4B3D356B883D35
:10D3BC006E2EBA3D2549123EABAAAA3E21A215BD3E
:10D3CC006BF16E3D95879D3D388EE33DCDCC4C3E4B
:10D3DC0064F6000874F60008CAF24971FFFF973F23
:10D3EC00DB0FC9BFFFFF1B40000080BF20F00040D7
:10D3FC00704700BF30F0004001D102207047A0F50B
:10D40C000003B3F1FE4F01D204207047054B421EBE
:10D41C009A4201D803207047A0F1FF40B0FA80F087
:10D42C0040097047FEFF7F00014B1868704700BF32
:10D43C00A000002000000000000000000102030416
:10D44C0006070809001001400040100200100140BE
:10D45C00002010020010014000801002CCD4000803
:10D46C00C0D40008BED40008BCD400080000803F23
:10D47C00000080BF0000803F000080BF0000803FA4
:10D48C00000080BF000080BF0000803F0000803F94
:10D49C000000803F0000803F0000803F0000803F84
:10D4AC000000803F000080BF000080BF0800140215
:10D4BC00FFFFFFFF000106030D0307030C03FFFF33
:10D4CC0000020102020203020802090206030D0314
:10D4DC0007030C03FFFF000000540040000C014048
:10D4EC00400080001F200000000020000058004079
:10D4FC00000C014000040008212200000000400044
:10D50C0001000102000103000104000105000106F5
:10D51C0000010700010800010900010A00010B00CD
:10D52C00010C01030D00010E00010F0001100001A0
:10D53C00110001120001130001140001524F4C4C58
:10D54C003B50495443483B5941573B414C543B5049
:10D55C006F733B506F73523B4E6176523B4C45564A
:10D56C00454C3B4D41473B56454C3B0000000000B1
:10D57C00F5E500080000000001000000FAE50008D5
:10D58C00010000000200000001E60008020000009B
:10D59C00030000000AE6000803000000040000007D
:10D5AC0010E60008050000000500000015E6000864
:10D5BC0006000000060000001FE60008070000003F
:10D5CC000700000028E60008080000000800000022
:10D5DC0031E6000809000000090000003AE60008E6
:10D5EC000A0000000A00000044E600080B000000DE
:10D5FC000B0000004EE600080C0000000C000000C0
:10D60C0058E600080D0000000D00000060E6000860
:10D61C000E0000000E00000068E600080F0000007D
:10D62C000F00000070E60008100000001000000061
:10D63C0079E60008110000001100000080E60008E7
:10D64C0012000000120000008AE60008130000001F
:10D65C001300000092E60008140000001400000003
:10D66C009DE600081500000015000000A7E6000864
:10D67C001600000016000000AEE6000817000000BF
:10D68C0017000000B6E600081800000018000000A3
:10D69C00BEE600081900000019000000C6E60008EC
:10D6AC001A0000001A000000D0E600081B00000061
:10D6BC001B00000000000000FF000000EDE500086A
:10D6CC00E4E50008D8E500081EE9000825E9000893
:10D6DC002AE900083BE9000845E9000850E9000880
:10D6EC005BE9000866E900086AE9000873E90008CC
:10D6FC0079E9000883E9000891E9000894E9000839
:10D70C00A4E90008ABE90008B4E90008BEE9000888
:10D71C00C6E90008D1E90008DAE9000800000000B9
:10D72C0061687300000103030102000000000000A7
:10D73C0080250000004B00000096000000E1000076
:10D74C0000C201000084030090D00300010000001F
:10D75C002CD800080201000019D8000803020000B0
:10D76C0016D800080403000011D8000805040000B6
:10D77C000CD800080605000003D8000807060000B6
:10D78C0000D8000808070000FDD7000809080000B1
:10D79C00D80700200A090000FAD700080C0A00007C
:10D7AC00F5D700080D0B0000F0D700080E0C000098
:10D7BC00E1D700080F0D0000D80700200B0E000069
:10D7CC00DDD70008100F0000D8D7000800F50A05B7
:10D7DC00FF00640AFF0405040508050F050805048D
:10D7EC00050405FF140F2305FF05050505FF0A0AAF
:10D7FC00FF1932FF3202FF05050F0505050F1EFF4D
:10D80C001E050505FF0F050F05FF3232FF0A0A0A38
:10D81C000A0A28280A280A28280A0A0A0A0A46FF95
:10D82C00140A140A140AFF00000000000102030489
:10D83C0001020304060708090204060829750008FA
:10D84C00D774000891740008E3750008C1740008CF
:10D85C00DD75000827F500082AF5000832F50008E8
:10D86C003BF50008B8ED000844000000F409002066
:10D87C0000000000A00F0000C1ED000841000000F6
:10D88C00F70900200000000001000000D3ED0008A3
:10D89C0041000000F609002000000000010000001B
:10D8AC00E1ED000841000000F80900200000000034
:10D8BC0001000000EEED000844000000100B0020F9
:10D8CC00B0040000A4060000F5ED000844000000C0
:10D8DC00120B002000000000D0070000FFED000834
:10D8EC0044000000140B002000000000D0070000D2
:10D8FC0009EE0008420000000C0B002000000000A4
:10D90C001200000016EE0008410000000D0B002074
:10D91C0001000000FF00000021EE000842000000A2
:10D92C000E0B0020000000000100000031EE00088A
:10D93C00420000004E0B002000000000010000001F
:10D94C00E7F1000844000000BC0A002000000000C1
:10D95C00D007000046EE000844000000BE0A00207C
:10D96C0000000000D007000053EE00084400000047
:10D97C00C00A002000000000D00700005FEE000885
:10D98C0044000000C20A002000000000D007000084
:10D99C0072EE000844000000C40A002000000000E1
:10D9AC00D007000082EE000844000000C60A0020E8
:10D9BC0000000000D007000093EE000844000000B7
:10D9CC00C80A002000000000D00700009EEE0008EE
:10D9DC0044000000CA0A002000000000D00700002C
:10D9EC00B3EE000844000000CC0A00203200000016
:10D9FC00007D0000C2EE000844000000CE0A0020AA
:10DA0C0032000000F2010000D1EE000841000000DD
:10DA1C00580B00200000000001000000DEEE0008A2
:10DA2C0041000000590B0020000000000100000024
:10DA3C00F1EE0008410000005A0B0020000000002D
:10DA4C003C00000003EF0008410000005B0B0020CD
:10DA5C0000000000B40000000FEF000842000000BE
:10DA6C00600B0020FFFFFFFF0100000025EF000806
:10DA7C0041000000620B0020300000007E0000001E
:10DA8C0036EF0008410000000A0B002000000000E7
:10DA9C000600000048EF0008410000000B0B0020BE
:10DAAC00000000000A0000005AEF000841000000CE
:10DABC00740B002000000000010000006BEF000858
:10DACC0041000000750B0020000000000100000068
:10DADC007FEF000860000000780B0020A6FFFFFF1E
:10DAEC005A00000097EF0008600000007C0B00203B
:10DAFC004CFFFFFFB4000000AFEF00084100000036
:10DB0C00800B00200000000001000000C8EF00089E
:10DB1C0041000000810B002000000000010000000B
:10DB2C00D3EF000841000000820B00200000000031
:10DB3C0001000000E8EF000841000000830B00200A
:10DB4C00000000007800000002F000084400000013
:10DB5C00000B002000000000204E000013F0000815
:10DB6C0041000000F40A002000000000FF0000004B
:10DB7C001EF0000841000000F70A00200A00000017
:10DB8C003200000034F0000841000000F80A0020C8
:10DB9C000A000000320000004AF0000841000000BA
:10DBAC00F90A00200A0000003200000064F00008AE
:10DBBC0048000000FA0A0020F0D8FFFF10270000F0
:10DBCC0078F0000844000000FC0A0020000000006F
:10DBDC00E40C00008DF0000841000000FF0A00205A
:10DBEC000000000001000000ABF000084100000044
:10DBFC00FE0A00200000000002000000BEF0000839
:10DC0C0041000000D00A00200000000008000000C5
:10DC1C00C9F0000841000000D10A002000000000FB
:10DC2C0008000000D3F0000841000000D20A0020D8
:10DC3C000000000008000000DDF0000848000000B3
:10DC4C00D40A00204CFFFFFF68010000EEF0000832
:10DC5C0048000000D60A00204CFFFFFF68010000BE
:10DC6C0000F1000848000000D80A00204CFFFFFF1C
:10DC7C006801000010F1000844000000E60A0020D2
:10DC8C00640000008403000026F10008440000003A
:10DC9C00DC0A002000000000000100002FF1000849
:10DCAC0041000000E20A002000000000800000009B
:10DCBC003FF1000844000000DE0A00206400000070
:10DCCC00E803000050F1000844000000E00A0020C6
:10DCDC0064000000E803000062F10008810000000D
:10DCEC00970C002001000000FA00000074F10008FD
:10DCFC0081000000980C00200000000001000000D2
:10DD0C006BF1000881000000950C00200000000061
:10DD1C002000000089F1000881000000960C002012
:10DD2C00000000006400000096F100088100000073
:10DD3C009C0C00200000000096000000B0F10008D0
:10DD4C00840000009A0C00200100000084030000F5
:10DD5C00CAF1000842000000DA0A0020FFFFFFFFB2
:10DD6C0001000000E0F10008410000005C0B002005
:10DD7C000000000001000000F4F100084200000067
:10DD8C005D0B0020FFFFFFFF0100000008F2000800
:10DD9C00440000005E0B002050000000F401000065
:10DDAC0022F2000881000000D80B002000000000C7
:10DDBC000200000037F2000801010000DA0E00201A
:10DDCC0000000000FA0000003FF200080101000012
:10DDDC00DB0E0020000000006400000047F2000889
:10DDEC0001010000E20E00200000000064000000B1
:10DDFC0053F2000801010000DC0E002000000000BE
:10DE0C00640000005BF2000801010000DD0E002040
:10DE1C00000000006400000064F200080101000032
:10DE2C00DE0E002000000000640000006EF200080E
:10DE3C0001010000DF0E0020000000006400000063
:10DE4C0079F2000801010000E00E00200000000043
:10DE5C00FF00000082F2000801010000E10E00202A
:10DE6C0000000000640000008BF2000804010000B8
:10DE7C00E40E0020E8030000D00700009AF200082E
:10DE8C0041000000500B002000000000C800000002
:10DE9C00A9F2000841000000510B00200000000016
:10DEAC00C8000000BCF2000844000000520B002027
:10DEBC00E8030000D0070000CEF20008410000008B
:10DECC00540B00200000000001000000E3F20008E9
:10DEDC0044000000560B0020000000002C01000044
:10DEEC00FFF2000844000000160B0020EE020000B8
:10DEFC00CA0800000BF3000844000000180B0020B7
:10DF0C00EE020000CA08000017F3000841000000F0
:10DF1C00DB0A0020000000000900000024F30008C8
:10DF2C0081000000E00B002000000000FA0000005F
:10DF3C0033F3000881000000E80B00200000000013
:10DF4C006400000042F3000881000000E90B00208F
:10DF5C00000000006400000050F30008A000000066
:10DF6C00E40B0020010000001400000060F3000826
:10DF7C0081000000FC0B00200000000001000000EC
:10DF8C006FF3000888000000DE0B0020D4FEFFFFBA
:10DF9C002C0100007EF3000888000000DC0B002040
:10DFAC00D4FEFFFF2C0100008CF300088100000060
:10DFBC00EC0B002000000000300000009AF3000879
:10DFCC00A0000000F00B0020000000000100000089
:10DFDC00A9F30008A0000000F40B002000000000D2
:10DFEC0001000000B5F30008A0000000F80B0020B1
:10DFFC000000000001000000C1F300084100000017
:10E00C00E40A00200000000004000000CFF3000828
:10E01C0041000000E30A00200000000003000000A3
:10E02C00DCF3000888000000DA0B0020B0B9FFFF19
:10E03C0050460000ECF3000881000000840B002027
:10E04C000000000005000000FBF300088100000048
:10E05C00860B002000000000C800000003F400083C
:10E06C0081000000900B002000000000C8000000A0
:10E07C00F8F00008810000009A0B0020000000005E
:10E08C00C80000000BF4000881000000850B002084
:10E09C0000000000C800000012F40008810000001D
:10E0AC008F0B002000000000C8000000E7F0000803
:10E0BC0081000000990B002000000000C800000047
:10E0CC0019F4000881000000870B002000000000FC
:10E0DC00C80000001FF4000881000000910B002014
:10E0EC0000000000C80000000AF1000881000000D8
:10E0FC009B0B002000000000C800000025F4000865
:10E10C00A0000000A80B002000000000640000002C
:10E11C002EF40008A0000000B40B0020000000004A
:10E12C006400000037F40008A0000000C00B0020C1
:10E13C00000000006400000040F40008A000000093
:10E14C00A40B0020000000006400000048F400084C
:10E15C00A0000000B00B00200000000064000000D4
:10E16C0050F40008A0000000BC0B002000000000D0
:10E17C006400000058F40008A0000000AC0B002064
:10E18C0000000000640000005FF40008A000000024
:10E19C00B80B0020000000006400000066F40008CA
:10E1AC00A0000000C40B0020000000006400000070
:10E1BC006DF40008A0000000CC0B00200000000053
:10E1CC000A0000007BF40008A0000000C80B00202F
:10E1DC00000000000A00000087F400088100000025
:10E1EC00D00B002000000000FA0000009BF4000897
:10E1FC0081000000880B002000000000C800000017
:10E20C00A1F4000881000000920B00200000000027
:10E21C00C8000000A7F40008810000009C0B00203F
:10E22C0000000000C8000000ADF4000881000000F0
:10E23C008C0B002000000000C8000000B5F40008A2
:10E24C0081000000960B002000000000C8000000B8
:10E25C00BDF4000881000000A00B002000000000AD
:10E26C00C8000000C5F40008810000008E0B0020DF
:10E27C0000000000C8000000CBF400088100000082
:10E28C00980B002000000000C8000000D1F400082A
:10E29C0081000000A20B002000000000C80000005C
:10E2AC00D7F4000884000000D20B002064000000AA
:10E2BC00F4010000E3F4000881000000D60B0020FC
:10E2CC0000000000C8000000EFF40008810000000E
:10E2DC00D50B002000000000C8000000FCF4000872
:10E2EC0081000000D40B002000000000C8000000DA
:10E2FC0009F5000848000000EE0A00200080FFFF2E
:10E30C00FF7F000013F5000848000000F00A002011
:10E31C000080FFFFFF7F00001DF500084800000093
:10E32C00F20A00200080FFFFFF7F000086EB000850
:10E33C008FEB00080000000015400008ABEB000854
:10E34C00AFEB0008000000002B3E000876EB000845
:10E35C00BFEB000800000000D58C0008DCEB0008C7
:10E36C00E1EB0008F4EB00087D44000805EC000824
:10E37C000000000000000000613D00080AEC0008ED
:10E38C0012EC000825EC00085B3C000838EC000897
:10E39C003CEC000831EC0008998800084FEC0008B0
:10E3AC000000000000000000558C000854EC000830
:10E3BC0058EC000873EC0008B18B00087BEC0008EB
:10E3CC0080EC000800000000593C00089BEC0008A1
:10E3DC0093EC0008A1EC000849860008B3EC000897
:10E3EC0000000000BEEC000885850008D1EC000898
:10E3FC00CAEC0008D9EC000809860008E3EC000818
:10E40C00EFEC0008D9EC0008BD85000803ED00080E
:10E41C000BED000800000000293F000827ED000864
:10E42C002EED000800000000754100084CED0008BE
:10E43C0051ED000800000000F18C000861ED0008AF
:10E44C0068ED00080000000031430008BAE700083E
:10E45C007FED00088EED0008F1880008A4ED00089F
:10E46C009FED00080000000011880008B0ED0008C6
:10E47C00ABED000800000000878500080D1B5B4B0E
:10E48C00000D0A2320001B5B324A1B5B313B3148D9
:10E49C0000556E6B6E6F776E20636F6D6D616E6481
:10E4AC002C20747279202768656C7027000820086E
:10E4BC00000D0A456E746572696E6720434C4920E5
:10E4CC004D6F64652C2074797065202765786974AC
:10E4DC002720746F2072657475726E2C206F7220F9
:10E4EC002768656C70270D0A0000000000000040D2
:10E4FC00000801400100001C002800000000004042
:10E50C00000801400200041C00280000000000402C
:10E51C00000801400400081C002800000000004016
:10E52C000008014008000C1C0028000000040040FA
:10E53C00000801404000001D0028000000040040BD
:10E54C00000801408000041D002800000004004069
:10E55C00000C01400100081D0028000000040040D0
:10E56C00000C014002000C1D00280000002C014092
:10E57C00000801400001001B01280000002C014094
:10E58C000008014000080C1B012800000008004096
:10E59C00000C01404000001E002800000008004054
:10E5AC00000C01408000041E002800000008004000
:10E5BC00000C01400001081E00280000000800406B
:10E5CC00000C014000020C1E002800005365702056
:10E5DC00203720323031350030393A32353A313843
:10E5EC0000363262313165630041524D3B00414E81
:10E5FC00474C453B00484F52495A4F4E3B00424115
:10E60C00524F3B004D41473B004845414446524523
:10E61C00453B004845414441444A3B0043414D532E
:10E62C005441423B0043414D545249473B004750F3
:10E63C005320484F4D453B0047505320484F4C44C6
:10E64C003B0050415353544852553B0042454550B2
:10E65C0045523B004C45444D41583B004C45444CC5
:10E66C004F573B004C4C49474854533B0043414C9B
:10E67C0049423B00474F5645524E4F523B004F5379
:10E68C00442053573B0054454C454D455452593B3F
:10E69C00004155544F54554E453B00534F4E41523B
:10E6AC003B00534552564F313B00534552564F3267
:10E6BC003B00534552564F333B00424C41434B4277
:10E6CC004F583B004641494C534146453B00456E33
:10E6DC0061626C65643A2000257320006C69737468
:10E6EC0000417661696C61626C653A2000496E7616
:10E6FC00616C6964206E616D650D0A00756E6176E2
:10E70C0061696C61626C650D0A0044697361626CCD
:10E71C00656400456E61626C6564000D0A4C656150
:10E72C0076696E6720434C49206D6F64652C2075AB
:10E73C006E7361766564206368616E676573206CC7
:10E74C006F73742E0D0A00736574202573203D20A1
:10E75C000061757820257520257520257520257577
:10E76C002025750D0A002573206D75737420626564
:10E77C00206265747765656E20256420616E642067
:10E78C0025640D0A00696E646578005061727365CA
:10E79C00206572726F720D0A00727872616E676515
:10E7AC002025752025752025750D0A007265736569
:10E7BC00740061646A72616E676520257520257529
:10E7CC002025752025752025752025752025750D8E
:10E7DC000A0072786661696C2025752025632025F6
:10E7EC00640D0A0072786661696C202575202563BA
:10E7FC000D0A0073657269616C2025642025642004
:10E80C00256C6420256C6420256C6420256C640DBB
:10E81C000A006D6173746572007261746573000D2A
:10E82C000A232076657273696F6E0D0A000D0A2338
:10E83C002064756D70206D61737465720D0A000D26
:10E84C000A23206D697865720D0A000D0A0D0A23E2
:10E85C0020666561747572650D0A00666561747574
:10E86C007265202D25730D0A0066656174757265DD
:10E87C002025730D0A000D0A0D0A23206D61700D01
:10E88C000A006D61702025730D0A000D0A0D0A2314
:10E89C002073657269616C0D0A000D0A2320727871
:10E8AC006661696C0D0A000D0A232064756D702079
:10E8BC0070726F66696C650D0A000D0A2320707208
:10E8CC006F66696C650D0A000D0A23206175780D61
:10E8DC000A000D0A232061646A72616E67650D0A75
:10E8EC00000D0A2320727872616E67650D0A000DA7
:10E8FC000A232064756D702072617465730D0A00B3
:10E90C000D0A23207261746570726F66696C650DF7
:10E91C000A0052585F50504D005642415400494E27
:10E92C00464C494748545F4143435F43414C005276
:10E93C00585F53455249414C004D4F544F525F5311
:10E94C00544F5000534552564F5F54494C5400534A
:10E95C004F465453455249414C0047505300464191
:10E96C00494C5341464500534F4E41520054454C7F
:10E97C00454D455452590043555252454E545F4DE6
:10E98C00455445520033440052585F504152414C5B
:10E99C004C454C5F50574D0052585F4D53500052F0
:10E9AC005353495F414443004C45445F53545249CF
:10E9BC005000444953504C4159004F4E4553484F19
:10E9CC005431323500424C41434B424F580043487E
:10E9DC00414E4E454C5F464F5257415244494E476B
:10E9EC00002E00303132333435363738394142431A
:10E9FC004445464748494A4B4C4D4E4F5051525353
:10EA0C005455565758595A004145525431323334A3
:10EA1C003536373861626364656667680041455412
:10EA2C00523132333400232042657461466C69677D
:10EA3C0068742F2573202573202573202F202573B0
:10EA4C00202825732900434A4D435500312E31307F
:10EA5C002E30007261746570726F66696C6520256A
:10EA6C00640D0A006D6F746F722025643A20256462
:10EA7C000D0A002025642025640053797374656D9C
:10EA8C0020557074696D653A202564207365636F39
:10EA9C006E64732C20566F6C746167653A20256424
:10EAAC00202A20302E315620282564532062617490
:10EABC0074657279202D202573290D0A0043505559
:10EACC0020436C6F636B3D25644D487A004379633A
:10EADC006C652054696D653A2025642C20493243BD
:10EAEC00204572726F72733A2025642C20636F6E0E
:10EAFC006669672073697A653A2025640D0A0043BC
:10EB0C00757272656E742073657474696E67733A8E
:10EB1C00200D0A0025732073657420746F20005635
:10EB2C00616C75652061737369676E6D656E7420B9
:10EB3C006F7574206F662072616E67650D0A004DEB
:10EB4C0061703A2000202D202573000D0A092573D1
:10EB5C00000D0A5265626F6F74696E6700526573BF
:10EB6C00657474696E6720746F2064656661756C7A
:10EB7C00747300536176696E670061646A72616ECA
:10EB8C00676500636F6E6669677572652061646A9C
:10EB9C007573746D656E742072616E676573006158
:10EBAC00757800636F6E666967757265206D6F644A
:10EBBC00657300726573657420746F20646566619B
:10EBCC00756C747320616E64207265626F6F740073
:10EBDC0064756D700064756D7020636F6E66696727
:10EBEC0075726174696F6E005B6D61737465727CB4
:10EBFC0070726F66696C655D006578697400666536
:10EC0C00617475726500636F6E66696775726520F5
:10EC1C006665617475726573006C6973740D0A09AD
:10EC2C003C2B7C2D3E5B6E616D655D0067657400F1
:10EC3C00676574207661726961626C652076616CBF
:10EC4C0075650068656C70006D617000636F6E6651
:10EC5C006967757265207263206368616E6E656C9E
:10EC6C00206F72646572005B3C6D61703E5D006D7F
:10EC7C006D697800637573746F6D206D6F746F724E
:10EC8C00206D69786572006765742F736574206DEB
:10EC9C006F746F72003C696E6465783E205B3C76E5
:10ECAC00616C75653E5D00706C61795F736F756E3C
:10ECBC0064005B3C696E6465783E5D0D0A006368B8
:10ECCC00616E67652070726F66696C65005B3C698C
:10ECDC006E6465783E5D007261746570726F666912
:10ECEC006C65006368616E67652072617465207085
:10ECFC00726F66696C6500727872616E676500632D
:10ED0C006F6E666967757265207278206368616ED4
:10ED1C006E656C2072616E676573007278666169EE
:10ED2C006C0073686F772F7365742072782066613E
:10ED3C00696C736166652073657474696E677300C2
:10ED4C0073617665007361766520616E642072650F
:10ED5C00626F6F740073657269616C00636F6E66CD
:10ED6C0069677572652073657269616C20706F726A
:10ED7C007473006368616E67652073657474696E83
:10ED8C0067005B3C6E616D653E3D3C76616C756504
:10ED9C003E5D0073686F77207374617475730073D4
:10EDAC00686F772076657273696F6E006C6F6F7029
:10EDBC0074696D650073796E635F6779726F5F74E8
:10EDCC006F5F6C6F6F7000656D665F61766F696405
:10EDDC00616E63650072635F736D6F6F7468696EEB
:10EDEC0067006D69645F7263006D696E5F6368656F
:10EDFC00636B006D61785F636865636B007273733E
:10EE0C00695F6368616E6E656C00727373695F73C2
:10EE1C0063616C6500727373695F70706D5F696EAE
:10EE2C007665727400696E7075745F66696C746572
:10EE3C0072696E675F6D6F6465006D61785F746891
:10EE4C00726F74746C65006D696E5F636F6D6D616C
:10EE5C006E6400736572766F5F63656E7465725F66
:10EE6C0070756C73650033645F6465616462616EB8
:10EE7C00645F6C6F770033645F6465616462616EBC
:10EE8C00645F686967680033645F6E65757472618E
:10EE9C006C0033645F6465616462616E645F7468A6
:10EEAC00726F74746C65006D6F746F725F70776DD8
:10EEBC005F7261746500736572766F5F70776D5FFA
:10EECC00726174650072657461726465645F61720D
:10EEDC006D0064697361726D5F6B696C6C5F7377E5
:10EEEC0069746368006175746F5F64697361726DD6
:10EEFC005F64656C617900736D616C6C5F616E67EA
:10EF0C006C6500666978656477696E675F616C74BF
:10EF1C00686F6C645F646972007265626F6F745FB6
:10EF2C006368617261637465720073657269616CA8
:10EF3C0072785F70726F7669646572007370656B5E
:10EF4C007472756D5F7361745F62696E6400746571
:10EF5C006C656D657472795F73776974636800743E
:10EF6C00656C656D657472795F696E7665727369CF
:10EF7C006F6E006672736B795F64656661756C7435
:10EF8C005F6C6174746974756465006672736B7917
:10EF9C005F64656661756C745F6C6F6E67697475C0
:10EFAC006465006672736B795F636F6F7264696E10
:10EFBC00617465735F666F726D6174006672736BFA
:10EFCC00795F756E6974006672736B795F766661D2
:10EFDC00735F707265636973696F6E00686F7474C8
:10EFEC005F616C61726D5F736F756E645F696E7477
:10EFFC00657276616C00626174746572795F6361CD
:10F00C0070616369747900766261745F7363616CBB
:10F01C006500766261745F6D61785F63656C6C5FCF
:10F02C00766F6C7461676500766261745F6D696E92
:10F03C005F63656C6C5F766F6C746167650076629C
:10F04C0061745F7761726E696E675F63656C6C5F2C
:10F05C00766F6C746167650063757272656E745F50
:10F06C006D657465725F7363616C65006375727254
:10F07C00656E745F6D657465725F6F6666736574DB
:10F08C00006D756C74697769695F63757272656E12
:10F09C00745F6D657465725F6F7574707574006301
:10F0AC00757272656E745F6D657465725F7479707C
:10F0BC006500616C69676E5F6779726F00616C697E
:10F0CC00676E5F61636300616C69676E5F6D61673A
:10F0DC0000616C69676E5F626F6172645F726F6C06
:10F0EC006C00616C69676E5F626F6172645F7069FE
:10F0FC0074636800616C69676E5F626F6172645FF4
:10F10C00796177006D61785F616E676C655F696EC0
:10F11C00636C696E6174696F6E006779726F5F6C96
:10F12C007066006D6F726F6E5F7468726573686F76
:10F13C006C64006779726F5F636D70665F666163A4
:10F14C00746F72006779726F5F636D70666D5F6666
:10F15C006163746F7200616C745F686F6C645F6480
:10F16C0065616462616E6400616C745F686F6C648D
:10F17C005F666173745F6368616E67650079617760
:10F18C005F6465616462616E64007468726F74744C
:10F19C006C655F636F7272656374696F6E5F7661C5
:10F1AC006C7565007468726F74746C655F636F72F4
:10F1BC0072656374696F6E5F616E676C650079610F
:10F1CC00775F636F6E74726F6C5F64697265637482
:10F1DC00696F6E007069645F61745F6D696E5F74F6
:10F1EC0068726F74746C65007961775F6D6F746FA2
:10F1FC00725F646972656374696F6E007961775FC1
:10F20C006A756D705F70726576656E74696F6E5F2E
:10F21C006C696D69740064656661756C745F7261AC
:10F22C0074655F70726F66696C650072635F7261A2
:10F23C0074650072635F6578706F0072635F7961EB
:10F24C00775F6578706F007468725F6D69640074C5
:10F25C0068725F6578706F00726F6C6C5F7261744E
:10F26C00650070697463685F7261746500796177B9
:10F27C005F72617465007470615F726174650074B3
:10F28C0070615F627265616B706F696E740066614C
:10F29C00696C736166655F64656C61790066616950
:10F2AC006C736166655F6F66665F64656C6179003F
:10F2BC006661696C736166655F7468726F74746C97
:10F2CC0065006661696C736166655F6B696C6C5F28
:10F2DC00737769746368006661696C736166655FF6
:10F2EC007468726F74746C655F6C6F775F64656C57
:10F2FC0061790072785F6D696E5F7573656300721A
:10F30C00785F6D61785F75736563006163635F68D7
:10F31C0061726477617265006163635F6C70665FD4
:10F32C00666163746F720061636378795F646561B1
:10F33C006462616E64006163637A5F6465616462D8
:10F34C00616E64006163637A5F6C70665F63757491
:10F35C006F6666006163635F756E61726D65646391
:10F36C00616C006163635F7472696D5F7069746373
:10F37C0068006163635F7472696D5F726F6C6C00BF
:10F38C006261726F5F7461625F73697A650062615A
:10F39C00726F5F6E6F6973655F6C7066006261722D
:10F3AC006F5F63665F76656C006261726F5F636648
:10F3BC005F616C74006261726F5F68617264776127
:10F3CC007265006D61675F68617264776172650078
:10F3DC006D61675F6465636C696E6174696F6E0003
:10F3EC007069645F636F6E74726F6C6C65720070C1
:10F3FC005F706974636800695F706974636800703A
:10F40C005F726F6C6C00695F726F6C6C00705F790F
:10F41C00617700695F79617700705F706974636808
:10F42C006600695F70697463686600645F70697414
:10F43C0063686600705F726F6C6C6600695F726FF8
:10F44C006C6C6600645F726F6C6C6600705F7961E7
:10F45C00776600695F7961776600645F79617766CA
:10F46C00006C6576656C5F686F72697A6F6E006CA4
:10F47C006576656C5F616E676C650073656E73694C
:10F48C007469766974795F686F72697A6F6E0070EF
:10F49C005F616C7400695F616C7400645F616C74B3
:10F4AC0000705F6C6576656C00695F6C6576656C89
:10F4BC0000645F6C6576656C00705F76656C0069E6
:10F4CC005F76656C00645F76656C007961775F7060
:10F4DC005F6C696D6974006779726F5F6375745FD7
:10F4EC00687A00707465726D5F6375745F687A001A
:10F4FC00647465726D5F6375745F687A006D6167C3
:10F50C007A65726F5F78006D61677A65726F5F798B
:10F51C00006D61677A65726F5F7A004F4B005741DF
:10F52C00524E494E4700435249544943414C004EB8
:10F53C004F542050524553454E540000202020205B
:10F54C002020202020282828282820202020202087
:10F55C002020202020202020202020208810101067
:10F56C0010101010101010101010101004040404BF
:10F57C000404040404041010101010101041414134
:10F58C00414141010101010101010101010101019F
:10F59C000101010101010110101010101042424232
:10F5AC00424242020202020202020202020202026F
:10F5BC0002020202020202101010102000000000D1
:10F5CC00000000000000000000000000000000002F
:10F5DC00000000000000000000000000000000001F
:10F5EC00000000000000000000000000000000000F
:10F5FC0000000000000000000000000000000000FF
:10F60C0000000000000000000000000000000000EE
:10F61C0000000000000000000000000000000000DE
:10F62C0000000000000000000000000000000000CE
:10F63C000000000000000000000000000000004B73
:10F64C00000000CB61636F736600000000000000D7
:10F65C0073717274660000006937AC316821223313
:10F66C00B40F14336821A2333863ED3EDA0F493FEF
:08F67C005E987B3FDA0FC93FE5
:08F6840058A6FF7F0100000001
:10F68C000000803F000000000000000003000000AC
:10F69C000000803F0000803F0000803F010000011F
:10F6AC006157000800127A000100000000010101FE
:10F6BC00C17E00080300000000A24A0447F50008C0
:10F6CC00000000000000000000000000000000002E
:10F6DC00000000000000000000000000000000001E
:10F6EC00B2E900080000000000000000000000006B
:10F6FC0000000000000000000000000000000000FE
:10F70C0000000000000000000000000000000000ED
:10F71C0000000000000000000000000000000000DD
:08F72C00400000200100000074
:0400000508000000EF
:00000001FF
